:1000000000800020BD010000E1D8000099D8000068
:1000100099D8000099D8000099D8000099D800001C
:1000200099D8000099D8000099D80000E1D80000C4
:10003000E1D8000099D8000061CF000065D0000031
:10004000E1D80000E1D80000E1D80000E1D80000CC
:10005000E1D80000E1D80000E1D80000E1D80000BC
:10006000E1D80000E1D80000E1D80000E1D80000AC
:10007000E1D80000E1D80000E1D80000E1D800009C
:10008000E1D80000E1D80000E1D80000E1D800008C
:10009000E1D80000E1D80000E1D80000E1D800007C
:1000A0009DB40000A9B40000E1D80000E1D8000030
:1000B000E1D80000E1D80000E1D80000E1D800005C
:1000C000E1D80000E1D80000E1D80000E1D800004C
:1000D000E1D80000E1D80000E1D80000E1D800003C
:1000E000E1D80000E1D80000E1D80000E1D800002C
:1000F000E1D80000FDFC0000E1D80000CDE30000E5
:10010000E1D8000069E60000E1D80000E1D8000075
:10011000E1D80000E1D80000E1D80000E1D80000FB
:10012000E1D80000E1D80000E1D80000E1D80000EB
:10013000E1D80000E1D80000E1D80000E1D80000DB
:10014000E1D80000E1D80000E1D80000E1D80000CB
:1001500051D1000065D1000079D100008DD100009F
:10016000E1D8000085E90000E1D80000E1D80000F6
:10017000E1D80000E1D80000E1D80000E1D800009B
:10018000E1D80000E1D80000E1D80000E1D800008B
:10019000E1D80000E1D80000E1D80000E1D800007B
:1001A000E1D80000E1D80000E1D80000E1D800006B
:1001B000E1D80000E1D80000E1D80000564B4CF235
:1001C000205210B51A804DF628121A8000BF00BFC9
:1001D0000DF08AFB514B4FF010621A60504A9A6042
:1001E000504ADA60504A136813F4807304D14F49BF
:1001F0000B604FF4A85313604D4B1A78110703D5C9
:100200001A7842F008021A704A4B4B492A221A7097
:100210004A4A4B4B8B4204D252F8040F43F8040B6A
:10022000F8E7484B484900228B4202D243F8042B9E
:10023000FAE74649464A002352F8230041F82300D2
:1002400001336F2BF8D1434B434A802103F8011B44
:100250009342FBD1414B3D4A1A60414B8A221A70AE
:10026000A3F5805324225A70A0221A709A7992071B
:10027000FCD59A79D406FCD43A4A937903F00C035E
:10028000082B384BF9D103221A7140225A719A79FE
:100290009006FCD5334A9179324B4906FBD5324A58
:1002A000324911600221516020221A709A7902F0BD
:1002B0000C020C2AFAD12E4B2E4A1A602E4B2F4AD2
:1002C0001A6000225A60072243F8042C2C4AC3F813
:1002D0000C2D62B60DF0B8FE144B1B68DA0705D57D
:1002E00028480DF085FC284B284A1A60284B1B78BB
:1002F0005B0609D5244C254B22689A4204D121483B
:100300000DF076FC0023236010F0B2FF0DF0F2FA3E
:100310000DF020FAFEE700BF0E20054030800440BB
:10032000823F04000100002B10D0034014D0034092
:1003300002D0074000E007405C9CFF1FB44E010064
:100340004088FF1F5C9CFF1F84A4FF1F0082FF1FCB
:100350000000000000E400E05FE400E008ED00E0E1
:100360000050064000400640448004400000030165
:1003700004800440C010050014E000E0FF76010096
:100380000000202088CCD9601CE00340A5C3945A0B
:1003900000F00740FFFFFFFFFFFFFFFFFFFFFFFF32
:1003A000FFFFFFFFFFFFFFFFFFFFFFFFFFFFFFFF5D
:1003B000FFFFFFFFFFFFFFFFFFFFFFFFFFFFFFFF4D
:1003C000FFFFFFFFFFFFFFFFFFFFFFFFFFFFFFFF3D
:1003D000FFFFFFFFFFFFFFFFFFFFFFFFFFFFFFFF2D
:1003E000FFFFFFFFFFFFFFFFFFFFFFFFFFFFFFFF1D
:1003F000FFFFFFFFFFFFFFFFFFFFFFFFFFFFFFFF0D
:10040000FFFFFFFFFFFFFFFFFFFFFFFFDEF9FFFF23
:1004100010B5054C237833B9044B13B10448AFF33E
:1004200000800123237010BD5C9CFF1F00000000B2
:10043000B84E0100084B10B51BB108490848AFF38E
:1004400000800848036803B910BD074B002BFBD0A0
:10045000BDE81040184700BF00000000609CFF1F6F
:10046000B84E01005C9CFF1F0000000038B5044638
:10047000104621700A491D4610F0DCFC01464FF081
:100480007E5010F08BFD074910F0D4FCE5606060F1
:10049000256165610DF068FDE061204638BD00BF53
:1004A000DB0FC9400024744938B50446104621705A
:1004B00009491D4610F0BEFC01464FF07E5010F079
:1004C0006DFD064910F0B6FCE56060602561656170
:1004D0000DF04AFDE06138BDDB0FC94000247449CE
:1004E00038B503780446032B20D8DFE803F01A1848
:1004F0001002C168406910F093FB0D490546606821
:1005000010F04CFD0146284610F048FD38BD084962
:10051000406810F043FDE16810F08CFC38BDC06805
:1005200038BDC168406910F07BFB38BD002038BD84
:100530000024744970B504460E460DF015FD0546BD
:10054000E069281A10F022FCE3682361E561666126
:10055000A0610146606810F021FD0146A0601048CE
:1005600010F01CFD0FF0F2FF0FF092FC10F004FBF6
:10057000054601464FF07E5010F052FB616910F0C5
:1005800059FC21690646284610F054FC01463046C5
:1005900010F048FBE0602046BDE87040FFF7A0BFC8
:1005A000000080BF08B50E200CF0AEFF114B1B8879
:1005B000012B19D0104B1B88984213DB40F6FF71BA
:1005C0008842D4BFC3EB0001C3EB0101C1EB013191
:1005D000C3F57F630F33282091FBF3F1BDE808409A
:1005E0000DF018BB0021F3E70146BDE808401420D8
:1005F0000DF010BBB49EFF1F489DFF1F10B50446B1
:100600000CF084FD204610BD70B44C88A04220D967
:1006100001230133DBB21CB2660031F8144084427E
:100620001D46F6D3A04211D005F10045013D965B71
:1006300031F8151032F81530401AF21A00FB02F0AA
:10064000641A90FBF4F4E01870BC7047905B70BCC7
:10065000704702260125E5E700280CDA064A4342E6
:1006600082FB0320DA17C2EB600000EB4000A3EB33
:100670008000C0F10C007047ABAAAA2A38B5234B02
:100680001B78002B2CD015200CF03EFF204B18605F
:10069000204B1B88984203DA1F4C237863BB38BD7C
:1006A0001E4A1488A042A4EB0302A8BF20467F2A5A
:1006B0001CDDC01AC001541C90FBF4F4002CEBD0DC
:1006C000154B1A780AB901221A70154D2B689C42F5
:1006D00004D0144BE1B2187808F08AFF2C6038BDC2
:1006E00011200EF02DF80A4B1860D1E7C01AC0EBAC
:1006F000C01090FBF2F4E1E70A4B0021187808F0F3
:1007000077FF0023064A2370136038BD689EFF1FE1
:10071000889CFF1F029DFF1F409FFF1FE09EFF1F41
:10072000389FFF1FDC9CFF1F38B50F200EF008F824
:100730001B4A1C4B12881860C0F53B600830904281
:1007400020DB194B1B889842A3EB0204A8BF184674
:10075000801A7F2CC6BFC0010134C0EBC01090FBD3
:10076000F4F47CB1114B1A780AB901221A70104DB9
:100770002B689C4204D00F4BE1B2187808F038FF88
:100780002C6038BD094C237803B938BD094B0021D2
:10079000187808F02DFF0023054A2370136038BD38
:1007A0004C9DFF1FA09CFF1FCC9EFF1FF09EFF1FB4
:1007B0000C9DFF1FFA9CFF1FF0B40E8886420DD2DD
:1007C00003F10043013B31F81350854202D9F0BCDC
:1007D000FFF71ABF32F81300F0BC70471088F0BC66
:1007E000704700BF094B1B880C2B09D8084A80B200
:1007F00052F8232028B143F6FE73984203D9108C97
:100800007047108870470349FFF7FEBEB69CFF1F74
:10081000A4280100402A01004B4B4C4A2DE9F04727
:100820001E8814684A4BB442B3F80080494B33DB4E
:100830004445A8BF4446A6421C60C8BF00202DDD29
:10084000C6EB0807B7F5804F33DB80037B1C90FBBA
:10085000F3F0FFF7C7FF404A404B15881B88C0F3F1
:10086000C61909FB05F57F2D8246A8BF7F252BB34E
:10087000A64253DC4445D4BFC6EB0404C6EB0804CF
:100880009F42CCBF03FB04445C43354BC8BF0137D8
:1008900094FBF7F71F6013E034461E60C6EB0807B1
:1008A000A045D4BFC6EB0800C6EB0400B7F5804FE7
:1008B000CBDAC0EB803090FBF7F0CAE7284A136030
:1008C000284C2368994508D0274B1B88002B34D12E
:1008D000264B1B886BBBC4F80090254C23689A45B7
:1008E00006D0214B1B885A1F032A19D9C4F800A02F
:1008F000204C23689D420FD01F4B188848B11A4BDB
:100900001E4A1B88D35C834203D0C0B2E9B208F010
:100910006FFE2560BDE8F087BDE8F0870024AFE7F3
:10092000164AD05C2030C0B20AF07F0108F060FEA9
:10093000DCE7484608F0FCFECDE7104A4946D05CAB
:1009400008F056FEC4E700BF489DFF1FB09EFF1F82
:10095000129FFF1F809CFF1F909CFF1F929CFF1FF8
:10096000189FFF1FF49CFF1F969EFF1F3E9DFF1FB9
:10097000B09CFF1F409DFF1FA69EFF1FA489FF1F65
:100980002DE9F04F17208BB00DF0DAFEDFF850B3F1
:10099000CBF8000016200DF0D3FEB34BB34A1B88F2
:1009A00010600C2B00F00582B14A00211F2B117042
:1009B00037D0B04FB04B3A88B04E53F82250002396
:1009C0003370AF4BAF4A1B88AF491288013B012AF5
:1009D00031F91330059300F00682AC4B0193AC4B18
:1009E0000293DFF80083DFF8009300230093A94B04
:1009F0001B88012B00F04D82DFF8F0A2A64B039379
:100A0000DAF80040A54B04930023A54A1288013A66
:100A1000032A00F28682DFE812F00101DC001100F7
:100A20007101A04B934F1B783988934A934E52F82B
:100A30002150003318BF01233370C2E720460593CD
:100A400010F0A4F9984910F0F5F9059B04461846F2
:100A500010F09CF9954910F0EDF90146204610F090
:100A6000E1F810F0ADFB0446CAF80040D8F80000E9
:100A700010F08CF98C4910F0DDF98246009810F0E6
:100A800085F98A4910F0D6F90146504610F0CAF8A7
:100A900010F096FBC8F80000854A864BB2F800E0DB
:100AA0001988854BDBF800201B88DFF844C2CEEBA9
:100AB000040804EB0E0AC1EB000E08440499039CE1
:100AC000C1F800A00199C4F80080C1F800E00299C3
:100AD0009A420860BCF8001080F25281C3EB010C0E
:100AE000624865454FF0000E006880F256816C1C2C
:100AF00083420CF1010C0EFB04FE9EFBFCFE00F396
:100B000092838142A8BF0146C91A04FB01F191FBFF
:100B1000FCF19A4200F317818342C0F21481DFF89E
:100B2000D4A1DAF8000010F031F9644910F082F92C
:100B3000634910F077F810F043FBA0F5FF531C3B1E
:100B4000082B98BF4FF40050D9F80040DFF8A88177
:100B5000044443F6FF77BC42A8BF3C4624EAE47451
:100B60002046CAF8004010F011F98146307805FBA4
:100B700000F010F00BF94FF07A5110F05BF90146DC
:100B8000484610F04DF810F01BFB4E4BB842A8BF82
:100B900038461B7820EAE070C8F80000002B00F00F
:100BA000E380B4F5005F00F0DF8005F0B9FD464B4F
:100BB000D8F8000001221A70444C2368834205D003
:100BC00080B208F0E5FCD8F8003023600BB0BDE837
:100BD000F08F2046059310F0D9F83D4910F02AF91E
:100BE000059B0446184610F0D1F83A4910F022F956
:100BF0000146204610F016F810F0E2FA0446CAF852
:100C00000040D8F8000010F0C1F8314910F012F996
:100C10008246009810F0BAF82E4933E72046059333
:100C200010F0B4F82C4910F005F9059B044618465D
:100C300010F0ACF8294910F0FDF8014620460FF0FD
:100C4000F1FF10F0BDFA0446CAF80040D8F80000E1
:100C500010F09CF8204910F0EDF88246009810F052
:100C600095F81E490EE700BFE29EFF1FAC9CFF1FD8
:100C7000869CFF1FE89CFF1F6089FF1FC69EFF1F09
:100C80002089FF1FB69EFF1FE42C01003C9FFF1F21
:100C90001C9DFF1F449EFF1FD49EFF1F489EFF1FE9
:100CA0003489FF1F949EFF1FCDCC4C3FCDCC4C3ED2
:100CB000B089FF1F2C89FF1FAC9EFF1F9A99193F17
:100CC000CDCC4C45F29FFF1F3D9DFF1F2489FF1F88
:100CD0006666663FCDCCCC3D3333733FCDCC4C3DC7
:100CE000E49CFF1F789CFF1FEC9EFF1FD09EFF1F00
:100CF000C89CFF1F9889FF1F3089FF1F204605935E
:100D000010F044F8C54910F095F8059B04461846C4
:100D100010F03CF8C24910F08DF8014620460FF063
:100D200081FF10F04DFA0446CAF80040D8F80000E0
:100D300010F02CF8B94910F07DF88246009810F0B8
:100D400025F8B7499EE63B88002B3FF4E8AEC1EB9F
:100D50000E03002BB8BF5B42092B00F3E5804FF474
:100D60000050DFF808A3EFE6AE4C2378002B3FF4E9
:100D700023AF05F0D1FC0023D8F8000023701BE757
:100D8000C3EB010CA8488A42D4BFC3EB020EC3EBED
:100D9000010E65450068FFF6AAAE83420EFB05FE14
:100DA000C8BF00249EFBFCFE40F3348294FBFCF1A0
:100DB000AFE69E4B1B78002B00F0D5809C4F9D4BDF
:100DC00039889D4A53F821009C4E0121002311705F
:100DD00033700FF0DBFF4FF07C5110F02BF810F068
:100DE000EFF90546EDE5964B964A1B889649127831
:100DF000013B31F91340002A40F0B08011200DF082
:100E00009FFC0090914B0193D3F80090009B994573
:100E100040F3AC808E4BDFF858821B888D4A012B43
:100E2000D8F80030B2F800A08B4A02922846A3EB13
:100E3000040400F0CE800FF0A9FF029A52F82A10A5
:100E40000FF0F8FF014600200FF0EAFE10F0B8F9AD
:100E5000009BC9EB04029C42B8BF1C469042C9EB00
:100E6000040480F2CA8000FB0444013294FBF2F4D3
:100E70007A4BDFF800920293D9F80030234403EB59
:100E8000D3735B10C9F80030754B1B88012B7FF4BE
:100E9000B3AD744B03931C460F200DF051FC226838
:100EA00004929042034680F2E980694A1288012A3E
:100EB00000F02E81674A07901288674C06922846F8
:100EC0000FF064FF069ADFF8B0A154F82210DAF8A8
:100ED00000400FF0AFFF014600200FF0A1FE059B80
:100EE000E21A059210F06CF9059A079B04999A4250
:100EF000C1EB020EB8BF1A46704580F23381521A18
:100F000000FB02220EF1010192FBF1F2D9F8001070
:100F1000554804900A4402EBD2725210C9F80020DE
:100F200073E5D8F80000B7E50EF500500130401A1F
:100F30000FF02CFF3A49DFF834A10FF07BFF044695
:100F4000DAF800000FF022FF34490FF073FF01467A
:100F500020460FF067FE10F033F9F5E515200CF090
:100F6000D3FA00904EE7344A137022E53B4B0293CC
:100F7000D3F80090009B994544DA354BDFF8F080B8
:100F80001B88344A012BD8F80030B2F800A0324A4E
:100F9000039228461C4400F0EC800FF0F7FE039A01
:100FA00052F82A100FF046FF10F00AF9009B9C42FD
:100FB000C9EB0402A8BF1C46C9EB04049042BABFA7
:100FC00000FB04440132444394FBF2F4DFF8A490A4
:100FD00052E70FF0DBFE029A52F82A100FF02AFFB8
:100FE00010F0EEF8009BC9EB04029C42B8BF1C460F
:100FF0008242C9EB04043FF736AF00FB04F494FBD4
:10100000F2F435E7DFF86C90DFF86480D9F800304F
:1010100003EBD3735B10C9F80030E8E49A99193FE9
:10102000CDCCCC3E3D9DFF1FAC9CFF1F949EFF1F6F
:10103000E89CFF1F6089FF1F869CFF1FC69EFF1F45
:10104000B489FF1F689EFF1FF82901003C9FFF1F06
:10105000229DFF1FD09CFF1FFC2C01001C9DFF1F29
:10106000449EFF1FD49EFF1F489EFF1F9889FF1FAD
:10107000789CFF1FEC9EFF1FD09EFF1F6B4A0492BF
:1010800012680692904237DD694A1288012A00F000
:101090008E80684A09901188674A0891284607920D
:1010A0000FF074FE079A0899DFF890A152F821100A
:1010B000DAF800400FF0BEFE059B2344059310F0C4
:1010C0007FF80599099B069A9942C2EB010EA8BFC9
:1010D0001946704580F29080891A00FB01110EF1CB
:1010E000010291FBF2F2D9F800100A4402EBD2722D
:1010F0005210C9F8002088E4D9F80020DFF83CA19C
:1011000002EBD2725210DAF80040C9F800207CE4F9
:10111000484A08901188484A0791284606920FF0DD
:1011200035FE069A0799DFF814A152F82110DAF873
:1011300000400FF07FFE059BE11A059110F040F88A
:101140000599089B049A9942C2EB010EB8BF194653
:10115000704558DA891A00FB01110EF1010291FB6A
:10116000F2F2D3E60499521A00FB02F292FBFEF26D
:10117000CCE60FF00BFE039A52F82A100FF05AFE3D
:10118000014600200FF04CFD10F01AF8009A94422E
:10119000C9EB0403A8BF1446C9EB04049842BABFC4
:1011A00000FB04440133444394FBF3F40EE721496C
:1011B000214A089028460C8807920FF0E7FD079A0D
:1011C000DFF878A052F82410DAF800400FF032FE71
:1011D000014600200FF024FD059B234405930FF0EA
:1011E000EFFF0599089B069A9942C2EB010EA8BF32
:1011F00019467045FFF670AF069A891A00FB01F197
:1012000091FBFEF26FE7049A891A00FB01F191FB52
:10121000FEF27BE68842D4BFC3EB0004C3EB0104BB
:1012200005FB04F4C2E519466EE400BF489EFF1FAB
:10123000229DFF1FD09CFF1FFC2C0100D09EFF1F92
:1012400008B5244B1B88FBB1234B1B78FBB1234B08
:101250001B78E3B1224B1B78CBB1224B1B78B3B187
:10126000214B22481A78C2B9214A224900881288A3
:1012700009680244B1EB620F09DD01221A70642093
:10128000BDE8084005F060BA174A117801B908BDF9
:101290001370BDE8084008F01FBA154A16490088C7
:1012A000128809680244B1EB620FF0DD00221A7067
:1012B00008F012FA642005F047FA642005F044FAB9
:1012C000642005F041FA4FF41670BDE808400CF0B8
:1012D0006DBE00BF5A9EFF1F449FFF1F0C9FFF1F44
:1012E0000D9FFF1F0E9FFF1FB49CFF1FC89CFF1F79
:1012F000AC9EFF1FE49CFF1FAC9CFF1F38B5114C38
:10130000232025780CF000F90F4A42F82500131F1E
:1013100002F1C400002253F8041F83420A44FAD1A8
:1013200023780A4907480A4C0133DBB2322B81FB90
:10133000025108BF0023D217C2EB211203702260B2
:1013400038BD00BF949CFF1F589DFF1F1F85EB51A8
:10135000A89EFF1F2DE9F04FB74DB84E2868B84C36
:1013600083B00FF013FDB7490FF064FD074610205E
:101370000DF0E6F90FF00AFDB3490FF05BFD3946B9
:101380000FF050FC0FF01CFF318828608842238842
:101390007EDA1F4600225B1ADFF8D482DFF8D4E23F
:1013A0007F2BCABFD201C2EBC212013392FBF3F30F
:1013B000B8F80020CEF80030192A00F0DF801A2A91
:1013C00000F02B811E2A00F05B814FF00108C1461E
:1013D0009E4B1B88002B66D09D4A1288032A00F280
:1013E00009818842C0F25F81B842D4BFC1EB0000DE
:1013F000C1EB0700791A8B42B4BF03FB00005843CE
:10140000944F954BB8BF013190FBF1F018603888CC
:1014100000284FD03188D5F800E0884ADFF818A2BC
:10142000714500F38280DFF83CC29CF80030002B4D
:101430004CD14FF0010B04288CF800B046D1B8F124
:10144000000F40F0CB81854B1888F0B1B9F1000F47
:101450001BD02B68318822888B4280F29C8100232C
:10146000541A7E2C7E4DD5BFC3EB8313C3EBC3133D
:101470005B00013493FBF4F42B680134A34203D0E6
:10148000C0B2E1B208F0B4F82C6003B0BDE8F08F50
:101490009842D4BFC1EB0002C1EB03021F467AE7BA
:1014A00099464FF001081E2A00F0D281694F388812
:1014B0000028AFD1694B1B88002BABD1694A11784A
:1014C0000029E2D0137003B0BDE8F08F012800F0CE
:1014D0001281022800F003810328B4D1624B1B88DB
:1014E000092BB0D0B8F1000FADD02B683788228817
:1014F000BB4280F295810023D71B7E2FDFF86CB1B1
:10150000D5BFC3EB8313C3EBC3135B00013793FB5E
:10151000F7F7DBF800300137BB4203D0F9B24A20BD
:1015200008F066F8CBF800708DE74E4B1A78002A69
:10153000ABD0002401281C7000F0C280022840F0CB
:101540003181B8F1000F00F0C280484D2B68002BAC
:1015500000F0BD800420214608F04AF83F4B2C6083
:101560001888002891D0B9F1000F8ED0C0B20021A8
:1015700008F03EF83A4B00221A6086E7DFF8F8A040
:10158000DFF8F8909AF80030BBB1DFF8D0E0BEF891
:1015900000E0BEF1000F10D099F800C09C4500F0AB
:1015A00099805FFA8EF07F2108F022F89AF80030D7
:1015B000B8F8002089F800300FE099F800E09E4567
:1015C00000F08880254B0021187808F011F89AF86F
:1015D0000030B8F8002089F800301C4B1B88002B25
:1015E0003FF45EAF1E2A40F02B814FF001084FF010
:1015F000000951E0884258DBB842A1EB0701A8BFBF
:1016000038468B42A0EB070055DA03FB00004B1C69
:1016100090FBF3F3104A136048E7DFF85CA09AF8F8
:101620000030002B0BBF4FF001084FF000084FF0C7
:1016300000094FF00109CBE6D89CFF1F609EFF1FF9
:101640005C9EFF1F9A99193FCDCCCC3E1C9FFF1F7B
:10165000D89EFF1FE09CFF1F509DFF1FF49EFF1FA1
:10166000BC9CFF1FE99EFF1F969EFF1F549DFF1FFE
:10167000E29EFF1FC89EFF1F949EFF1F9A9CFF1FA4
:10168000DFF8E8A1744B9AF800801B88B8FA88F854
:101690004FEA58184FF000099AF8002042B3286822
:1016A0003188278898E60020A4E60846C91B8B42AB
:1016B000A0EB0700A9DB03FB00F393FBF1F3A9E721
:1016C000B8F1000F03D0654D2B68002B7FD1644B20
:1016D000188846E74FF001084FF0000978E6B8F1A6
:1016E000000F3FF4B0AEDFF874B1DBF8003030E04B
:1016F0005C4B1A60DAE6B8F1000F3FF4A4AEB4F820
:1017000000A0F245D4BFC1EB0A03C1EB0E03C1EB4D
:101710000A0ABAF17E0FDFF844B1D5BFC3EB8313D9
:10172000C3EBC3135B000AF1010A93FBFAFADBF87F
:1017300000300AF1010A534504D05FFA8AF1012012
:1017400007F056FF3888CBF800A002287FF4C4AE1B
:1017500053462A68B6F800A02188524559DA00227B
:10176000CAEB010ABAF17E0FD3BFC2EB8212C2EB01
:10177000C2120AF1010A520092FBFAFA0AF1010AB6
:101780009A4504D05FFA8AF1042007F031FF3888C7
:10179000CBF800A0A0E69342D4BFC1EB0303C1EB9A
:1017A00002035DE6032828D12F4B1B88092B8ED01E
:1017B000B8F1000F8BD0294D2B68002B87D04A2021
:1017C000214607F015FF264B2C601888C9E62146F4
:1017D00007F00EFF224B2C601888C2E640207F21C4
:1017E0008DE80C0007F004FF388858459DE80C0090
:1017F0001DD002287FF470AE75E704287FF467AF30
:10180000B8F1000F3FF463AF2146402007F0F0FE2F
:101810005DE78A42D4BFCAEB0202CAEB01029FE72E
:101820009342D4BFC7EB0303C7EB020364E6DAF8C5
:1018300000E01188B4F800A08E45FFF668AF60E7BD
:101840002868318827884FF001084FF00009C3E568
:101850000023DFF818A01FE71C9FFF1F549DFF1FE8
:10186000F49EFF1F509DFF1F969EFF1F949EFF1F1B
:1018700008B5114B1B88022B09D0052B07D0032B71
:1018800015D0042B0BD00D4B01221A7008BD7F21FF
:10189000412007F0ADFE094B01221A7008BD7F21DF
:1018A000092007F0A5FE054B01221A7008BD402152
:1018B000092007F09DFEE6E74E9DFF1F049DFF1FD8
:1018C00038B5074B074D1B88052B044606D02B68FF
:1018D000834203D0C1B2052007F08AFE2C6038BDD8
:1018E0004E9DFF1FF89EFF1F38B5124D124C2B88DE
:1018F000052B12D022684AB9022B0ED0033B012BD4
:1019000013D90E4A00231370236038BD002105202F
:1019100007F06EFE2B88022B04D10021412007F036
:1019200067FEEEE7052BE9D1F7E70021092007F074
:101930005FFEE6E74E9DFF1FF89EFF1F049DFF1F01
:10194000464B1B881D2B70B541D0454D0024454B9F
:101950001B88022B16D0444B1B88022B54D028889E
:10196000424B002C1B780ADB8442A8BF044634B1EA
:10197000002B3AD02046BDE87040FFF7A1BF002BF6
:101980002FD170BD3A4B1B78002B37D015200BF0B0
:10199000BBFD384B1860384A1288002ADBD0374A22
:1019A000186811888142D6DC354B2A881B8883420F
:1019B000A3EB0106A8BF03465B1AB242BABF02FB03
:1019C00003330136534393FBF6F31C44C3E72A4B1E
:1019D0001C888CB12B4B224D1C78002CB7D02C8846
:1019E000B5E7BDE87040FFF77FBFFFF741FF204636
:1019F000BDE87040FFF764BF194DA8E711200CF057
:101A00009FFE1C4B1860C6E70F200CF099FE1A4B86
:101A10001D4A1B881060002BA1D01C4AC0F53B63F7
:101A2000118808338B429ADB194A2888128893421E
:101A3000A2EB0105A8BF1346A842A3EB010306DAF7
:101A400000FB0333013593FBF5F31C4488E700FBEF
:101A500003F292FBF5F31C4482E700BFE29EFF1FF6
:101A6000E69EFF1FB69EFF1F449EFF1F049DFF1FA3
:101A7000689EFF1F889CFF1F4E9DFF1F029DFF1F3A
:101A8000E09EFF1F949EFF1FA09CFF1F4C9DFF1F09
:101A9000CC9EFF1F38B510200CF052FEC830B0F5B8
:101AA000FA7FC0F2EE80B0F57A6F0146A8BF4FF41E
:101AB0007A6101F51673B3F57A6FA8BF4FF47A63B4
:101AC0009BB289B28E4A8F4C11802220238007F06E
:101AD000E9FE21888C4D8D4C242007F0E3FE0E207A
:101AE0000BF012FD40F6FF71C8308842A8BF0846CF
:101AF00020EAE07000F2DC5283B28A42A8BF0A46B4
:101B00000220194622802B8007F0CCFE2188042079
:101B100007F0C8FE17200CF013FE044616200CF048
:101B20000FFEA042B8BF204600F1C801B1F5FA7F10
:101B3000C0F2A280B1F57A6FA8BF4FF47A6101F5C7
:101B40004873B3F57A6FA8BF4FF47A639BB289B23A
:101B50006F4A704C11800A20238007F0A3FE218871
:101B60000C2007F09FFE0F200CF0EAFDC0F53F614E
:101B70000431B1F5AF6F7CDBB1F5FA6FA8BF4FF45C
:101B8000FA6189B2644BC0F54360B0F5AF6F19805C
:101B90006CDBB0F5FA6FA8BF4FF4FA6083B25F4C0C
:101BA000A420238007F07EFEA620218807F07AFE7D
:101BB0000B200CF0C5F9002868D011200CF0C0FDF6
:101BC00000F1C801B1F52F7F6EDA40F214534FF4E3
:101BD0002F71534A1180534C0620238007F062FE78
:101BE0002188082007F05EFE00244FF4AF75E1B2B3
:101BF0004D4809F0C7FC01348542A8BF05460C2CAE
:101C0000F5D101200CF09CFD044600200CF098FD5D
:101C1000323CA0F1320345496FF4957000FB03F3A9
:101C200000FB04F081FB034281FB0041DB17C0177E
:101C3000C3EB6223C0EB612003F5AF7200F5AF7315
:101C40009342A8BF13469D42A8BF1D46A5F11401AB
:101C5000312938DC40F26C7332213548354A018035
:101C600013602A20BDE8384007F01CBE4FF4AF6374
:101C700095E74FF4AF6185E740F214534FF4FA71E2
:101C800066E740F24C434FF4FA711BE715200BF066
:101C90003BFC00F59671B1F52F7F96DB41F25C239A
:101CA00099421FDD194694E741F25C239942F9DC21
:101CB0001B4A00F5487089B2B0F52F7F118019DA00
:101CC0004FF42F7387E740F23A72A5F5B9751A4BB6
:101CD00002FB05F583FB0523ED17A5EB631389B222
:101CE0003233BAE70E4A00F5617089B2B0F52F7F42
:101CF0001180E5DB8342A8BF03469BB26BE700BFC0
:101D0000609EFF1F5C9EFF1F489DFF1F129FFF1FCD
:101D1000AC9EFF1FC89CFF1F4C9DFF1FCC9EFF1F4A
:101D2000029DFF1FE09EFF1F3C9DFF1F67BBCF462C
:101D30000A9FFF1FA089FF1FB5814E1B2DE9F84F99
:101D40000C200BF0ADFB0C200CF062F8C149DFF861
:101D50008CA314200CF06CF8BF49C04809F0A4F81B
:101D6000022103200CF0FAF8022104200CF0F6F80E
:101D7000022105200CF0F2F8022106200CF0EEF80A
:101D800001210A200CF0EAF8012109200CF0E6F804
:101D900001210D200CF0E2F8012128200CF0DEF8E2
:101DA000012114200CF0DAF802210B200CF0D6F8F7
:101DB00001210C200CF0D2F800210C200CF0BAF814
:101DC000012121200CF0CAF802211C200CF0C6F8D9
:101DD00001211B200CF0C2F800211B200CF0AAF8F6
:101DE0001C200CF0ADF8B0FA80F35B091A208AF8D9
:101DF00000300CF049FA1F2000210CF00BFA0420EF
:101E00000CF09EF8002800F0EA8005200CF098F80D
:101E1000002800F017810023914C062023700CF05D
:101E20008FF8B0FA80F35B094FF0000B8D4A137006
:101E300006F0B6F82378002B40F0CD80584607F026
:101E40005BFD894B894A1B8889491488894D8A48DA
:101E500040F23A72A3F5AF7302FB03F381FB031266
:101E6000DB17A3EB621332332B60844B5A211C70B7
:101E700009F0C4FB002800F03781814A81481268CC
:101E8000DFF85C9200230121FEF70EFB0B200CF023
:101E900057F8011E0CBF0123002389F8003000F021
:101EA000B780794F794D7A4EDFF8388200233B6056
:101EB0002B60336004240F200CF042FC3368034491
:101EC0000E2033600BF020FB3B6899F8002018448B
:101ED0003860002A78D015200BF016FB2B681844C8
:101EE000286004F0010080F0010004F01DFCB8F847
:101EF0000030002B14BF4B20DC200CF057F8013CC5
:101F0000D9D133683968604A2868624F002BB8BF5E
:101F100003330029B8BF0331891011605E495F4A5D
:101F2000098814889B1000283360B8BF03305C4ECA
:101F30008210581A19442A6031603860594D5A4845
:101F40005A49161B22442E6002600B60BBF1000F41
:101F500062D1B8F80030002B4DD0554B012404203D
:101F60001C600BF0EDFF18B9524B444A1C70107006
:101F7000514B1B881C2B56D0504C04F1C805232014
:101F80000BF0C2FA44F8040F01200CF00FF8AC4239
:101F9000F5D19AF800301BB1494B1B78002B4CD17E
:101FA000002121200BF0C6FF464A474B10781870DD
:101FB00007F0AAFA04F0B0FB45F6BF524349444883
:101FC000BDE8F84F0BF058B811200CF0B9FB2B68A6
:101FD0001844286085E7BDE8F84F08F075BE062074
:101FE0000BF0AEFF00287FF410AF1D4C03462070AD
:101FF0004FF0010B1AE74FF4FA7004F0A5FB04F060
:102000008FFB06F021FB4FF4AF600BF0CFFFA4E78E
:1020100011200BF0A3FF44E7FFF73CFDB8F80030B8
:10202000002B9AD1E7E72B4B18880028A4D02A4B25
:10203000C0B2197807F0DCFA9EE7012121200BF0ED
:1020400079FFB1E703200BF07BFFB0FA80F35B0967
:10205000E2E600BF001B374640420F006491FF1FBD
:10206000BA9CFF1F4C9EFF1F0A9FFF1FE49EFF1F8D
:10207000B5814E1BA089FF1F3C9DFF1F189DFF1FB0
:102080002889FF1F749EFF1F8C9CFF1F789CFF1FD9
:10209000D09EFF1FD49EFF1FB089FF1F2C89FF1FFA
:1020A000489EFF1F3C9FFF1F1C9DFF1F249FFF1F7B
:1020B000DC9EFF1FA49CFF1FE29EFF1F549DFF1F7D
:1020C000629EFF1F649EFF1F429EFF1FA50500002A
:1020D000009FFF1F209DFF1FD49CFF1F469EFF1FD8
:1020E000689EFF1FA29EFF1F03200BF029FF002800
:1020F000FAD104200BF024FF0028F5D105200BF0C5
:102100001FFF0028F0D106200BF01AFF0028EBD1AA
:102110000CF036FC2DE9F04F89B005ADA14F2C46EF
:1021200008AE611BC9B2A04809F02CFA3B88834273
:1021300094BF0020012004F8010BA642F1D19B4876
:102140009B4A9DF814E09B4980F800E09DF816003A
:10215000994D10709DF818209DF81C30974E984CA2
:102160000A709DF81A10297000253370257073B914
:10217000002940F00F81934F1AB13B78002B40F0BB
:102180001F82002800F0F2810222227005E0002A5E
:1021900040F0B08005228B4F22708B4BDFF8889285
:1021A0009DF815109DF81900DFF880A2DFF880B2C5
:1021B000864DDFF88082864E3A709DF81EE01970D9
:1021C0009DF81F209DF81D109DF817C09DF81B70ED
:1021D00089F80000012000938BF800E088F80010D7
:1021E00032708AF800C02F700CF0AAFA79497A4A46
:1021F000D1F800E0009B7045CCBF01210021117097
:102200007CDD764A1288182A78D875490F880C3AEE
:10221000002F78D1734993F800C00B7899F800909B
:102220009AF800109BF8007095F800B02478A3EBA2
:102230004C03A9EB890A5B1A5344C7EB877AC7EBB7
:102240008A07DFF8A8A11F4498F80030BAF800A068
:1022500007EB4B0796F800B03B440BFB0A33624F89
:102260004FF00C0A1AFB043AC7F800A0B9F1000FAE
:102270000BD033784BB15D4B1B88042B0CBF0AF19C
:10228000020A0AF1040AC7F800A0594B594CDFF8BA
:10229000A8B11B882488DBF800B0574F574E3F8801
:1022A0003688033BC4EBC4045C4403EB4303DFF810
:1022B0008CB10AEB83033B44DBF800B0504FC6EB14
:1022C000C60657F824404F4F5E440C3B134457F862
:1022D00026601A193244BCF1000F27D02B782BB39B
:1022E00000295BD1B9FA89F9474B4FEA591983F8AC
:1022F000009023E006222270324F4EE738490F88C3
:102300000022002F86D0012F00F0CF80022F00F096
:10231000FB80032F00F09480334F9AF8001093F85D
:1023200000C099F80090D7F800A09FE7364B002432
:102330001C7011B198F8003023BB0021334B70455D
:102340001970C8BF324B3349C8BFC3F800A00B682F
:102350009A4213D0304B314C186803900398206098
:102360001B6804932E4C049B24880A601B1AA3420A
:1023700084BF2C4B1A6009B0BDE8F08F2748264B6C
:102380000068EDE7BCF1000FD7D1B9F1000FD4D14F
:102390000121D3E7042222700A4FFEE61A4B0021E6
:1023A0001970CAE70A9FFF1F3C9DFF1F0C9FFF1F6C
:1023B0000D9FFF1F0E9FFF1F0F9FFF1F109FFF1FEF
:1023C0004E9EFF1F5E9EFF1F419FFF1F459FFF1FE9
:1023D000E89EFF1FA089FF1F949EFF1FE29EFF1F24
:1023E000849CFF1FB289FF1F9C9EFF1FF09CFF1F54
:1023F000BA9EFF1FD89EFF1F969CFF1F069DFF1FC2
:10240000882A0100402501001E9FFF1F1F9FFF1FFC
:10241000289FFF1FFC9CFF1F30A0FF1FEC9CFF1F8D
:10242000F29EFF1F309FFF1F439FFF1F429FFF1F12
:10243000449FFF1F469FFF1F509DFF1F189FFF1FB8
:10244000664993F800C00B7899F800909AF800104C
:102450009BF8007094F800A02C78A3EB4C03A9EB38
:10246000890B5B1A5B444FF0050B1BFB0733009392
:1024700098F800300193009BDFF86CB1C7EBC707F9
:10248000BA440533019FBBF800B003EB4403347832
:102490003B4404FB0B33524C524F54F82A400C334C
:1024A00003EB040AC7F800A0E0E64C4993F800C02B
:1024B0000B7899F800909AF800109BF8007095F846
:1024C00000A02478A3EB4C03A9EB890B5B1A5B44B7
:1024D000C7EB877BC7EB8B07DFF80CB13B4498F861
:1024E0000070BBF800B003EB4A0A3378BA44C4F179
:1024F000060403FB0BA3E4B24FF00C0A394F1AFB9E
:10250000043AC7F800A0B1E6344993F800C00B784C
:1025100001932B780093019B9AF8001099F8009092
:102520009BF800A02478A3EB4C03A9EB890B5B1A62
:102530005B44A3F1020B2C4BCAEBCA0A54441B8820
:10254000DFF8C8A00193BDF800305AF824A098F82D
:10255000004017FB03BB3778019B5C4407FB034338
:102560001833204F9A44C7F800A07FE6BEF1000F51
:1025700029D13A78012A2FD91C4B22701B882BB302
:102580001B4B1B88013B9BB2062B1FD8194B1B789A
:10259000E3B1194B1B68012B7FF4FFAD1749184BB2
:1025A0000968184D83FB0130CB17C3EB600303EBC5
:1025B0004303A1EB83032B80134B03211970ECE53C
:1025C00003222270E9E501222270E6E50A4B1B682E
:1025D000012B7FF4E2ADEFE77246DEE5B289FF1F23
:1025E000442E01009C9EFF1FF09CFF1FC49EFF1FF6
:1025F000669EFF1F4A9DFF1FDC9EFF1F309FFF1F2F
:10260000ABAAAA2AA09EFF1F9489FF1FAC2C010031
:102610002DE9F04F3A4B1B788BB0002B6BD10E207D
:102620000AF072FF0EF0B2FB01463648364E374DC7
:10263000FDF780FF3348FDF753FF0EF0C1FD80F337
:102640000C003060FFF766FD2C68012C7AD0022C5C
:1026500000F0D182032C00F037842D4E2D4C3368CE
:102660002D4A2E4E0993099B316812882360591A0E
:10267000013A9142274F00F2B982294E32689A1AE4
:10268000092A00F2A282274E32689A1A0D2A00F215
:102690009782254E32689A1A252A1AD9234B1B880D
:1026A000002B40F06481224B1B78002B40F05F81AF
:1026B000FEF724FE1F4B1B881B3B9BB2022B04D84A
:1026C0001D4B1B78002B40F0558104F04FF8236818
:1026D00033601A4D2A689B1A502B00F21982184B4E
:1026E0001B88012B00F0318206F006FF06F0EAFDA0
:1026F0000BB0BDE8F08F08F06FF90BB0BDE8F08FBC
:10270000BA9CFF1F749EFF1FB09EFF1FDC9EFF1F21
:1027100030A0FF1F709EFF1F9C89FF1F449DFF1F5D
:10272000309DFF1F109DFF1F149DFF1F5A9EFF1F0E
:10273000B49CFF1FE29EFF1F949EFF1F549EFF1F2D
:10274000B49EFF1FDFF83893A44AB9F8000013784D
:10275000834204D0C3B21846137006F0BFFEDFF800
:102760001C839F4AB8F800301178994204D09D4FDD
:102770003978002940F066879B4A336812889B4E5F
:102780009A42C0F201819A4A1278002A40F0FC80F5
:10279000DFF8F0A2BAF8003023B9964B1B88002B63
:1027A00000F07685944A954B11881B88944A0B4417
:1027B00012685B109342934A126880F218850021D8
:1027C0009342B4BF01230B4604910093ACBF4FF07A
:1027D000010B8B4605910E200AF096FE8A4B8B4A20
:1027E0001B68176803930133A7F25232002B84460B
:1027F000029240F33887802BA8BF8023844A854902
:1028000012780191002A00F0C9800978914200F005
:10281000C580B8F80010DFF864E2994201F0238126
:102820007049AEF800307C4B4FF0010E81F800E0AB
:102830001978DFF854E2019B8EF800101A70009BA3
:10284000002B00F02381BAF80030002B00F01E812D
:10285000724B1B685A1C002A40F30987802A00F338
:1028600005876F4C6F4970482488098800682144A7
:10287000B0EB610FC1F26883A3F148020F2A02D8BE
:10288000473BA9F800300E200AF03EFE6FF4547367
:102890001F44874202DC654B00221A7000200BF0B7
:1028A0004FFF634A634B1168634C1B888842D4BF57
:1028B000002201222270002B00F08F845F4B1C78D5
:1028C000944243D0884241DD5D490C78002C00F0F1
:1028D00092875C4991F800C0BCF1000F40F08987F5
:1028E000594F0097594F5A480297574F007887F829
:1028F00000C0564F4FF0010E87F800C081F800E08D
:10290000002841F0008153490978002901F05480E2
:10291000514903910C460978002941F04A804F48FB
:102920004A4F0078397001210297217070B14648F2
:10293000444900904A480327077000200870009916
:10294000029F0870039901243C7008701A70454B6F
:102950001B88A3F11B02012A40F238861D2B7FF44D
:102960007DAE3E4A404B12781A70404C77E6FEF737
:1029700067FC9DE63E4B1B78002B3FF4A6AE2B6810
:10298000012B7FF4A2AEA2E631683A4A069106987E
:102990003949106002220B602A60F9E61E49DFF80F
:1029A000E8E0097800293FF446AF9EF80000814234
:1029B0003FF441AF03984B2841F31C801833802B20
:1029C000B8F80000A8BF802398423FF434AF2B48EA
:1029D00003800448012303702DE700BF429EFF1FC0
:1029E000189DFF1FA49CFF1F489DFF1F30A0FF1FC5
:1029F000B49CFF1F369DFF1FC89CFF1FAC9EFF1F8E
:102A0000E49CFF1FAC9CFF1F289FFF1F8C9CFF1F97
:102A10001E9FFF1FF89CFF1F1F9FFF1F9C9EFF1FF5
:102A2000609EFF1F5C9EFF1FD89CFF1F4D9EFF1FD7
:102A3000A089FF1F669EFF1FCE9CFF1F7C9CFF1F6F
:102A4000449FFF1FA49EFF1FF69EFF1F4A9DFF1F6E
:102A5000459FFF1F419FFF1F7D9CFF1F949EFF1FEF
:102A60009489FF1FE29EFF1F9A9CFF1F709EFF1F0D
:102A7000E89EFF1F089DFF1F6C9EFF1FE49EFF1F27
:102A8000649EFF1F009DFF1FF99CFF1F029B9C453A
:102A9000BFF6F9AE954B1B88002B3FF4F4AEBBF1AB
:102AA000000F7FF4D5AE924B1B881BB1059B002B0A
:102AB0007FF4CEAE049B002B3FF4E5AE8D4B1A782D
:102AC000002A7FF4E0AEDFF8B09299F800400122CE
:102AD0001A70002C40F0A983874B1B78002B02F062
:102AE000CC80864B1B78002B02F0A083844B1B7894
:102AF000002B7FF4C8AE834B1B78002B3FF4C3AE92
:102B0000B8F8003080490A3BA8F800300A70BAE6ED
:102B100005F08EFA7D4B1B7873B97D4B1B785BB942
:102B20007C4B1B7843B97C4B1B782BB97B4B1B78B8
:102B300013B903F0F1FD01E003F0FAFD23682B6007
:102B4000774B1B88012B7FF4CFAD764B764A196803
:102B50001778764EA92303FB01F10029744BB8BF07
:102B600001F57F511868734BB8BF3F3189132A2292
:102B70005439183802FB00111D786FF0140202FB63
:102B8000071232606C49002D00F04E810B689A42AA
:102B900000F3C08380F24881684D2878002840F017
:102BA0009F8767480568D5F17F0548BF0335AD109D
:102BB00001355B1B9A4200F337810B601A4634E102
:102BC000FEF7BEFE2368336063E5FDF7D9FEFEF72E
:102BD000C1FB5C4B1B88032B00F069855A4B1B889B
:102BE000032B00F06085236833604CE5FDF714FE8D
:102BF0003B68336041E5554A34681288A24204DBE1
:102C0000464B1B78002B00F0B583514E514833687A
:102C10000793514B079900681B88091A994200F2E3
:102C2000B180002B00F0AE804C4B198800293FF496
:102C300015AD4B4B4B481B680088A342B8BF2346D9
:102C40009A4241F37A81484B1A60DFF8308188F864
:102C50000010374FFDF7E0FD38687F2840F3C58549
:102C6000424B7F3883FB0032C317C3EB620303EB95
:102C70004303A0EB830073303D4B01931B88386006
:102C8000002B40F0E986234B00931B78002B00F0CB
:102C90001E84384C2378002B00F01984DFF8E09074
:102CA000DFF8C8A04FF0000B0CE003F17300C0B2D6
:102CB00098F8001006F0CCFC23780BF1010B5B4573
:102CC00040F305843B6859F8040F1844A0F17F03D2
:102CD0008AFB0321DA17C2EB610202EB42027F2872
:102CE000A3EB8203E1DCFDF7B7FCE0E7369DFF1FB5
:102CF0006A9EFF1F4D9EFF1F419FFF1F429FFF1FA8
:102D0000439FFF1F449FFF1FA49CFF1F4A9DFF1F5F
:102D1000A49EFF1FF69EFF1F7D9CFF1FB49CFF1FFC
:102D2000B49EFF1F9889FF1FC69EFF1F289DFF1F8F
:102D3000309FFF1F049DFF1F389DFF1FFC9EFF1F3C
:102D4000F89EFF1FB69EFF1F449EFF1F489DFF1F5A
:102D500030A0FF1F089DFF1F349DFF1F9C9CFF1F7D
:102D60006C9EFF1F129FFF1F809CFF1FABAAAA2A09
:102D7000DE9CFF1F5C89FF1F4E9EFF1F249DFF1FCF
:102D80003489FF1F7E4B7F491B6808887E49A34218
:102D9000B8BF23469A4200F3D4827C4C0988834210
:102DA000A8BF0346236000297FF44FAF9A42C8BFF3
:102DB0000B4640F3CD82801AB0F5804FAABF9B032B
:102DC000C3EB8333013093FBF0F0FDF70BFDC0F351
:102DD000C6100DF0DBFF6E4B044618880DF0D6FFD1
:102DE0006C49074620460EF025F8014638460EF09D
:102DF00021F821460DF016FF4FF07E5104460EF0EB
:102E0000B7F9002841F07D80634920460EF0CEF9E5
:102E1000002840F0728620460EF0F8F9C0B2DFF8C4
:102E2000BC8188F8000014E70A605C4B188858B32E
:102E30005B4B256853F82040B5FBF4F3772C04FB7B
:102E4000135300F32982C3EBC30303EB031393FB78
:102E5000F4F35448544C50F823002468534BA0F228
:102E6000FF7004FB00F000F57D3000F5607000EBB2
:102E70004004C0EBC40083FB00430344C017C0EB15
:102E8000A3400B3802440A6049494A4B0888198814
:102E900000F27C704300B3F57C6FA1F164014FEA4E
:102EA0004100B5BF4449454903FB02225A4381FB17
:102EB00002311144D317C3EBE123C11881F30C0194
:102EC00028200AF0A7FE0FE43D4BD6F800801988B1
:102ED000414540F387803B4B1B78002B40F08280BC
:102EE000DFF8FC9099F800007F2840F3F585A3F106
:102EF00055337F3803F1004383FB0032C317C3EB24
:102F0000620303EB4303A0EB830073302E4B01936A
:102F10001B88C0B289F80000002B40F0EE872B4BD5
:102F200000931B78002B00F09384294C2378002B0E
:102F300000F08E84274FDFF8A0804FF0000A0AE0EF
:102F400003F17300C0B206F0A7FB23780AF1010A6F
:102F5000534540F37D8457F8043F99F80000184426
:102F6000A0F17F0388FB0321DA17C2EB610202EBB9
:102F700042027F28A3EB8203E2DCFDF76DFBE1E771
:102F80006C9EFF1F129FFF1F9C9CFF1F809CFF1FBA
:102F9000209FFF1FCDCCCC3D0000FE42989CFF1F20
:102FA000642A01003C230100C89EFF1F4D261281A8
:102FB000349FFF1F089FFF1F81DFFF81832008824E
:102FC000489DFF1FB49CFF1FDE9CFF1FF69EFF1F46
:102FD0005C89FF1F3489FF1FABAAAA2A249DFF1F0B
:102FE000989EFF1FB04F38687F2840F3B881AF4BE1
:102FF0007F3883FB0032C317C3EB620303EB430349
:10300000A0EB83007330DFF8FC9299F80040844213
:1030100000F00282A64B1B88002B43D1A54AA6488C
:1030200012680088914205DC8242D4BFC1EB0203E2
:10303000C1EB0003411AB1F5804FA6BF9B030131DC
:10304000C3EB833393FBF1F0FDF7CCFBC0F3C61069
:103050000DF09CFE994B804618880DF097FE98491C
:10306000824640460DF0E6FE014650460DF0E2FE77
:1030700041460DF0D7FD4FF07E5180460EF078F8B6
:10308000002840F0AA868F4940460EF08FF80028AD
:1030900040F0308540460EF0B9F8C0B2DFF86882E3
:1030A00088F800007F2C40F3928380487F3C80FBAF
:1030B0000430E317C3EB600000EB4000A4EB80009A
:1030C0007330814B00931B78C0B289F80000002B4D
:1030D00040F0F4827D4B03931B78002B40F0DF849B
:1030E0007B4B02931B78002B40F01F87794B019399
:1030F000029B1B78FBB1784B1B88012B00F0648589
:10310000022B00F07387032B01F00A81042B01F0DE
:103110001483052B01F0B483062B01F07A85072B6D
:1031200001F0DE85082B01F0F087092B02F03981D0
:103130000A2B02F03A83009B1B78002B00F04C8492
:10314000019B644C1988002900F0A28438687F280C
:1031500040F3B182554B7F3883FB0032C317C3EB7A
:10316000620303EB4303A0EB830073303860002954
:1031700040F05184009B1B78002B00F05981574C84
:103180002378002B00F05481DFF880A1DFF87881EC
:103190004FF0000B0CE003F17300C0B298F8001080
:1031A00006F056FA23780BF1010B5B4540F34081A2
:1031B0003B685AF8040F3D4A1844A0F17F0382FB94
:1031C0000321DA17C2EB610202EB42027F28A3EB74
:1031D0008203E0DCFDF740FADFE73D4C40483A4926
:1031E0003A4A237003700B701370FFF7B0BB934221
:1031F0004FF0000B80F2B6800123CDF800B0CDF87F
:1032000014B00493FFF7E7BA364B1B78002B7FF41A
:103210003AAB039B344A243B83F34703D9B25B2088
:10322000136006F0E5F999F80040032C30D1DFF87F
:10323000E08098F80030002B42F045812B4F3B781E
:10324000002B42F03381274C2378002B42F0218160
:10325000274B1B78002B42F00F81264A1380264B08
:103260001B78002B42F03B81114B7F221A8098F88B
:1032700000306BB93B785BB923784BB91F4A7F218B
:103280000720138006F0B4F97F210B2006F0B0F977
:103290001B4B1F68FFF7F7BAC3EB0313D800631C7F
:1032A00090FBF3F3D5E500BF309FFF1FABAAAA2A1E
:1032B0009C9CFF1F809CFF1F129FFF1F209FFF1FD2
:1032C000CDCCCC3D0000FE42F69EFF1F7D9CFF1F33
:1032D0004A9DFF1FDE9CFF1F669EFF1F5C89FF1F2C
:1032E000A49EFF1F449FFF1FC49CFF1F439FFF1FFF
:1032F000429FFF1F3E9DFF1F459FFF1F969EFF1F82
:103300008C9CFF1F989EFF1F249DFF1F3489FF1F69
:10331000419FFF1FB6480578002D40F04083B54817
:103320000068D0F17F0048BF033003EBA000431CCE
:10333000B1480B609A42B8BF0260FFF676AD1A46FC
:1033400073E5AE4B09881A6000297FF47EAC134602
:103350009842D4BFC2EB0003C2EB03032BE5FDF799
:103360007BF950E60123CDF810B0CDF800B00593FD
:10337000FFF731BA01232B60FFF76FB9029B1B786F
:10338000FBB19F4B1B88012B00F0A084022B00F0A7
:10339000AB86032B01F03A80042B01F0F381052B5F
:1033A00001F0E482062B01F03D84072B01F0378504
:1033B000082B01F0E286092B01F0BC870A2B02F0F2
:1033C000B981019B1B88002B00F02E83009B1B788A
:1033D0003BB9039B1B7823B9029B1B78002B01F0A0
:1033E0008E80884B1B78002B00F0008186490B787B
:1033F000082B00F2FB8085483A680068844C013352
:10340000DBB25F1E101A44F827000B70814BD6F810
:103410000080198889F8002088457F4E7FF71EA913
:1034200032687E4B0892089A7D4C1A60FFF717B9F4
:10343000039B1B78002BA1D03B68A3F10C007F28D5
:1034400040F3418377488B3B80FB0320DA17C2EBC4
:10345000600000EB4000A3EB800303F17300DFF892
:10346000D881C0B298F8001006F0F2F8009B1B78E3
:10347000002B83D0644C2378002B3FF47FAFDFF820
:10348000BCA14FF0000B0CE003F17300C0B298F840
:10349000001006F0DDF823780BF1010B5B457FF798
:1034A0006DAF3B685AF8040F5E4A1844A0F18B03D5
:1034B00082FB0321DA17C2EB61020C3802EB4202F5
:1034C0007F28A3EB8203DFDCFDF7C6F8DEE74D4B78
:1034D0001B78002B40F0B5823B68534A1278002AD3
:1034E00045D0A3F10C007F2840F3F3824D4A8B3B7B
:1034F00082FB0321DA17C2EB610202EB4202A3EB6B
:10350000820303F17300C0B298F8001006F0A0F82F
:10351000009B1B7853B33C4C23783BB3DFF81C91E2
:10352000DFF800A14FF0000B0BE003F17300C0B215
:1035300098F8001006F08CF823780BF1010B5B452E
:1035400014DD3B6859F8040F1844A0F18B038AFB83
:103550000321DA17C2EB61020C3802EB42027F282A
:10356000A3EB8203E1DCFDF777F8E0E73B682F4A45
:103570001278FAB1224A1288012A00F03184022A14
:1035800000F03386032A00F0CC87042A01F0218161
:10359000052A01F05E82062A01F04C83072A01F019
:1035A000F184082A01F05586092A01F026870A2AA3
:1035B00002F08980019A1288002A00F03B821C4A9E
:1035C000174C137003232B60FFF749B8DFF87080A6
:1035D00098F80030002B40F0FE80164F3B78002B0F
:1035E00040F0C8840E4C3B70FFF739B83A680DE7DD
:1035F000FC9EFF1FF89EFF1F389DFF1F809CFF1F32
:10360000669EFF1FA49EFF1F5C89FF1FA89CFF1FD3
:103610003889FF1F489DFF1F30A0FF1FDC9FFF1F41
:10362000709EFF1FABAAAA2A7D9CFF1F4A9DFF1F09
:10363000989EFF1F9A9CFF1F249DFF1F3489FF1F28
:10364000949EFF1FDBB21846137006F08FF8A54B4F
:10365000A5491A46A54B184600230B703B70137002
:103660000370FFF789B80123FFF7C8B88024A04989
:10367000A04BA14A09881B8812680B44B2EB630F68
:10368000BFF601A99D4B1B78002B40F0F281B8F8E2
:1036900000309B4AA3423FF4F6A89A4B14800122C3
:1036A0001A70FFF7F0B8FDF73FF8FFF79CBAFCF788
:1036B000E5FFFFF793BAFCF7CFFF57E5924B019375
:1036C0001B8863BB894B0393904B0293904C2378E8
:1036D0007BB3DFF85882DFF83CA24FF0000B09E023
:1036E00003F17300C0B205F0D7FF23780BF1010B93
:1036F0005B451EDD58F8043F99F800001844A0F11E
:103700007F038AFB0321DA17C2EB610202EB42025C
:103710007F28A3EB8203E3DCFCF79EFFE2E7734B19
:1037200003937A4B029305F0B7FF009B1B78002BA5
:10373000CCD1039B1B78002B3FF4DAAC99F8003016
:10374000A3F10C007F2840F3C18172488B3B80FBC2
:103750000320DA17C2EB600000EB4000A3EB80030C
:1037600003F17300C0B205F097FF009B1B78002B9C
:1037700000F09E81664C2378002B01F07782DFF801
:10378000AC81DFF890A14FF0000B0AE003F1730069
:10379000C0B205F081FF23780BF1010B5B457FF789
:1037A000A7AC58F8043F99F800001844A0F18B0327
:1037B0008AFB0321DA17C2EB61020C3802EB4202EA
:1037C0007F28A3EB8203E1DCFCF746FFE0E720461D
:1037D000FCF742FF75E4504A1278002A40F0A081BD
:1037E0004E4F4F4C3B70FEF73ABFFCF735FFFFF7EB
:1037F00043BA002008704B49087840B1394900911C
:103800000978002900F07C81009F00213970464929
:10381000097800297FF47CA8002C40F0CD80002896
:1038200040F0CA80354C2F4F94F800E02F4C0394A1
:10383000364C02942D4C2C492070344C0097087063
:1038400038702070BEF1000F7FF474A8FFF77EB8C7
:10385000264B1B78002B6BD099F80030A3F10C009D
:103860007F2840F392832B4A8B3B82FB0321DA179C
:10387000C2EB610202EB4202A3EB820303F173008D
:10388000C0B205F009FF009B1B78002B50D0204CE4
:103890002378002B4CD0254FDFF878804FF0000ABA
:1038A00009E003F17300C0B205F0F6FE23780AF1D7
:1038B000010A53453CDD57F8043F99F800001844CD
:1038C000A0F18B0388FB0321DA17C2EB61020C38ED
:1038D00002EB42027F28A3EB8203E2DCFCF7BCFE92
:1038E000E1E700BFF69EFF1FA49EFF1F7D9CFF1F08
:1038F0005C9EFF1F609EFF1FD89CFF1F949EFF1FB2
:10390000E49EFF1FA49CFF1FDE9CFF1F4A9DFF1F1C
:103910005C89FF1FABAAAA2AE89EFF1F9A9CFF1F83
:10392000709EFF1F459FFF1F419FFF1F3489FF1F90
:10393000914B1B78FBB1914B1B88012B00F07686D5
:10394000022B00F07087032B01F0EA80042B01F0BA
:103950007881052B01F0BB83062B01F0E084072B57
:1039600001F0CA85082B01F07D86092B01F08B87B9
:103970000A2B01F06887019B1B88002B00F0B8829E
:103980007F4B1B78002B40F0AE827E4B7E4A19881D
:10399000D6F800800020012310602B603CE5013543
:1039A000EDB2022D86BF0022027005701A46FFF7A5
:1039B0003CBA0398002101707449097800293EF44B
:1039C000C5AF6D4902910978002900F0528702982D
:1039D00000210170FEF7BABF039B1B78002B7FF418
:1039E000AFAB029B1B78002B7FF4AAAB019B19881D
:1039F000FFF7ACBB243B002BB8F8000040F3748405
:103A000098423EF418AF9BB26148A8F800300123F9
:103A10000370FEF710BFDFF87C81C0B298F8001089
:103A200005F016FEFFF7A6BB5A4B3878197805F05B
:103A30000FFECBE4D8B298F8001005F009FE3B6801
:103A4000BDE57F21402005F0D3FD5349534A3B6833
:103A50000B600021117040E5C0B298F8001005F02D
:103A6000F7FDFFF710B94E4BDFF854E11978FEF778
:103A7000E2BE4B2C40F348821834802CB8F800305A
:103A8000484AA8BF8024A3427FF407AEFEF7FBBEDE
:103A900099F8000005F000FE2188FFF757BB424B64
:103AA00001931B88002B41F03487334B029345E68A
:103AB000029B1B78002B7FF41EAB039B1B78002B13
:103AC0007FF43EAB92E7FCF7C7FDC8E4FCF7C4FD0A
:103AD00048E6FCF7C1FD16E5FCF7BEFDFFF716BA98
:103AE000421CD2B2022A40F2568200222A701A46A2
:103AF000FFF79BB97F20FFF7D1BA7F20FFF78FB97F
:103B00001D4F1F4902974FF0000C81F800C0009F25
:103B100002994FF0010E87F800E081F800C076E6C8
:103B2000224F387802F072FE214B1B78002B00F0F8
:103B300040823B887E2B00F23C821E4CDFF8849052
:103B40002268D9F80010521A0F2A40F229821A4A24
:103B50000133108899B23980002800F04382C9B23D
:103B6000C0B205F045FD154F226898F80030C9F83D
:103B700000203B70FEF773BD4A9DFF1F669EFF1F2E
:103B8000A49EFF1F489DFF1F809CFF1F949EFF1F48
:103B9000A49CFF1F249DFF1FA89CFF1F5C89FF1F83
:103BA0001F9FFF1FE49EFF1FDE9CFF1FD49CFF1F73
:103BB000469FFF1F709EFF1F209DFF1F9A9CFF1FA7
:103BC000F99CFF1F2C9FFF1FDFF89CA399F80000B2
:103BD000BAF80030DF4AE04CC31A82FB031ED91743
:103BE000C1EB6E0101EB4101A3EB810303EB430346
:103BF00054F8233018447F2840F38F847F3882FBA9
:103C00000032C317C3EB620303EB4303A0EB830053
:103C10007330DFF858B3C0B205F03EFDBBF800309A
:103C2000022B7FF688AA99F80010BAF80030C94A2A
:103C3000CB1A82FB030ED817C0EB6E0000EB4000DE
:103C4000A3EB800303EB430304EB830358680844AE
:103C50007F2840F3FA867F3882FB0032C317C3EB1C
:103C6000620202EB4202A0EB82007330C0B205F0A8
:103C700013FDBBF80030032B7FF65DAA99F8001006
:103C8000BAF80030B34ACB1A82FB030ED817C0EB48
:103C90006E0000EB4000A3EB800303EB430304EB57
:103CA0008304A06808447F2840F351817F3882FB59
:103CB0000032C317C3EB620202EB4202A0EB8200A8
:103CC0007330C0B205F0E8FCFFF735BADFF898A210
:103CD0003868BAF800309F4A9F4CC31A82FB031E13
:103CE000D917C1EB6E0101EB4101A3EB810303EB9B
:103CF000430354F8233018447F2840F30A847F3864
:103D000082FB0032C317C3EB620303EB4303A0EB58
:103D100083007330DFF85882DFF850B298F8001053
:103D2000C0B205F095FCBBF80030022B7FF649AB22
:103D30003968BAF80030874ACB1A82FB030ED817CD
:103D4000C0EB6E0000EB4000A3EB800303EB4303EA
:103D500004EB8303586808447F2840F372867F3859
:103D600082FB0032C317C3EB620202EB4202A0EBFC
:103D700082007330C0B298F8001005F069FCBBF8FF
:103D80000030032B7FF61DAB3968BAF80030714A5A
:103D9000CB1A82FB030ED817C0EB6E0000EB40007D
:103DA000A3EB800303EB430304EB8304A068084404
:103DB0007F2840F3FB807F3882FB0032C317C3EBC0
:103DC000620202EB4202A0EB8200733098F800100E
:103DD000C0B205F03DFCFFF7F4BA0120FFF75EB971
:103DE000DFF884A15B49BAF800205B4C9A1A81FB8A
:103DF000020ED017C0EB6E0000EB4000A2EB800279
:103E000002EB420254F8220018447F2840F3008459
:103E1000A0F17F0381FB0321DA17C2EB610000EB05
:103E20004000A3EB80007330DFF840B198F8001039
:103E3000C0B205F00DFCBBF80030022B50D9396838
:103E4000BAF80030434ACB1A82FB030ED817C0EBF6
:103E50006E0000EB4000A3EB800303EB430304EB95
:103E60008303586808447F2840F356867F3882FBD6
:103E70000032C317C3EB620202EB4202A0EB8200E6
:103E80007330C0B298F8001005F0E2FBBBF80030C8
:103E9000032B25D93868BAF800302E4AC31A82FBA2
:103EA000031ED917C1EB6E0101EB4101A3EB8103A6
:103EB00003EB430304EB8304A36818447F2867DD06
:103EC0007F3882FB0032C317C3EB620202EB42026F
:103ED000A0EB82007330C0B298F8001005F0B8FB78
:103EE0003B68FFF767BB0021402005F081FB4CE5F4
:103EF00099F8000005F0D0FB42E505F0CDFBFFF797
:103F00000EB80120FEF78BBF243C002CB8F800301F
:103F100040F39185A3423EF4B6ACA4B20F4BA8F88F
:103F2000004001221A70FEF7AEBC0D4B01931B88B6
:103F3000002B3FF4DDA8FFF7F6BB0A4A8342A8BF77
:103F400003461360FEF781BE1446FFF79BBBFCF7E8
:103F500083FBB6E6ABAAAA2A68290100A49CFF1F2E
:103F6000DE9CFF1F809CFF1FA09EFF1FB89CFF1FB1
:103F7000249DFF1FDF4BE04C19886A2005F092FC5E
:103F800098F800303B70FEF76ABBFCF765FB77E4FE
:103F9000FCF762FB9FE72A701A46FEF746BFD64C35
:103FA000D64F98F800303B70FEF759BBFCF754FB36
:103FB0000CE7D34B1B78002BF1D03B88CD4F002B67
:103FC000EDD0CD4CDFF848932268D9F80010521A92
:103FD0000F2AE5D9CB4A013B108899B239800028D5
:103FE0007FF4BDADC8B205F0A3FBBCE5DFF824A3A8
:103FF00099F80000BAF80030C34AC44CC31A82FBD7
:10400000031ED917C1EB6E0101EB4101A3EB810344
:1040100003EB430354F8233018447F2840F3FD8317
:104020007F3882FB0032C317C3EB620303EB430309
:10403000A0EB83007330DFF8E0B2C0B205F02CFBD8
:10404000BBF80030022B7FF676A899F80010BAF87A
:104050000030AD4ACB1A82FB030ED817C0EB6E00BE
:1040600000EB4000A3EB800303EB430304EB83036B
:10407000586808447F2840F3F1857F3882FB00327E
:10408000C317C3EB620303EB4303A0EB830073305E
:10409000C0B205F001FBBBF80030032B7FF64BA844
:1040A00099F80010BAF80030974ACB1A82FB030E39
:1040B000D817C0EB6E0000EB4000A3EB800303EBCE
:1040C000430304EB8304A06808447F287FF73FAFD5
:1040D0007F3882FB0032C317C3EB620303EB430359
:1040E000A0EB83007330ECE5DFF828A23868BAF85B
:1040F0000030854A854CC31A82FB031ED917C1EBD9
:104100006E0101EB4101A3EB810303EB430354F880
:10411000233018447F2840F359837F3882FB0032D4
:10412000C317C3EB620303EB4303A0EB83007330BD
:10413000DFF8E881DFF8E0B198F80010C0B205F0D0
:1041400087FABBF80030022B7FF63BA93968BAF832
:1041500000306D4ACB1A82FB030ED817C0EB6E00FD
:1041600000EB4000A3EB800303EB430304EB83036A
:10417000586808447F2840F36D857F3882FB003201
:10418000C317C3EB620303EB4303A0EB830073305D
:10419000C0B298F8001005F05BFABBF80030032BB2
:1041A0007FF60FA93868BAF80030574AC31A82FB65
:1041B000031ED917C1EB6E0101EB4101A3EB810393
:1041C00003EB430304EB8304A36818447F287FF7C1
:1041D000EDAE7F3882FB0032C317C3EB620303EB03
:1041E0004303A0EB83007330F0E5DFF828A14649D4
:1041F000BAF80020454C9A1A81FB020ED017C0EB8A
:104200006E0000EB4000A2EB800202EB420254F889
:10421000220018447F2840F30383A0F17F0381FB31
:104220000321DA17C2EB610000EB4000A3EB800032
:104230007330DFF8E4B098F80010C0B205F008FA67
:10424000BBF80030022B7FF64BAE3968BAF800306D
:104250002D4ACB1A82FB030ED817C0EB6E0000EB81
:104260004000A3EB800303EB430304EB8303586894
:1042700008447F2840F3F6847F3882FB0032C3175E
:10428000C3EB620303EB4303A0EB83007330C0B2C4
:1042900098F8001005F0DCF9BBF80030032B7FF62E
:1042A0001FAE3868BAF80030174AC31A82FB031EE3
:1042B000D917C1EB6E0101EB4101A3EB810303EBC5
:1042C000430304EB8304A36818447F287FF760AEA0
:1042D0007F3882FB0032C317C3EB620303EB430357
:1042E000A0EB83007330F6E501283EF4A4AA012375
:1042F000FFF78ABBD49CFF1F709EFF1F9A9CFF1F75
:10430000459FFF1F209DFF1FABAAAA2A682B010013
:104310002C9FFF1FA09EFF1FB89CFF1F249DFF1F07
:10432000DFF8FCA299F80000BAF80030BA4ABB4C9A
:10433000C31A82FB031ED917C1EB6E0101EB4101C9
:10434000A3EB810303EB430354F8233018447F2885
:1043500040F3E7817F3882FB0032C317C3EB620270
:1043600002EB4202A0EB82007330DFF8B8B2C0B2B9
:1043700005F092F9BBF80030022B7EF6DCAE99F81E
:104380000000BAF80030A44AC31A82FB0321DA17EE
:10439000C2EB610202EB4202A3EB820303EB430395
:1043A00004EB83035B6818447F2840F328847F383C
:1043B0000C2290FBF2F302FB13007330C0B205F045
:1043C0006BF9BBF80030032B7EF6B5AE99F8000010
:1043D000BAF80030904AC31A82FB0321DA17C2EB05
:1043E000610202EB4202A3EB820303EB430304EB03
:1043F0008304A36818447F287FF7A9AD7F380C2277
:1044000090FBF2F302FB130073305AE4DFF810A2C2
:104410003868BAF80030804A804CC31A82FB031E09
:10442000D917C1EB6E0101EB4101A3EB810303EB53
:10443000430354F8233018447F2840F36F817F38BA
:1044400082FB0032C317C3EB620202EB4202A0EB15
:1044500082007330DFF8D081DFF8C8B198F800101F
:10446000C0B205F0F5F8BBF80030022B7EF6A9AF1C
:104470003868BAF80030684AC31A82FB0321DA1799
:10448000C2EB610202EB4202A3EB820303EB4303A4
:1044900004EB83035B6818447F2840F3AD837F38C7
:1044A0000C2290FBF2F302FB13007330C0B298F8B9
:1044B000001005F0CDF8BBF80030032B7EF681AF7D
:1044C0003868BAF80030544AC31A82FB0321DA175D
:1044D000C2EB610202EB4202A3EB820303EB430354
:1044E00004EB8304A36818447F287FF75FAD7F380F
:1044F0000C2290FBF2F302FB1300733066E44FF4DE
:104500007A43013BFDD199F8000005F0C5F8FEF7AC
:1045100068BFFCF7A1F8FFF7FDBBFCF79DF8FFF7BC
:1045200078BBDFF8FCA03C49BAF800203B4C9A1A53
:1045300081FB020ED017C0EB6E0000EB4000A2EB37
:10454000800202EB420254F8220018447F2840F314
:10455000EB80A0F17F0381FB0321DA17C2EB61013D
:1045600001EB4101A3EB81007330DFF8B8B098F89C
:104570000010C0B205F06CF8BBF80030022B7FF6DB
:10458000AFAC3868BAF80030234AC31A82FB032163
:10459000DA17C2EB610202EB4202A3EB820303EBE8
:1045A000430304EB83035B6818447F2840F32E83A6
:1045B0007F380C2290FBF2F302FB13007330C0B281
:1045C00098F8001005F044F8BBF80030032B7FF694
:1045D00087AC3868BAF800300F4AC31A82FB03214F
:1045E000DA17C2EB610202EB4202A3EB820303EB98
:1045F000430304EB8304A36818447F287FF7C8AC07
:104600007F380C2290FBF2F302FB1300733062E45C
:10461000FCF722F808E400BFABAAAA2AF82B010095
:10462000A09EFF1FB89CFF1F249DFF1FDFF834A32F
:1046300099F80000BAF80030C24AC34CC31A82FB92
:104640000317D917C1EB670101EB4101A3EB81030C
:1046500003EB430354F8233018447F286ADD7F3886
:1046600082FB0032C317C3EB620202EB4202A0EBF3
:1046700082007330DFF8F0B2C0B205F00DF8BBF87D
:104680000030022B7FF677A999F80000BAF80030C5
:10469000AC4AC31A82FB0321DA17C2EB610202EBB8
:1046A0004202A3EB820303EB430304EB83035B6847
:1046B00018447F2840F3A7827F380C2290FBF2F346
:1046C00002FB13007330C0B204F0E6FFBBF8003009
:1046D000032B7FF650A999F80000BAF80030994AE8
:1046E000C31A82FB0321DA17C2EB610202EB42021A
:1046F000A3EB820303EB430304EB8304A368184496
:104700007F2814DD7F380C2290FBF2F302FB1300AC
:104710007330C0B204F0C0FFFFF72DB9FBF79CFF68
:1047200098E6FBF799FF20E6FBF796FF1DE7FBF7FE
:1047300093FFEEE7FBF790FF9CE7DFF828A299F8DC
:104740000000BAF800307F4A804CC31A82FB031E77
:10475000D917C1EB6E0101EB4101A3EB810303EB20
:10476000430354F8233018447F28DADD7F3882FB76
:104770000032C317C3EB620303EB4303A0EB8300D8
:104780007330F2E5DFF8DCA13868BAF800306D4A22
:104790006E4CC31A82FB031ED917C1EB6E0101EBED
:1047A0004101A3EB810303EB430354F82330184486
:1047B0007F28B3DD7F3882FB0032C317C3EB62036F
:1047C00003EB4303A0EB8300733043E6FBF744FFA6
:1047D000AEE4DFF890A15B49BAF800205B4C9A1A6E
:1047E00081FB020ED017C0EB6E0000EB4000A2EB85
:1047F000800202EB420254F8220018447F2893DD25
:10480000A0F17F0381FB0321DA17C2EB610000EB0B
:104810004000A3EB80007330A7E6FBF71DFF0AE41E
:10482000FBF71AFF05E5DFF83CA199F80000BAF89C
:104830000030444A464CC31A82FB0317D917C1EB18
:10484000670101EB4101A3EB810303EB430354F840
:10485000233018447F287FF76DAF7F3882FB00320A
:10486000C317C3EB620303EB4303A0EB8300733076
:1048700000E738480090384838490390FEF75AB8A6
:10488000DFF8E0A099F80000BAF800302D4A344C67
:10489000C31A82FB0321DA17C2EB610202EB420268
:1048A000A3EB820303EB430354F8233018447F281F
:1048B00040F39F817F380C2290FBF2F302FB130040
:1048C0007330DFF8A4B0C0B204F0E6FEBBF80030ED
:1048D000022B19D999F80000BAF800300C22C11A3D
:1048E00091FBF2F302FB131302FB03435B681844D2
:1048F0007F2840F33B847F3890FBF2F302FB1300E8
:104900007330C0B204F0C8FEBBF80030032B7EF653
:1049100012ACBAF8003099F800000C22C11A91FBD1
:10492000F2F302FB131302FB0344A36818447F282D
:104930007FF70DAB7F3890FBF2F302FB130073306F
:10494000FFF7BFB9ABAAAA2A68290100D425010044
:10495000682B0100F69EFF1F7D9CFF1FA49EFF1F7A
:104960007C2E0100A09EFF1FB89CFF1FDFF864A3F0
:104970003868BAF80030CE4ACE4CC31A82FB032105
:10498000DA17C2EB610202EB4202A3EB820303EBF4
:10499000430354F8233018447F2840F327817F389D
:1049A0000C2290FBF2F302FB13007330DFF8288334
:1049B000DFF828B398F80010C0B204F049FEBBF845
:1049C0000030022B1AD93868BAF800300C22C11A0C
:1049D00091FBF2F302FB131302FB03435B681844E1
:1049E0007F2840F3C7837F3890FBF2F302FB13006C
:1049F0007330C0B298F8001004F02AFEBBF8003003
:104A0000032B7EF6DEACBAF8003038680C22C11AEF
:104A100091FBF2F302FB131302FB0344A368184457
:104A20007F287FF7C3AA7F3890FBF2F302FB1300C5
:104A30007330FFF7CBB9012B3DF425AF0124FFF70D
:104A40006DBAFBF709FEFFF795B9FBF705FEFFF717
:104A50000DB9DFF880A29649BAF80020954C9A1A51
:104A600081FB0210D117C1EB600101EB4101A2EB08
:104A7000810202EB420254F8220018447F2840F3DE
:104A8000B280A0F17F030C2093FBF0F200FB123008
:104A90007330DFF848B298F80010C0B204F0D8FDC7
:104AA000BBF80030022B1AD93868BAF800300C2253
:104AB000C11A91FBF2F302FB131302FB03435B6881
:104AC00018447F2840F31E837F3890FBF2F302FBEB
:104AD00013007330C0B298F8001004F0B9FDBBF8B1
:104AE0000030032B7FF6FCA9BAF8003038680C229E
:104AF000C11A91FBF2F302FB131302FB0344A368F8
:104B000018447F287FF744AA7F3890FBF2F302FB1A
:104B100013007330FFF7DFB9FBF79EFDFFF7B1B964
:104B2000DFF8B0A199F80000BAF80030604A624C92
:104B3000C31A82FB0321DA17C2EB610202EB4202C5
:104B4000A3EB820303EB430354F8233018447F287C
:104B500046DD7F380C2290FBF2F302FB130073302A
:104B6000DFF878B1C0B204F097FDBBF80030022B3B
:104B700019D999F80000BAF800300C22C11A91FB3B
:104B8000F2F302FB131302FB03435B6818447F2814
:104B900040F38B807F3890FBF2F302FB13007330FD
:104BA000C0B204F079FDBBF80030032B7EF6E3AE13
:104BB000BAF8003099F800000C22C11A91FBF2F308
:104BC00002FB131302FB0344A36818447F287FF7FA
:104BD000AEAD7F3890FBF2F302FB1300733098E523
:104BE000FBF73AFDBCE7FBF737FD52E7FBF734FD77
:104BF000DCE6FBF731FD64E6FBF72EFD56E4FBF740
:104C00002BFDFFF7DBBBFBF727FD5CE5FBF724FD86
:104C1000D5E4DFF8C0A099F80000BAF80030244AC3
:104C2000264C35E6DFF8ACA03868BAF80030204AE8
:104C3000224CA2E6DFF89CA01D49BAF800201F4CC8
:104C40000DE7DFF890A099F80000BAF80030184A94
:104C50001B4C6DE7FBF700FDFFF79ABAFBF7FCFC76
:104C6000FFF716BAFBF7F8FCFFF711BB029B1B78A6
:104C7000002B7EF440AAFEF763BA124B1B78002B80
:104C800000F0C182104B1B78002B7DF4FCAD0F4B64
:104C90001B78002B3DF4F7ADB8F800300C490A330F
:104CA000A8F800300A70FDF7EEBDFBF7D5FC77E7FA
:104CB000ABAAAA2A7C2E0100F82B0100242D0100AA
:104CC000D4250100429FFF1F439FFF1F449FFF1FEA
:104CD000A49CFF1FA09EFF1F249DFF1FB89CFF1FC9
:104CE000A14C2388002B40F07D83DFF894B29F49CC
:104CF0009F4A098899F80000B2F800E0DFF878824E
:104D0000C1EB000C0C229CFBF2F102FB11C14FF035
:104D1000900C0CFB0EFE02FB01E16FF00B0E58F83D
:104D2000011008440EFB03007F2840F35F85A0F1CB
:104D30007F0393FBF2F002FB10307330C0B204F03B
:104D4000ABFCBBF8002023881344022B22DD874AEA
:104D5000874B118899F80000B3F800C0DFF818E21B
:104D6000411A0C2291FBF2F302FB1311902303FB77
:104D70000CF302FB013373445B6818447F2840F353
:104D800053857F3890FBF2F302FB13007330C0B2FF
:104D900004F082FCBBF8002023881344032B22DD9F
:104DA000724A734B118899F80000B3F800C0DFF81D
:104DB000C8E1411A0C2291FBF2F302FB131190237C
:104DC00003FB0CF302FB013373449B6818447F28F8
:104DD00040F310857F3890FBF2F302FB1300733031
:104DE000C0B204F059FCBBF8002023881344042B04
:104DF0007EF7A1A95F4B1B88012B7EF49CA999F833
:104E00000020A2F10C007F287FF7A1A88B3A0C208C
:104E100092FBF0F300FB13207330FEF752BF524CAD
:104E20002388002B40F01D83DFF854B14F49504ACE
:104E30000988D7F80080B2F800E04F48C1EB080CB1
:104E40000C229CFBF2F102FB11C14FF0900C0CFB09
:104E50000EFE02FB01E16FF00B0E405880440EFB8A
:104E600003807F2840F39D84A0F17F0393FBF2F041
:104E700002FB10307330414BC0B2197804F0E8FBEC
:104E8000BBF8002023881344022B23DD374A384B1C
:104E900011883868B3F800C0DFF8DCE0411A0C2252
:104EA00091FBF2F302FB1311902303FB0CF302FBC3
:104EB000013373445B6818447F2840F3AB847F3828
:104EC00090FBF2F302FB130073302C4BC0B2197845
:104ED00004F0BEFBBBF8002023881344032B23DD22
:104EE000224A234B11883868B3F800C0DFF888E005
:104EF000411A0C2291FBF2F302FB1311902303FBE6
:104F00000CF302FB013373449B6818447F2840F381
:104F10008F847F3890FBF2F302FB13007330174B42
:104F2000C0B2197804F094FBBBF800202388134426
:104F3000042B7EF746AA0F4B1B88012B7EF441AA57
:104F40003A68A2F10C007F2840F3E6818B3A0C20EE
:104F500092FBF0F300FB13207330084BC0B21978BA
:104F600004F076FBFEF72DBA2C9DFF1FA09EFF1FBD
:104F7000509EFF1FD29CFF1F64260100249DFF1F2F
:104F8000B89CFF1FCD4C2288002A00F0D081CC496C
:104F9000DFF858B30988BBF800000331884227DDE9
:104FA000C848C9490088B1F800E0DFF844C3181ABE
:104FB0000C2190FBF1F901FB19004FF0900909FB5E
:104FC0000EFE01FB00E06FF00B0E5CF800000344E6
:104FD0000EFB02307F2840F3AA837F3890FBF1F369
:104FE00001FB13007330C0B298F8001004F030FBDE
:104FF000BBF8002023881344022B23DDB14BB24AB7
:1050000038681B88B2F800C0DFF8E4E2C31A0C214C
:1050100093FBF1F201FB1232902303FB0CF301FB33
:10502000023373445B6818447F2840F308847F3858
:1050300090FBF1F301FB13007330C0B298F800103D
:1050400004F006FBBBF8002023881344032B23DD68
:105050009C4B9D4A38681B88B2F800C0DFF890E28C
:10506000C31A0C2193FBF1F201FB1232902303FBD4
:105070000CF301FB023373449B6818447F2840F310
:10508000DB837F3890FBF1F301FB13007330C0B278
:1050900098F8001004F0DCFABBF8002023881344D1
:1050A000042B7EF71DAF864B1B88012B7EF418AFB7
:1050B0003A68A2F10C007F287EF76AAF8B3A0C2089
:1050C00092FBF0F300FB13207330FEF704BFDFF810
:1050D000F4A199F80000BAF800307C4CC11A0C22F7
:1050E00091FBF2F302FB131302FB03F3E3581844A2
:1050F0007F287FF775AD7F3890FBF2F302FB13003A
:1051000073302DE5FBF7A8FAE4E4714B1B88182BEC
:1051100012D099F800201344A3F118007F2840F31F
:1051200076830C20973B93FBF0F200FB123303F1E4
:105130007300C0B204F0B0FA664A674B127833F8D5
:105140001230182B3DF4F7AF99F800201344A3F167
:1051500018007F287EF7FBAE0C20973B93FBF0F204
:1051600000FB123303F17300FEF7ABBDFBF774FADB
:10517000FFF7C7BBFBF770FA3BE4554B1A88182AB8
:1051800013D03B681344A3F118007F2840F33C83FD
:105190000C20973B93FBF0F200FB123303F17300FA
:1051A0004E4BC0B2197804F053FA4A4B4A491A7868
:1051B000022A94BF013200221A701A7831F81200C4
:1051C000182810D10424022A02F10100C2B288BFBB
:1051D000002231F81200182804D1013CF3D11A70D2
:1051E000FEF7EFB81A703B680344A3F118007F285C
:1051F00040F392800C20973B93FBF0F200FB1233BC
:1052000003F17300A9E6364B1B78002B7DF4FCAF4D
:10521000344B1B78002B3DF436ABB8F800303249E4
:105220000133A8F800300A70FDF72DBB2C4B1B781A
:10523000002B7DF428AB2B4B1B78002B3DF423ABCC
:10524000B8F800302849013BA8F800300A70FDF793
:105250001ABB1F4A1288182A12D01344A3F118004F
:105260007F2840F3CE820C20973B93FBF0F200FBAB
:10527000123303F17300C0B298F8001004F0E8F99B
:10528000144B15491A78022A94BF013200221A7071
:105290001A7831F8120018282DD10424022A02F1BC
:1052A0000100C2B288BF002231F81200182821D1B3
:1052B000013CF3D11A703B68FEF77CB92C9DFF1FAF
:1052C000D29CFF1FA09EFF1F509EFF1F7C2E01003F
:1052D000C09CFF1F9489FF1FBC9EFF1F249DFF1FC2
:1052E000439FFF1F449FFF1FA49CFF1FB89CFF1FED
:1052F000642601001A703B680344A3F118007F285C
:105300007EF746AE0C20973B93FBF0F200FB123386
:1053100003F17300FEF7DFBDFBF79EF91DE6DFF832
:1053200034A399F80000BAF80030C04CD6E6DFF894
:1053300030B335E6BE4B1A88182A13D03B681344A5
:10534000A3F118007F2840F369820C20973B93FB60
:10535000F0F200FB123303F17300B64BC0B21978C0
:1053600004F076F9B44BB5491A78022A94BF013299
:1053700000221A701A7831F8120018287FF433AF1F
:105380000424022A02F1010294BFD2B2002231F8B1
:10539000120018287FF426AF013CF2D11A70FEF7F4
:1053A00010B8A34B1B88182B12D099F80020134477
:1053B000A3F118007F2840F334820C20973B93FB25
:1053C000F0F200FB123303F17300C0B204F064F991
:1053D000994A9A4B127833F81230182B7FF4B4AEF6
:1053E000FDF7A9BE964ADFF878B21288BBF8001024
:1053F000033291427FF7A5AC79E48D4A1288182ACE
:1054000012D01344A3F118007F2840F3F7810C2039
:10541000973B93FBF0F200FB123303F17300C0B231
:1054200098F8001004F014F9834B84491A78022A82
:1054300094BF013200221A701A7831F8120018282D
:105440007FF459AF0424022A02F1010294BFD2B2C0
:10545000002231F8120018287FF44CAF013CF2D141
:1054600028E7774ADFF8F8B11288BBF8001003325A
:1054700091427FF705ADD9E4724B01227F210720CD
:105480001A8004F0B5F87F210B2004F0B1F8FDF785
:10549000E6BE6D4B04227F2107201A8004F0A8F895
:1054A00000210B2004F0A4F8FDF7D2BE664B0222C7
:1054B0007F2107201A8004F09BF87F210B2004F045
:1054C00097F8FDF7C0BE604B002107201C8004F058
:1054D0008FF87F210B2004F08BF8FDF7AFBE5B4BFC
:1054E00000227F2107201A8004F082F87F210B2000
:1054F00004F07EF8FDF7BBBE554C2388002B40F02E
:10550000E581DFF85CB1534999F80000524A0988F7
:105510001788DFF848E1411A0C2291FBF2FC02FBEC
:105520001C114FF0900C0CFB07F702FB01716FF0A0
:105530000B075EF80110014407FB03107F2840F3BE
:10554000C2817F3890FBF2F302FB13007330C0B2CC
:1055500004F0A2F8BBF8002023881344022B21DDBD
:105560003C4B3D4A99F800001B88B2F800E03B4FE5
:10557000C31A0C2193FBF1F201FB1232902303FBBF
:105580000EF301FB02333B445B6818447F2840F371
:10559000B4817F3890FBF1F301FB13007330C0B28C
:1055A00004F07AF8BBF8002023881344032B21DD94
:1055B000284B294A99F800001B88B2F800E0274FD1
:1055C000C31A0C2193FBF1F201FB1232902303FB6F
:1055D0000EF301FB02333B449B6818447F2840F3E1
:1055E00089817F3890FBF1F301FB13007330C0B267
:1055F00004F052F8BBF8002023881344042B7EF7F4
:10560000BAA90F4B1B88012B7EF4B5A999F800208D
:10561000A2F10C007F287FF78AA88B3A0C2092FB1E
:10562000F0F300FB13207330FFF773B8242D010053
:10563000CA9CFF1F249DFF1F9489FF1F309EFF1FE0
:10564000D29CFF1F3E9DFF1F969EFF1F9C9CFF1F2D
:105650002C9DFF1FA09EFF1F509EFF1F6426010070
:10566000B89CFF1FAD4B1B88182B12D099F8002057
:105670001344A3F118007F2840F342810C20973B8C
:1056800093FBF0F200FB123303F17300C0B204F09D
:1056900003F8A34AA34B127833F81230182B3EF4C8
:1056A0006AA999F800201344A3F118007F287FF716
:1056B0003EA80C20973B93FBF0F200FB123303F162
:1056C0007300FFF726B8984A1288182A12D013449C
:1056D000A3F118007F2840F30A810C20973B93FB2D
:1056E000F0F200FB123303F17300C0B298F800101F
:1056F00003F0AEFF8A4B8D491A78022A94BF01321B
:1057000000221A701A7831F8120018287FF4F3ADCD
:105710000424022A02F1010294BFD2B2002231F81D
:10572000120018287FF4E6AD013CF2D1C2E5FAF789
:1057300093FF58E47C4B1A88182A13D03B68134413
:10574000A3F118007F2840F3E1800C20973B93FBE6
:10575000F0F200FB123303F17300754BC0B21978FD
:1057600003F076FF6E4B71491A78022A94BF01321A
:1057700000221A701A7831F8120018287FF433AD1D
:105780000424022A02F1010294BFD2B2002231F8AD
:10579000120018287FF426AD013CF2D11A70FDF7F3
:1057A00010BEFAF759FFFFF766BB5F4B1B88182B3B
:1057B00012D099F800201344A3F118007F2840F379
:1057C000A2800C20973B93FBF0F200FB123303F115
:1057D0007300C0B203F060FF514A544B127833F8A3
:1057E0001230182B7FF4B0ACFDF7A5BCFAF734FFEC
:1057F000FFF7A4BAFAF730FFFFF7F2BAFAF72CFF77
:105800000DE6FAF729FF36E5FAF726FFC8E4FAF7BE
:1058100023FF8EE4FAF720FFFFF757BBFAF71CFFD0
:105820009BE5FAF719FFD0E5FAF716FFFFF7AFBAD5
:10583000FAF712FFFFF773BBFAF70EFF27E4FAF748
:105840000BFFFFF7FABB384B1B88182B11D099F8C8
:1058500000201344A3F118007F2845DD0C20973B5E
:1058600093FBF0F200FB123303F17300C0B203F0BC
:1058700013FF2B4A2D4B127833F81230182B7FF47C
:1058800010AFFEF778B82B4B1B88182B11D099F866
:1058900000201344A3F118007F2822DD0C20973B41
:1058A00093FBF0F200FB123303F17300C0B203F07C
:1058B000F3FE1B4A204B127833F81230182B7FF47A
:1058C000F0AEFEF758B8FAF7C7FE40E61B4ADFF81D
:1058D00074B01288BBF80010033291427FF73AAEE1
:1058E00011E6FAF7B9FEE1E7FAF7B6FEBEE7FAF716
:1058F000B3FEFAE6FAF7B0FE79E6FAF7ADFE4EE649
:10590000FAF7AAFEC2E6FAF7A7FE62E7FAF7A4FEE4
:1059100023E70B4B0293FDF706BF00BFC09CFF1FA0
:105920009489FF1FBC9EFF1FCC9CFF1F389EFF1F4A
:10593000249DFF1FCA9CFF1F309EFF1FD29CFF1F8C
:105940004A9DFF1FB89CFF1F38B507F079FE0B4832
:1059500005F0B0FD00234FF07E5201210848FAF710
:1059600085FD084B084A0949802400251C7118460A
:105970001D60BDE838400BF069BC00BF3C9DFF1FB7
:10598000749EFF1F009FFF1F1C89FF1FFD05000065
:1059900010B50446A4206368198803F083FFE36808
:1059A000A6201988BDE8104003F07CBF43682A2078
:1059B000198803F077BF00BF10B504462220636842
:1059C000198803F06FFFE36824201988BDE81040B0
:1059D00003F068BF10B504460A206368198803F015
:1059E00061FFE3680C201988BDE8104003F05ABF3E
:1059F00010B5044606206368198803F053FFE36876
:105A000008201988BDE8104003F04CBF10B50446CB
:105A100002206368198803F045FFE36804201988B1
:105A2000BDE8104003F03EBF70B50E4C84B01225A7
:105A30000422012306460390029320468DE82400A9
:105A40001423102106F03AFF06220923029303963D
:105A50000195204600921423102106F02FFF04B078
:105A600070BD00BF789FFF1F70B5AE4CB4F9003019
:105A7000032B00F0E880002B4DD0022B6CD0052BBF
:105A800000F09880012B00F0C080042B00D070BD86
:105A900000244FF4AF75E1B2A34805F073FD013463
:105AA0008542A8BF05460C2CF5D1012008F048FE20
:105AB0000446002008F044FE323CA0F132039B492A
:105AC0006FF4957000FB03F300FB04F081FB0342CD
:105AD00081FB0041DB17C017C3EB6223C0EB6120E1
:105AE00003F5AF7200F5AF739342A8BF13469D4212
:105AF000A8BF1D46A5F11401312900F3E28040F250
:105B00006C7332218A488B4A0180BDE870402A209C
:105B1000136003F0C7BE0E2007F0F6FC40F6FF71DD
:105B2000C8308842A8BF084620EAE07000F2DC5284
:105B300083B28A42804D814EA8BF0A460220194690
:105B400033802A8003F0AEFE2988042003F0AAFEE9
:105B5000B4F90030022B92D1172008F0F1FD054670
:105B6000162008F0EDFDA842B8BF284600F1C80194
:105B7000B1F5FA7FC0F2BF80B1F57A6FA8BF4FF4DC
:105B80007A6101F54873B3F57A6FA8BF4FF47A6371
:105B90009BB289B26A4A6B4D11800A202B8003F0B8
:105BA00081FE29880C2003F07DFEB4F90030052B1E
:105BB0007FF468AF0F2008F0C3FDC0F53F630433E6
:105BC000B3F5AF6FC0F28F80B3F5FA6FA8BF4FF493
:105BD000FA6399B25C4BC0F54360B0F5AF6F1980C2
:105BE0007EDBB0F5FA6FA8BF4FF4FA6083B2574D71
:105BF000A4202B8003F056FE2988A62003F052FE35
:105C0000B4F90030012B7FF440AF0B2008F098F975
:105C100000283CD0112008F093FD00F1C801B1F537
:105C20002F7F3CDB41F25C23994278DC484A00F547
:105C3000487089B2B0F52F7F11806DDB8342A8BF19
:105C400003469BB231E0102008F07AFDC830B0F571
:105C5000FA7F4BDBB0F57A6F0146A8BF4FF47A614B
:105C600001F51673B3F57A6FA8BF4FF47A639BB250
:105C700089B2384A384D118022202B8003F012FE61
:105C80002988242003F00EFEB4F90030F3E6152035
:105C900007F03AFC00F59671B1F52F7F30DA40F24B
:105CA00014534FF42F712A4A11802C4D06202B805B
:105CB00003F0F8FD2988082003F0F4FDB4F9003062
:105CC000E3E640F23A72A5F5B975254B02FB05F5FE
:105CD00083FB0523ED17A5EB631389B2323311E77C
:105CE0004FF4AF6383E74FF4AF6173E740F24C4387
:105CF0004FF4FA71BDE740F214534FF4FA7149E7DB
:105D000041F25C2399420ADC114A00F5617089B2C4
:105D1000B0F52F7F118091DA4FF42F73C5E7194644
:105D2000C1E700BF509FFF1F3C9DFF1F67BBCF46D1
:105D30000A9FFF1FA089FF1F129FFF1F489DFF1F83
:105D4000AC9EFF1FC89CFF1F4C9DFF1FCC9EFF1FDA
:105D5000029DFF1F609EFF1F5C9EFF1FE09EFF1FB6
:105D6000B5814E1B2DE9F041224D82B0012602B2D1
:105D700084B20092284601967823192106F0E4FCAB
:105D800004F10C0212B28DE844002846A7197823CA
:105D9000192104F1020806F0D7FC3FB20FFA88F887
:105DA00019233A46284619460196CDF8008006F098
:105DB000CBFC78233A4628461946CDF80080019658
:105DC00004F10A070B3406F0BFFC3FB224B278237B
:105DD0003A46284619468DE8500006F0B5FC1923CE
:105DE00000943A4601962846194606F0ADFC02B0EA
:105DF000BDE8F081789FFF1F30B583B000230C46CB
:105E000005B2009326225B231C210C4806F0ECF916
:105E1000294601232622094805F0F6FC002C24B26D
:105E200005DB214601232622044805F0EDFC044A47
:105E3000044B15801C8003B030BD00BF789FFF1F4E
:105E4000B689FF1FB889FF1F70B5A54C237882B0B3
:105E50001BB1A44B4FF6FF721A80A34BB3F900306D
:105E6000C3B9A24A9F4B1068B3F9002080F30C001D
:105E70005B2303FB00F000131C3082424AD04FF03A
:105E8000FF31FFF7B9FF9A4806F012FA002323709A
:105E900002B070BD012B1BD0022B5AD0032B3FD078
:105EA000042B00F09A80052BF0D10F2008F048FC5D
:105EB000C0F53B600830B0F5AF6F48DBB0F5FA6F66
:105EC000A8BF4FF4FA60A0F5AF625B23894835E0C4
:105ED000894B1B78002B70D0152007F015FB874BE2
:105EE0001860B0F52F7F32DB41F25C239842A8BFE7
:105EF0001846A0F52F735B22814802FB03F380FB59
:105F00000320DB17C3EBA0201C30764BB3F9003025
:105F10008342B4D17B4BB3F900300133AFD1B5E745
:105F2000794B1B68B3F5FA7F11DBB3F57A6FA8BF25
:105F30004FF47A637548A3F5FA725B2303FB02F30F
:105F400080FB0320DB17C3EB20201C30DDE71C2087
:105F5000DBE76F4B1B68B3F5FA7F36DBB3F57A6F7F
:105F6000A8BF4FF47A63A3F5FA7268485B2303FB7A
:105F700002F380FB0320DB17C3EB20201C30654BB2
:105F80001B68B3F5FA7F1EDBB3F57A6FA8BF4FF439
:105F90007A63A3F5FA725D495B2303FB02F381FB8D
:105FA0000321DB17C3EB21211C314E4BB3F9003029
:105FB00083420CD0FFF720FF65E7112008F0C0FBFB
:105FC0004E4B18608DE71C21EFE71C20D7E74D4BA7
:105FD000B3F900308B42EDD158E7272200258DE838
:105FE000240076231C2142484B4E06F0ADFB16E000
:105FF000B0F5AF7FA8BF4FF4AF70323803FB00F3AA
:1060000086FB0321DB17C3EB61111C3109B20123AD
:106010001D442722364805F0F7FB0C2D09D0E9B2C4
:106020003E4805F0AFFA31284FF05B03E0DC1C215D
:10603000EDE7012008F084FB6FF495733238384A9D
:1060400003FB00F082FB0023C017C0EB632303F5C2
:10605000AF73312B42DDB3F5AF7FA8BF4FF4AF7301
:106060005B22323B2C4D02FB03F385FB0325DB1740
:10607000C3EB65151C35002008F062FB6FF49573C7
:106080003238274A03FB00F082FB0023C017C0EB25
:10609000632303F5AF73312B1EDDB3F5AF7FA8BFCC
:1060A0004FF4AF735B22323B1B4902FB03F381FBCE
:1060B0000321DB17C3EB61111C310A4BB3F900302C
:1060C000AB4201D0284675E70E4BB3F900308B4246
:1060D0003FF4D9AE28466DE71C21EEE71C25CAE740
:1060E0004A9FFF1FB689FF1F509FFF1FB09EFF1FD3
:1060F000789FFF1F37800B6D689EFF1F889CFF1FD6
:10610000D3058541B889FF1FD89CFF1F011FB81216
:10611000E49CFF1FAC9CFF1F4B48371B3C9DFF1F9F
:1061200067BBCF462DE9F041044682B0714827682D
:10613000E56805F0B1FF1120FFF714FE01261923D1
:106140004FF02808194624226A480196CDF80080AD
:1061500006F0FAFA78231946242266480196CDF80B
:10616000008006F0F1FA3146624806F083FE022212
:106170001921604806F07AFE38460BF041FE394698
:1061800002465C4807F00CF85A4807F01FF8142242
:106190000021584806F06AFE03225749554806F088
:1061A000FFFF544807F012F823220021514806F05F
:1061B0005DFE032251494F4806F0F2FF4D4807F0BB
:1061C00005F87DB12F20FFF7CDFD3222002149488F
:1061D00006F04CFE03224A49464806F0E1FF4548D6
:1061E00006F0F4FF0123474A18461370FFF71CFC22
:1061F0002189638962685B1A5C2B128854DD521A0C
:1062000002EB4202C2EB4212013392FBF3F31B3367
:106210003D4A3848138001261A221BB28DE84400FB
:106220001946142206F090FA002D4FD0218A638A75
:10623000E2685B1A5C2B12883EDC511A5C2202FB7E
:1062400001F292FBF3F31B33304A2A4813800125F5
:106250001BB2382219468DE82400322206F074FA67
:106260004023002209218DE806002248194606F045
:1062700039FA29461F4806F0FDFD022244211D4837
:1062800006F0F4FD63681B48198806F0EFFF2A4604
:106290001F49184806F084FFE3681648198802B0C1
:1062A000BDE8F04106F0E2BF511A5C2202FB01F2A8
:1062B00092FBF3F31B33ABE7521A02EB4202C2EB41
:1062C0004212334492FBF3F31B33BDE74023092111
:1062D0002A46009107480195194606F003FA31460F
:1062E000044806F0C7FD02226821024806F0BEFD00
:1062F0006368D2E7789FFF1F542F0100582F0100D9
:106300005C2F0100F19FFF1F4C9FFF1F4E9FFF1F3F
:10631000602F01002DE9F0471F4682B01446002A85
:106320004ED0052A0646D0F80C8000F0AB800B9BBF
:10633000894A00EBC305012CB5F80AE02989686891
:10634000C1EB0E0382FB03C21A444FEAE373C3EBB3
:10635000A213028851D0042C00F08D80002240232B
:1063600009218DE806007D48194606F0BBF9012198
:106370007A4806F07FFD0222B8F1000F00F0E180BC
:106380004421764806F072FD73687448198806F057
:106390006DFF73497148012206F002FFF3686F48F0
:1063A000198806F063FF6F4B022CB3F9001000F060
:1063B000A680082C00F0C280012002B0BDE8F08762
:1063C000694E6A4A33681268CB1A93420D4655D912
:1063D000674A3B8811786148012918BF012414706D
:1063E0000A9A06321BB212B28DE814001946BDF9A2
:1063F000282006F0A9F93560DEE79BB2D31A99424E
:1064000003DC9E457146A8BF19460A9A0180B7F978
:106410000030BDF928A0514802F106094FF0000EE6
:106420000FFA89F919465246CDF80090CDF804E0EC
:1064300006F08AF929896A896868521A03885C2AF1
:10644000A3EB010373DD03EB43030132C3EB4313FF
:1064500093FBF2F303F11B0213B201203A801946B9
:1064600052460190CDF800903C4806F06DF9404B43
:1064700000221A7072E712FA83F3C0E7204602B0D6
:10648000BDE8F08707254FF000095A2323228DE845
:1064900020021A21314806F025F901212F4806F083
:1064A000E9FC01212D4806F0EBFC232235212B4885
:1064B00006F0DCFC2A462F49284806F071FE2748E2
:1064C00006F084FE254805F0F3FE4FF4FA6007F06D
:1064D0006DFDFFF7C9FA5A2323221A218DE8200205
:1064E0001E4806F0FFF81D4805F0E2FE3046FFF7B3
:1064F00019FE214B01221A70FFF7A6FC2EE74A1C59
:1065000012B21A8091423FF457AF0A9AB7F900309D
:1065100012480632012412B2009219460194BDF9C4
:10652000282006F011F9204602B0BDE8F0875C2172
:1065300001FB03F393FBF2F21B328DE700221A807A
:10654000E0E76821054806F091FC73680348198864
:1065500006F08CFE27E700BFC94216B2789FFF1FE6
:10656000602F0100549FFF1FDC9FFF1F743F01003D
:10657000F19FFF1F642F01004A9FFF1F2DE9F04F7D
:106580005A4E5B4DB6F900704C7855F8277085B0BF
:106590008146984604B10C78DFF874A11AB99AF8CC
:1065A0000030002B39D0534D002338462B808AF819
:1065B0000030FFF7B7FD504A504BB5F900000121FC
:1065C00011704FF6FF721A8060B301285ED001206F
:1065D00032232246019000934946494B3846FFF743
:1065E00099FE00240346B5F90020022A39DD002275
:1065F0002A80B6F900203D49002A3BDB052AC4BFAA
:1066000000220A80B8F1000F39D1002C0CBF1846C7
:106610004FF0FF3005B0BDE8F08F364DB5F9000002
:106620000028D2D1DFF8ECB0364ADBF8003012682F
:10663000C3EB0903934227D9334B1A78012A18BFB9
:1066400001201870FFF7F0F90123CBF80090012C1E
:106650002AD0042C35D0022C3AD0082C3ED000246D
:10666000C1E7C6D1FA68002AC1D0B6F900201F4997
:10667000002AC3DA05220A80B8F1000FC5D00393BF
:10668000FFF7E2FB039BC0E70346E0E74FF0000E95
:10669000142322468DE8084049461C4B3846744670
:1066A000FFF738FE03469EE732888AF80040013241
:1066B00032807A6982B10024384603939047039B65
:1066C00091E732880121013A32808AF80010F0E720
:1066D00001222A8000248CE7144684E77A6900218D
:1066E00029804FF0FF34002AE6D182E7509FFF1F38
:1066F000BC89FF1F549FFF1F4A9FFF1FB689FF1FC2
:106700004E9FFF1F743F0100F19FFF1F4C9FFF1F13
:10671000529FFF1FDC9FFF1F01210D2007F00ABCC5
:1067200000210D2007F006BC01460D2007F002BC39
:1067300008B50D2007F004FCB0FA80F149090D20DE
:10674000BDE8084007F0F6BB10B5002144080D2055
:1067500007F0F0FB204607F029FC0D20012107F08F
:10676000E9FB2046BDE8104007F020BC214A224B3F
:1067700010881B68984210B535DA204A1288141A1E
:106780009A42A8BF1A46B4F5157F22DA121A40F2CF
:10679000532303FB02F393FBF4F105310A2007F0C6
:1067A00039FA174B197801B3164B17491B6840F299
:1067B000271283F3070302FB03F381FB0321194430
:1067C000DB17C3EBA11105310920BDE8104007F02C
:1067D00021BA131A4FF41572611C02FB03F393FBE9
:1067E000F1F10531DAE70021D8E70920BDE81040D2
:1067F00007F010BA489DFF1F809CFF1F129FFF1FCC
:10680000049DFF1FF89EFF1F090402817F2838B5F1
:10681000A8BF7F200F4C4FF4167202FB00F284FBDE
:1068200002311144D2170546C2EBA1110A2007F02C
:10683000F1F97F3D4FF4967303FB05F384FB0321CD
:106840001944DB17A3EBA1110920BDE8384007F07C
:10685000E1B900BF09040281C368B3F9003030B563
:1068600083EAE374A4EBE374002BA0B218DB0123EA
:1068700000E0134603EB830252009442F9DA0A4D1A
:1068800090FBF3F285FB03E403FB1200DB173032CD
:10689000D3EBA40380B201F8012BF1D10B7030BD12
:1068A0002D230B700131E2E76766666638B5094D46
:1068B0008224204603F010F835F8021B00B288420B
:1068C000204601D002F0EEFF0234A4B28A2CF0D1AF
:1068D00038BD00BF389EFF1F024B8020198802F090
:1068E000E1BF00BFCC9CFF1F38B5094D782420467E
:1068F00002F0F2FF35F8021B00B28842204601D0B8
:1069000002F0D0FF0234A4B2802CF0D138BD00BF19
:10691000309EFF1F024B7620198802F0C3BF00BFD4
:10692000CA9CFF1F38B5094D4624204602F0D4FF0B
:1069300035F8021B00B28842204601D002F0B2FFB7
:106940000234A4B24E2CF0D138BD00BFBC9EFF1F54
:10695000024B4420198802F0A5BF00BFC09CFF1F56
:10696000024B4E20198802F09DBF00BFDE9CFF1F26
:10697000024B9A20198802F095BF00BF2C9DFF1F83
:10698000024B9820198802F08DBF00BFD29CFF1FD8
:10699000024B8C20198802F085BF00BF509EFF1F5C
:1069A000024B9C20198802F07DBF00BFB89CFF1FDE
:1069B000024BA020198802F075BF00BFC49EFF1FC4
:1069C000024B9620198802F06DBF00BFA09EFF1FEA
:1069D000024B8A20198802F065BF00BF669EFF1F28
:1069E000024B1020198802F05DBF00BF649EFF1F9C
:1069F000024B2C20198802F055BF00BFB69CFF1F28
:106A0000024B1E20198802F04DBF00BFD09CFF1F13
:106A1000C3680E20198802F045BF00BF024B282032
:106A2000198802F03FBF00BFBA9EFF1F024B6220D1
:106A3000198802F037BF00BFF09CFF1F024B642093
:106A4000198802F02FBF00BFB49EFF1F024BB42075
:106A5000198802F027BF00BF089FFF1F024BB62016
:106A6000198802F01FBF00BF349FFF1F024B5A203E
:106A7000198802F017BF00BF909CFF1F024B162021
:106A8000198802F00FBF00BF9C9CFF1F024B2E20F5
:106A9000198802F007BF00BF349DFF1F024B302052
:106AA000198802F0FFBE00BF209FFF1F024B9E20EF
:106AB000198802F0F7BE00BF9C89FF1F024BAC2073
:106AC000198802F0EFBE00BFB69EFF1F024BAE203A
:106AD000198802F0E7BE00BFDC9CFF1F024BB0200C
:106AE000198802F0DFBE00BF449EFF1F024BB22098
:106AF000198802F0D7BE00BFFA9CFF1F024B182076
:106B0000198802F0CFBE00BF4E9DFF1F024BA2208E
:106B1000198802F0C7BE00BFE69EFF1F024B1A2075
:106B2000198802F0BFBE00BFE89CFF1F024B1C206B
:106B3000198802F0B7BE00BFE09CFF1F024B662021
:106B4000198802F0AFBE00BFF49EFF1F024B7220F7
:106B5000198802F0A7BE00BF1C9FFF1F024B202018
:106B6000198802F09FBE00BFF29EFF1F024B322029
:106B7000198802F097BE00BFE29EFF1F024B6820FB
:106B8000198802F08FBE00BF209DFF1F024B6C20B2
:106B9000198802F087BE00BF849CFF1F024B522061
:106BA000198802F07FBE00BF3489FF1F024B5020BE
:106BB000198802F077BE00BF2089FF1F024B5420C6
:106BC000198802F06FBE00BFB089FF1F024B5C2026
:106BD000198802F067BE00BFB489FF1F024B5E2018
:106BE000198802F05FBE00BF2C89FF1F024B5620A0
:106BF000198802F057BE00BF229DFF1F244B1B883F
:106C00000B2B43D8DFE803F00B10151A1F24292E95
:106C100033383D06084604221E490BF0AFB908463A
:106C200004221D490BF0AAB9084604221B490BF0A7
:106C3000A5B9084604221A490BF0A0B90846042257
:106C400018490BF09BB90846042217490BF096B976
:106C50000846042215490BF091B90846042214494C
:106C60000BF08CB90846042212490BF087B908468C
:106C7000042211490BF082B9084604220F490BF097
:106C80007DB9084604220E490BF078B9704700BF61
:106C9000A09EFF1FD83701003C3501009C33010046
:106CA000C4380100A0330100AC380100A433010056
:106CB000A83301006C360100AC330100E437010059
:106CC000B0330100064B074A10B41C88064B084637
:106CD000002C14BF11461946042210BC0BF04EB90B
:106CE000009DFF1FB4330100B8330100064B074A73
:106CF00010B41C88064B0846002C14BF11461946D8
:106D0000042210BC0BF03AB9369DFF1FB4330100CA
:106D1000B8330100064B074A10B41C88064B0846DE
:106D2000002C14BF11461946042210BC0BF026B9E2
:106D30005A9EFF1FB4330100B8330100064B074AC7
:106D400010B41C88064B0846002C14BF1146194687
:106D5000042210BC0BF012B96A9EFF1FB43301006D
:106D6000B8330100064B074A10B41C88064B08468E
:106D7000002C14BF11461946042210BC0BF0FEB8BB
:106D8000A29EFF1FB4330100B8330100064B074A2F
:106D900010B41C88064B0846002C14BF1146194637
:106DA000042210BC0BF0EAB83E9DFF1FB433010073
:106DB000B83301001B4B1B880A2B0AD8DFE803F00D
:106DC0000A0E12161A1E22262A2E0600164B1868C4
:106DD00008607047154B186808607047144B1868B6
:106DE00008607047134B186808607047124B1868AA
:106DF00008607047114B186808607047104B18689E
:106E0000086070470F4B1868086070470E4B186891
:106E1000086070470D4B1868086070470C4B186885
:106E200008607047669EFF1FE0330100B833010021
:106E3000BC330100C0330100C4330100C83301007A
:106E4000CC330100D0330100D4330100D83301002A
:106E5000DC330100F0B52B4E2B4FDFF8C4E00546C4
:106E60000FCE87B06C460FC496E803003B68274AF4
:106E7000274F44F8040B40F6CC308342C8BF3A4653
:106E8000BEF800602180012E11889278ADF80D10B7
:106E90008DF80F202AD032D340F6CA02022E18BF36
:106EA00000229A4226DAA3F698031A491A4AC3EB3B
:106EB000031381FB03011944DB17C3EB6123243364
:106EC00082FB0321DA17C2EBA10202EB8201A3EBE2
:106ED0004103303330328DF813308DF8112069467C
:106EE000284616220BF04AF807B0F0BD40F698028B
:106EF0009A42D8DB094B1868CDF81100EFE740F64D
:106F0000FC02CEE7F4330100A89EFF1FE833010026
:106F1000E43301003B773B9867666666EC3301001B
:106F2000409EFF1FF8B5174C174E2278174D337847
:106F30002F888E46003218BF012201467046FFF7A7
:106F40001DFB002398423370237015DB14BF012012
:106F500000202B889F420ED040F23A72A3F5AF7307
:106F60000B490C4C02FB03F381FB0312DB17A3EB71
:106F7000621332332360F8BD0749012218460A70B4
:106F80002270E6E7888AFF1F659FFF1F0A9FFF1F89
:106F9000B5814E1BA089FF1FF09FFF1F014B187882
:106FA00002F018BCD89FFF1F014B187802F02CBCD0
:106FB0009090FF1F134BB3F9003030B583EAE374B0
:106FC000A4EBE374002BA0B218DB012300E013460E
:106FD00003EB830252009442F9DA0B4D90FBF3F27B
:106FE00085FB03E403FB1200DB173032D3EBA40371
:106FF00080B201F8012BF1D10B7030BD2D230B7045
:107000000131E2E79090FF1F67666666144BB3F9A3
:10701000003070B583EAE375A5EBE375002BACB2E5
:107020001ADB012300E0034603EB830040008542A6
:10703000F9DA0C4E94FBF3F086FB03E503FB1044F6
:10704000DB173030D3EBA503A4B201F8010BF1D16B
:1070500005480B70106070BD2D230B700131E0E707
:10706000909CFF1F676666660C340100134BB3F9F2
:10707000003030B583EAE374A4EBE374002BA0B2D4
:1070800018DB012300E0134603EB83025200944215
:10709000F9DA0B4D90FBF3F285FB03E403FB1200DE
:1070A000DB173032D3EBA40380B201F8012BF1D10E
:1070B0000B7030BD2D230B700131E2E79C89FF1F5F
:1070C00067666666134BB3F9003030B583EAE37444
:1070D000A4EBE374002BA0B218DB012300E01346FD
:1070E00003EB830252009442F9DA0B4D90FBF3F26A
:1070F00085FB03E403FB1200DB173032D3EBA40360
:1071000080B201F8012BF1D10B7030BD2D230B7033
:107110000131E2E7DC9CFF1F67666666134BB3F93B
:10712000003030B583EAE374A4EBE374002BA0B223
:1071300018DB012300E0134603EB83025200944264
:10714000F9DA0B4D90FBF3F285FB03E403FB12002D
:10715000DB173032D3EBA40380B201F8012BF1D15D
:107160000B7030BD2D230B700131E2E7FA9CFF1F3D
:1071700067666666134BB3F9003030B583EAE37493
:10718000A4EBE374002BA0B218DB012300E013464C
:1071900003EB830252009442F9DA0B4D90FBF3F2B9
:1071A00085FB03E403FB1200DB173032D3EBA403AF
:1071B00080B201F8012BF1D10B7030BD2D230B7083
:1071C0000131E2E7E69EFF1F67666666134BB3F97F
:1071D000003030B583EAE374A4EBE374002BA0B273
:1071E00018DB012300E0134603EB830252009442B4
:1071F000F9DA0B4D90FBF3F285FB03E403FB12007D
:10720000DB173032D3EBA40380B201F8012BF1D1AC
:107210000B7030BD2D230B700131E2E73489FF1F65
:1072200067666666134BB3F9003030B583EAE374E2
:10723000A4EBE374002BA0B218DB012300E013469B
:1072400003EB830252009442F9DA0B4D90FBF3F208
:1072500085FB03E403FB1200DB173032D3EBA403FE
:1072600080B201F8012BF1D10B7030BD2D230B70D2
:107270000131E2E72089FF1F67666666134BB3F9A9
:10728000003030B583EAE374A4EBE374002BA0B2C2
:1072900018DB012300E0134603EB83025200944203
:1072A000F9DA0B4D90FBF3F285FB03E403FB1200CC
:1072B000DB173032D3EBA40380B201F8012BF1D1FC
:1072C0000B7030BD2D230B700131E2E7B089FF1F39
:1072D00067666666134BB3F9003030B583EAE37432
:1072E000A4EBE374002BA0B218DB012300E01346EB
:1072F00003EB830252009442F9DA0B4D90FBF3F258
:1073000085FB03E403FB1200DB173032D3EBA4034D
:1073100080B201F8012BF1D10B7030BD2D230B7021
:107320000131E2E7B489FF1F67666666134BB3F964
:10733000003030B583EAE374A4EBE374002BA0B211
:1073400018DB012300E0134603EB83025200944252
:10735000F9DA0B4D90FBF3F285FB03E403FB12001B
:10736000DB173032D3EBA40380B201F8012BF1D14B
:107370000B7030BD2D230B700131E2E72C89FF1F0C
:107380006766666608B5B82002F0A6FA044B19884D
:10739000884204D0B820BDE8084002F083BA08BD96
:1073A000989CFF1F08B5702002F096FA044B1988CC
:1073B000884204D07020BDE8084002F073BA08BDCE
:1073C000409EFF1F08B5742002F086FA044B19880E
:1073D000884204D07420BDE8084002F063BA08BDBA
:1073E000D89EFF1F054B1B880846042213B9044989
:1073F0000AF0C4BD03490AF0C1BD00BFDE9CFF1FF7
:1074000014340100103401000E4B1B88032B17D8D5
:10741000DFE803F0110C0702084604220A490AF0CB
:10742000ADBD0846042209490AF0A8BD0846042259
:1074300007490AF0A3BD0846042206490AF09EBD8A
:10744000704700BF509EFF1F24340100203401000C
:107450001C3401001834010010B40A4B0A4C0A46CF
:1074600093E8030083B0238802AC04E9030004EB33
:107470008303104653F8081C052203B010BC0AF021
:107480007DBD00BFE42F0100B49EFF1F30B40A4B46
:107490000A4D0C4693E8070084B02B8804AD05E93B
:1074A000070005EB8303204653F80C1C042204B0AC
:1074B00030BC0AF063BD00BFEC2F0100409EFF1FEF
:1074C000F0B40C4D0C4F0E460FCD8CB001AC0FC478
:1074D0000FCD0FC495E807003B8884E807000CAA8D
:1074E00002EB8303304653F82C1C04220CB0F0BC92
:1074F0000AF044BDF82F0100969EFF1F30B50A4BDD
:107500000A4D0C460FCB85B00DF1100E0EE90F00A1
:107510002B880EEB8303204653F8101C042205B081
:10752000BDE830400AF02ABD34300100B69EFF1F8E
:1075300030B50A4B0A4D0C460FCB85B00DF1100E3D
:107540000EE90F002B880EEB8303204653F8101C26
:10755000042205B0BDE830400AF010BD343001000F
:10756000449EFF1FF0B40B4D0B4F0E460FCD86B05F
:107570006C460FC495E803003B8884E8030006AA24
:1075800002EB8303304653F8181C042206B0F0BC0B
:107590000AF0F4BC443001004E9DFF1FF0B40A4DC8
:1075A0000A4F0E460FCD86B001AC0FC42A683B8847
:1075B000226006AA02EB8303304653F8141C0C2207
:1075C00006B0F0BC0AF0DABC5C300100E09CFF1FA2
:1075D000F0B40B4D0B4F0E460FCD88B06C460FC468
:1075E00095E80F0084E80F003B8808AA02EB8303AC
:1075F000304653F8201C042208B0F0BC0AF0BEBC90
:1076000070300100D89EFF1F164B1B880BB31BB2B6
:1076100083EAE370A0EBE370002B30B584B21DDB8E
:10762000012300E0134603EB830252009042F9DA93
:107630000D4894FBF3F280FB03E503FB1244DB17D8
:107640003032D3EBA503A4B201F8012BF1D10B70BA
:1076500030BD0846042205490AF090BC2D230B706A
:107660000131DDE7209DFF1F676666662834010053
:1076700030B50A4B0A4D0C460FCB85B00DF1100EFC
:107680000EE90F002B880EEB8303204653F8101CE5
:10769000042205B0BDE830400AF070BC9030010013
:1076A000849CFF1F054B1B881BB9054B186808609D
:1076B00070470846042203490AF060BC2C9DFF1F56
:1076C000B8330100B4330100164B1B880BB31BB257
:1076D00030B583EAE374A4EBE374002BA0B21CDBA7
:1076E000012300E0134603EB830252009442F9DACF
:1076F0000D4D90FBF3F285FB03E403FB1200DB1757
:107700003032D3EBA40380B201F8012BF1D10B701E
:1077100030BD064B1868086070472D230B7001318F
:10772000DEE700BFD09CFF1F67666666B8330100C6
:10773000164B1B880BB31BB230B583EAE374A4EB82
:10774000E374002BA0B21CDB012300E0134603EB23
:10775000830252009442F9DA0D4D90FBF3F285FB5F
:1077600003E403FB1200DB173032D3EBA40380B237
:1077700001F8012BF1D10B7030BD064B1868086081
:1077800070472D230B700131DEE700BF989CFF1F6F
:1077900067666666B8330100164B1B880BB31BB2D5
:1077A00030B583EAE374A4EBE374002BA0B21CDBD6
:1077B000012300E0134603EB830252009442F9DAFE
:1077C0000D4D90FBF3F285FB03E403FB1200DB1786
:1077D0003032D3EBA40380B201F8012BF1D10B704E
:1077E00030BD064B1868086070472D230B700131BF
:1077F000DEE700BFA69EFF1F67666666B83301001E
:10780000164B1B880BB31BB230B583EAE374A4EBB1
:10781000E374002BA0B21CDB012300E0134603EB52
:10782000830252009442F9DA0D4D90FBF3F285FB8E
:1078300003E403FB1200DB173032D3EBA40380B266
:1078400001F8012BF1D10B7030BD064B18680860B0
:1078500070472D230B700131DEE700BF9C9CFF1F9A
:10786000676666662C340100174B1B881BB31BB27E
:1078700070B583EAE375A5EBE375002BACB21EDBB4
:10788000012300E0034603EB830040008542F9DA60
:107890000E4E94FBF3F086FB03E503FB1044DB176D
:1078A0003030D3EBA503A4B201F8010BF1D10848A5
:1078B0000B70106070BD074B1868086070472D236F
:1078C0000B700131DCE700BF349DFF1F6766666601
:1078D00030340100B8330100164B1B880BB31BB2C8
:1078E00030B583EAE374A4EBE374002BA0B21CDB95
:1078F000012300E0134603EB830252009442F9DABD
:107900000D4D90FBF3F285FB03E403FB1200DB1744
:107910003032D3EBA40380B201F8012BF1D10B700C
:1079200030BD064B1868086070472D230B7001317D
:10793000DEE700BF209FFF1F67666666B833010061
:10794000164B1B880BB31BB230B583EAE374A4EB70
:10795000E374002BA0B21CDB012300E0134603EB11
:10796000830252009442F9DA0D4D90FBF3F285FB4D
:1079700003E403FB1200DB173032D3EBA40380B225
:1079800001F8012BF1D10B7030BD064B186808606F
:1079900070472D230B700131DEE700BFF49EFF1FFF
:1079A00067666666B8330100164B1B880BB31BB2C3
:1079B00030B583EAE374A4EBE374002BA0B21CDBC4
:1079C000012300E0134603EB830252009442F9DAEC
:1079D0000D4D90FBF3F285FB03E403FB1200DB1774
:1079E0003032D3EBA40380B201F8012BF1D10B703C
:1079F00030BD064B1868086070472D230B700131AD
:107A0000DEE700BF1C9FFF1F67666666B833010094
:107A1000174B1B881BB31BB270B583EAE375A5EB4C
:107A2000E375002BACB21EDB012300E0034603EB41
:107A3000830040008542F9DA0E4E94FBF3F086FB9A
:107A400003E503FB1044DB173030D3EBA503A4B2EE
:107A500001F8010BF1D108480B70106070BD074BA5
:107A60001868086070472D230B700131DCE700BFF8
:107A7000F29EFF1F6766666630340100B83301006E
:107A8000054B1B881BB1054B186808607047044BF9
:107A900018680860704700BF229DFF1F4434010032
:107AA0004034010070B5FAF735FB164B1B7813B163
:107AB000154C237833B9154B1020198801F0F2FECC
:107AC000012070BD124D134E2B783288B3FA83F328
:107AD00082F008025B09114642202B70328001F0CF
:107AE000E1FE23780BB12B782BB90021212006F081
:107AF00021FA002070BD0121212006F01BFA002090
:107B000070BD00BF949EFF1F469EFF1F649EFF1F17
:107B1000629EFF1F149FFF1F184B1A8852B3184A0A
:107B2000128830B50A80B3F90030002B83EAE37481
:107B3000A4EBE374BCBF2D238B70A0B2ACBF0231A9
:107B40000331012300E0134603EB83025200944209
:107B5000F9DA0C4D90FBF3F285FB03E403FB120012
:107B6000DB173032D3EBA40380B201F8012BF1D143
:107B70000B7030BD044B186808607047E89CFF1F0D
:107B80004834010067666666B833010070B53C4D45
:107B90002B780646002B35D11C4673780BB920464E
:107BA00070BDFAF7B7FA374A374B38481278317850
:107BB0001B78007802EB43034A1E03EB80030E2A76
:107BC000EDD801A050F822F0317C0000537C000079
:107BD0009F7B0000317C00009F7B00009F7B0000AA
:107BE0009F7B00001F7C00009F7B00009F7B0000AC
:107BF0009F7B00009F7B00009F7B00009F7B00001D
:107C00001B7C0000AE21224803F0F6FF204804F060
:107C100043FA00232B700124BFE706F0B1FEAF2129
:107C20001B4803F0E9FF1B4A012313702B70B6E7D2
:107C300083B91948038804294FF6FF7103F1FF3215
:107C40000CBF01230B46134403F07F030133038071
:107C50000FE073B1013B114A32F813304BB10E4EB5
:107C60000F481049104A33800123002606700B701C
:107C70001370084A0221012311702B70204670BD39
:107C8000888AFF1F459FFF1F469FFF1FE89EFF1F1B
:107C9000789FFF1FF09FFF1FE49EFF1F209EFF1F86
:107CA000189DFF1FA49CFF1FF39FFF1F10B5064BDD
:107CB000064C1A882046012101F0E2FD218842206D
:107CC000BDE8104001F0EEBD009DFF1F149FFF1F97
:107CD00010B5064B064C1A882046022101F0D0FD53
:107CE00021884220BDE8104001F0DCBD369DFF1F19
:107CF000149FFF1F10B5064B064C1A88204604211E
:107D000001F0BEFD21884220BDE8104001F0CABD4F
:107D10005A9EFF1F149FFF1F10B5064B064C1A8872
:107D20002046062101F0ACFD21884220BDE810402C
:107D300001F0B8BD6A9EFF1F149FFF1F10B5064BD0
:107D4000064C1A882046002101F09AFD2188422025
:107D5000BDE8104001F0A6BDA29EFF1F149FFF1FAB
:107D600008B5122001F0B8FD054B1988884206D0ED
:107D7000122001F097FDBDE8084001F05DBC08BD90
:107D8000969EFF1F08B5582001F0A6FD054B1988E7
:107D9000884206D0582001F085FDBDE8084001F07A
:107DA0004BBC08BDA69EFF1F08B5142001F094FD32
:107DB000054B1988884206D0142001F073FDBDE8F8
:107DC000084001F039BC08BD3E9DFF1FF0B480EAB9
:107DD000E075A5EBE0750028ACB21FDB1DBF2B23BF
:107DE0000B704E1C0E46012300E0134603EB83028A
:107DF00052009542F9DA0B4F94FBF3F287FB03052F
:107E000003FB1244DB173032D3EBA503A4B206F810
:107E1000012BF1D133700846F0BC70472D230B7055
:107E20004E1CE0E7676666661A4B18880C2815D06A
:107E3000192817D01A2819D01B281BD01C281DD090
:107E40001D281FD01E2821D01F2803D00C3800B2B7
:107E5000FFF7BCBF104A1068086070470F4A1068EF
:107E6000086070470E4A1068086070470D4A106835
:107E7000086070470C4A1068086070470B4A106829
:107E8000086070470A4A106808607047094A10681D
:107E900008607047E29EFF1F6C34010050340100FF
:107EA00054340100583401005C3401006034010096
:107EB0006434010068340100034B1888A0EB800093
:107EC000400000B2FFF782BFD89FFF1F024B188807
:107ED000643800B2FFF77ABF349FFF1F024B188847
:107EE000643800B2FFF772BF089FFF1F024BB3F95F
:107EF0000000FFF76BBF00BFF09CFF1F024B18880C
:107F0000033800B2FFF762BFBA9EFF1F024B18880A
:107F10000C3800B2FFF75ABF969CFF1F024B18881F
:107F2000183800B2FFF752BFCC9CFF1F024B1888D5
:107F3000183800B2FFF74ABFCA9CFF1F024B1888CF
:107F4000183800B2FFF742BFC09CFF1FC3681888F3
:107F5000183800B2FFF73ABF054B1B881BB9054B19
:107F60001868086070470846042203490AF006B8FA
:107F7000C49EFF1FB8330100B4330100054B1B88BA
:107F80001BB9054B1868086070470846042203496E
:107F900009F0F4BFD29CFF1FB8330100B4330100D5
:107FA00030B5134C85B001252B463C2202212046DA
:107FB000009503F097FE204604F06EF80022402161
:107FC000802320460191009311460A4B029504F04C
:107FD00011FD204604F06CF907480849084A0023BF
:107FE000036083800B608B801360938005B030BD8D
:107FF000789FFF1F083B0100589FFF1F709FFF1FC6
:10800000E09FFF1F10B500EBC00000F10F02D2B2DD
:1080100093B284B09C1E981C3D2303918DE81900F7
:108020003921024804F04AFC04B010BD789FFF1FBC
:10803000014B01221A707047659FFF1FF0B57A4B04
:108040007A4C7B4F7B4E7C4D85B004228DE80C0032
:1080500002932046794B4022802103F04BFC2046BE
:10806000774A7849784C09F0F1F8784A784B97616B
:10807000784FD761784F9F61784FDF61784FB76154
:10808000784FF761784FAF61784FEF61784FA76114
:108090007848794FE761794F87617949794FC761AE
:1080A000794F8F61794A7A4FCF617A4F97617A4BD6
:1080B0007A4FD7617A4F9F617A4E7B4FDF617B4F5A
:1080C0007B4DB7617B4FF7617B4F7C4CAF617C4F41
:1080D000EF617C4F7C48A7617C4FE7617C4F7D4915
:1080E00087617D4FC7617D4F7D4A8F617D4FCF6135
:1080F0007D4F7E4B97617E4FD7617E4F7E4E9F6155
:108100007E4FDF617E4FB7617E4D7F4FF7617F4FBE
:10811000AF617F4C7F4FEF617F4FA7617F48804FFA
:10812000E761804F87618049804FC761804F8F61D1
:10813000804A814FCF61814F9761814B814FD761D9
:10814000814F9F61814E824FDF61824FB761824DC7
:10815000824FF761824FAF61824C834FEF61834F53
:10816000A7618348834FE761834F84498761844FC8
:10817000C761844F844A8F61844FCF61844F854BA0
:108180009761854FD761854F854E9F61854FDF6130
:10819000854F864DB761864FF761864F864CAF613C
:1081A000864FEF61864F8748A761874FE761874F0A
:1081B00087618749874FC761874F8F61874A884F9B
:1081C000CF61884F9761884B884FD761884F9F61F7
:1081D000884E894FDF61894F894DB761894FF761BB
:1081E000894F8A4CAF618A4F8A488B49EF618B4F28
:1081F0008B4DA761E5618B4F8B4D8C4CDFF850E2C6
:108200008B4A8C4B8761C5618C618B4E8B4F8C4D3B
:108210008C4CC1F81CE08C488C499761D5619C61FD
:10822000D861B16005B0F0BD40420F00789FFF1FDC
:108230000D7F0000748EFF1F0090FF1F6491FF1FD1
:108240001C89FF1F4DB900004C8FFF1FF889FF1FCD
:10825000288FFF1F116A0000FD7E00001D6A0000CC
:10826000C56C0000AD7C0000ED6C0000D17C00000E
:10827000156D00001C8AFF1FF57C0000ED7E0000DC
:108280007C8CFF1F2D6A00003D6D0000308DFF1FAC
:10829000197D000059740000588CFF1F3D6A0000D2
:1082A000656D0000548DFF1F3D7D0000DD7E0000E8
:1082B000F890FF1F4D6A0000CD7E0000D490FF1F94
:1082C0005D6A0000317700000C8DFF1F8573000090
:1082D000B97E0000E88CFF1F9D6F0000B56F0000A5
:1082E000048FFF1FA96F00008D740000A48BFF1F77
:1082F000A5730000C1740000B88FFF1F617D0000EE
:1083000099770000348CFF1F857D00000D70000000
:10831000648BFF1F6D6A00008D6D00006C90FF1F65
:10832000A97D000001780000108CFF1F7D6A00000D
:10833000697800009C8DFF1F8D6A0000D9780000CD
:10834000EC8BFF1F9D6A00006D7000001C8BFF1FEF
:10835000AD6A0000FD7400002490FF1FBD6A00009C
:10836000C5700000BC8EFF1FCD6A00003175000093
:10837000F88AFF1FDD6A00001D710000788DFF1F65
:10838000ED6A000065750000408AFF1FFD6A00006D
:1083900075710000A08CFF1F0D6B0000197B0000A1
:1083A000E08EFF1F1D6B00009D7500002891FF1FD0
:1083B0002D6B000041790000508EFF1F3D6B0000C7
:1083C000A9790000D48AFF1F4D6B0000D175000011
:1083D000DC8FFF1FC5730000117A0000988EFF1F0D
:1083E0005D6B0000297E0000B08AFF1F6D6B0000EE
:1083F000097600008C8AFF1F7D6B000071760000FB
:10840000C48CFF1F8D6B0000CD710000C88BFF1F57
:108410009D6B0000648AFF1F408BFF1F25720000C8
:10842000AD6B00007D720000BD6B0000D5720000D6
:10843000708FFF1FD489FF1F1C91FF1F2D73000039
:10844000DD6B0000817A0000ED6B0000158A0000F2
:10845000CD6B0000F0B5461C83B00D460127032309
:1084600036B22AB2044631468DE888002348ADB2C0
:1084700004F0BAF90C23AA1C12B200930197052349
:1084800021B21E4804F0B0F91D4A1E4B12881B6829
:10849000BA422AD023D3022A10D11B4CA3F6CA0316
:1084A00084FB03241C44DB17C3EB24140A2CA8BF51
:1084B0000A2424EAE474A2B223B202E000231A469A
:1084C0001C460D35AA1A01200093019012B23146C4
:1084D00003230A4804F006F9204603B0F0BD0B4C14
:1084E000A3F6FC0384FB0324DDE7094CA3F6980301
:1084F00084FB0324DB17C3EBA404D7E7789FFF1F9B
:10850000409EFF1FA89EFF1F09CB3D8D1F85EB518D
:10851000398EE3382DE9F0438FB283B0DFF84C8019
:10852000BD1D461D2DB204B236B24FF001090AB28C
:108530002346314640460095CDF8049004F004F9F6
:108540002A463346214640468DE8200204F0FCF8D6
:1085500007F10C020095334612B22146CDF8049083
:10856000404604F0F1F803B0BDE8F083789FFF1FA8
:108570002DE9F043804685B0002956D101213048CD
:1085800004F078FC2F4998F8062098F8083011F884
:108590000290994522DA4FEA89064D460C24D8F814
:1085A0000C3027489B595F6822B2002104F05EFC22
:1085B000384609F025FC39460246214804F0F0FD12
:1085C0001F4804F003FE98F8083001350934AB4227
:1085D000A4B206F1040601DD422CE0D1B9F1000F8E
:1085E00013D109F1060999450CDA3C2301213B22FC
:1085F000039102930093019239233F223A211048BC
:1086000004F05CF905B0BDE8F0830F2301213B22A3
:10861000039102930093019239230C223A210848D6
:1086200004F04CF998F80830DBE70021342300937C
:1086300001913F230C22024804F054F89EE700BF4A
:10864000789FFF1F709FFF1F10B5104C012120461F
:1086500004F016FC2046012104F00CFC20463422D4
:10866000552104F003FC20460222094904F098FD3C
:1086700020460522074904F093FD204604F0A6FD9C
:108680002046BDE8104003F013BE00BF789FFF1FD7
:10869000B8340100BC34010070B50D46064609F03F
:1086A000AFFB00EB40008400002D36D0284609F0D7
:1086B000A7FB00EB4000400023185B1003F16001B2
:1086C000091A282209B21748C3F1600404F0CEFB4E
:1086D0000121144804F0CEFB284609F091FB2946FD
:1086E0000246104804F05CFD0E4804F06FFD0221C4
:1086F0000C4804F0BFFB21B221220A4804F0B6FB6B
:10870000304609F07DFB31460246064804F048FD3C
:108710000448BDE8704004F059BD6410C4F1600421
:10872000E5E700BF789FFF1F10B50D4B1B5C51F8AC
:108730002340237884B013B1012004B010BD04AAF3
:1087400001A942F8103D2046A3699847A38A9B07D8
:10875000F2D401A80099FFF79FFF012004B010BDDB
:10876000589FFF1F2DE9F04F2F4DDFF8CCB0DFF8F9
:10877000C4A0DFF8C8900FCD91B003AC0FC40FCDEB
:108780000FC40FCD0FC42B6823600025A8462F46C9
:108790002E4600E09846BAF8003024495BF82320C2
:1087A00028461123F8F708F800EBC00400EB84001A
:1087B00089FB00340444C017C0EB6434C4F13C00AE
:1087C000C6F13C0207F14101012600B208F1410364
:1087D00000901BB2019612B209B2154803F0B4FF23
:1087E00008EB060305F211153C2B2646ADB24746B1
:1087F000D0D134226B210E4804F038FB00210C4804
:1088000004F038FB0B4B1B8810AA02EB830353F8D0
:10881000344C204609F0F4FA02460548214611B0CE
:10882000BDE8F04F04F0BCBCA0300100402A0100BC
:10883000789FFF1FB69CFF1FA4280100090002803B
:10884000234B70B5B3F9003083EAE374A4EBE3740F
:10885000002B82B0A1B234DB68466D46012300E0F4
:10886000134603EB830252009442F9DA194E91FB4E
:10887000F3F286FB03E403FB1211DB173032D3EB78
:10888000A40389B205F8012BF1D119462B70FFF72B
:1088900003FF114B1B7813B1104B1B780BB902B0BF
:1088A00070BD01210E4804F0E5FA332264210C4822
:1088B00004F0DCFA04220B49094804F071FC02B010
:1088C00070BD2D238DF800300DF101056846C5E718
:1088D000649EFF1F67666666469EFF1F629EFF1FBF
:1088E000789FFF1FC434010010B5424C424882B04B
:1088F00003F0D2FB2378C3B906213F4804F0BAFA4B
:108900002378012B37D90A22022B11463A486BD023
:1089100004F0ACFA39490322374804F041FC3648E8
:1089200002B0BDE8104004F051BC354B1A7801216B
:108930000523002A35D10191009311462E4803F0FA
:1089400053FF304B1A78002A36D0052301220192BA
:10895000009300220A21284803F0C4FE2A4B1A780B
:10896000002A35D1012105230191009314212248C9
:1089700003F03AFFC0E7254C2388092B32D9632B3B
:108980008CBF0A211F210A221B4804F06FFA21889C
:10899000194804F06BFC184802B0BDE8104004F020
:1089A00015BC0022019100931146134803F09AFE72
:1089B000144B1A78002AC8D1052301210191009394
:1089C0000A210D4803F010FF0F4B1A78002AC9D076
:1089D000012205230192009300221421064803F08E
:1089E00081FE89E73021CEE704F040FA03220849EE
:1089F00092E700BFF39FFF1F789FFF1FD034010055
:108A0000459FFF1F469FFF1FE89EFF1FE49EFF1F1D
:108A1000CC340100F8B56D4D287840B96C4B1B681B
:108A200099425CD36B4A012313702B70F8BD0C463E
:108A300000266948664F03F02FFB04F6AC5332461C
:108A400065483B6031212E7004F010FA0121624824
:108A5000624D04F015FA31465F4804F00BFA052226
:108A60005F495D4804F09CFB5B4804F0AFFB0C22BF
:108A70001021594804F0FAF90B225A49564804F0DB
:108A80008FFB05225849544804F08AFB524804F0F1
:108A90009DFB564B50481C68A4F69803C3EB031388
:108AA00085FB03251D441021DB172022C3EB652520
:108AB00004F0DCF940F6CC339C4205F124054FF07C
:108AC00022014FF004000BDCFFF7C4FC484B1C886C
:108AD000064674B3012C46D0022C41D00120F8BDCB
:108AE000FFF718FD092243493B4804F059FB2A22AD
:108AF0001021394804F0BAF93F4C374884FB05345B
:108B0000EB17C3EBA404214604F0B0FB01223B4960
:108B1000314804F045FB04EB8401A5EB41012E48EC
:108B200004F0A4FB012236492B4804F039FB012054
:108B3000F8BD34491022284804F032FB264804F0DE
:108B400045FB2A221021244804F090F9314622489E
:108B500004F08CFB07222C491F4804F021FBCBE7D3
:108B60000C222A49E7E70C2229491B4804F018FB8C
:108B7000194804F02BFB2A221021174804F076F93B
:108B8000314615481C4E04F071FB07221E4912485D
:108B900004F006FB86FB0536EB17C3EBA606314651
:108BA0000D4804F063FB224614490B4804F0F8FA20
:108BB00006EB8601A5EB4101074804F057FB22466E
:108BC0000F49054804F0ECFA2046F8BD888AFF1FDB
:108BD0006C9FFF1FF09FFF1F789FFF1F3B773B9805
:108BE000D4340100DC340100BC340100A89EFF1F16
:108BF000409EFF1FE834010067666666F040010092
:108C000068400100F43401000835010020350100FE
:108C1000103501002DE9F041754C2278002A0546F7
:108C20000F4614BF4FF001084FF000084ED1714EAF
:108C30003368CB1AB3F5FA6F04D86B78A3B9404602
:108C4000BDE8F0816C4B6D486D49DFF8D0E11A70DA
:108C5000012303700988237026208EF8002000F07D
:108C600021FE6B78002BEAD03760F9F753FA654A9A
:108C7000654B6649127828781B78097802EB430324
:108C8000421E03EB81030E2AD9D801A151F822F02C
:108C9000818D00004D8D00003F8C0000818D000013
:108CA0003F8C00003F8C00003F8C0000358D0000A1
:108CB0003F8C0000E78C00003F8C00003F8C0000E0
:108CC0003F8C00003F8C0000E38C0000AF21504837
:108CD000484E02F091FFFFF707FE00233760237034
:108CE000ABE705F04DFE4A4803F0D6F902214848AB
:108CF00004F0C0F80F222321454804F0B7F80522FC
:108D00004449434804F04CFA414804F05FFA1E22FB
:108D100023213F4804F0AAF805223F493C4804F0CB
:108D20003FFA3B4804F052FA394803F0C1FA00F028
:108D3000D3FC84E7394D2B78012B50D9304B2620BA
:108D4000198800F0AFFD00232B7078E7002B3FF46B
:108D500076AF013B324A32F81330002B3FF46FAF4D
:108D6000274C304825492D4A23804FF00108002325
:108D7000037081F8008082F80080FFF7B5FD5EE7A0
:108D800093B1013B264A32F8131019B31C4B254D01
:108D90001A4C224A19800026012326202E702370A7
:108DA000137000F07FFD15E0154C1E4922880B70F2
:108DB00004284FF6FF7002F1FF310CBF012202467A
:108DC0000A440E4E154D02F07F020132012122802D
:108DD00031702B70FFF788FD4FF001082FE706492F
:108DE000064A01230020087013702370A6E700BF15
:108DF000888AFF1FEC9FFF1FF09FFF1FA49CFF1F8F
:108E0000E49EFF1F459FFF1F469FFF1FE89EFF1F19
:108E1000789FFF1F3035010038350100F39FFF1F99
:108E2000209EFF1F189DFF1F2DE9F04F05468BB0B8
:108E30000F46AD480121164604F022F8AA8812F028
:108E4000010440F0B080DFF8CC8298F80030002BAD
:108E50007DD1AB79A54AD15CA1B9DFF8BCA2797804
:108E60001AF8039041B339780139072900F2B78025
:108E7000DFE811F0F1005401B5006C01B500B50058
:108E8000B500E9007C78002C00F0CA800139EC685C
:108E9000387854F82170FC68411EB4F80080072926
:108EA00000F2A780DFE811F074015901A5006C0100
:108EB000A500A500A5009F00DFF854A2DAF8002065
:108EC000B21AB2F5967F75D9894A107801281ABF6F
:108ED000012010701170874A18BF0146D05CC0EBAA
:108EE0000900C0B2FFF78EF80124CAF80060AB8811
:108EF0009B0770D57B78002B6DD0F9F70BF97E4B73
:108F00007E4A7F481B78127839780078022515FB55
:108F100002330A2903EB800300F04E810C295AD159
:108F2000002B58D003F11900764E774A013B0021FF
:108F3000400080B226F813100123157088F8003025
:108F400000F0B0FC714B032220461A702FE06648F7
:108F500003F0A2F80121644803F08CFF6248224626
:108F6000214603F083FFAB88580725D42C682046A0
:108F700008F046FF214602465B4804F011F95A48C2
:108F800004F024F9092201238DE80C0000217F233D
:108F9000554803F0D9FB00212846FFF7E9FA0023E2
:108FA00088F8003055E7AB683146384698470BB033
:108FB000BDE8F08F0846FAE72B6804A8984704A894
:108FC00008F01EFF04A90246474804F0E9F84648A5
:108FD00004F0FCF8D6E720460BB0BDE8F08F002483
:108FE0000AF8039083E70021D1543846FB6998477B
:108FF000FC68A4F80080002725223C238DE884002B
:1090000041211822384803F06DFBE968A879FFF781
:109010008BFB374A3E4B17701E600BB0BDE8F08FDC
:109020003B490A68B21AB2F5967FD4D9304F0E6028
:109030003E78012E00F0B480E968184601233B70A9
:10904000FFF772FBB3E7304AE9791170012288F823
:1090500000200024C4E72A7A013A4A45BFDD09F11D
:109060000104E4B2A145BAD0224E16F803B0CBEB0E
:109070000900C0B20021FEF7C5FF2B7A052BD946A7
:109080001BD9CBEB0402042A40F3AE80A4F1040BFD
:10909000BBF1000FC0F2B080063B5B45A8BF5B464A
:1090A0005FFA83F9AA791348B15C994205D000F8B8
:1090B000029001212846FFF75BFAC9EB0400C0B219
:1090C00001210B4EFEF79EFF0021342301910093F6
:1090D0000548317040230B223F21A14603F002FBDB
:1090E0000124AB797CE700BF789FFF1FE09FFF1F43
:1090F000F19FFF1F709FFF1F459FFF1F469FFF1F90
:10910000E89EFF1F209EFF1FF09FFF1FF39FFF1F82
:10911000DC9FFF1F888AFF1F589FFF1F0FFA89F1EE
:10912000E868604C50F821602168049134785E4909
:1091300004980860002C71D0012C7FF450AF5B4A7A
:10914000317A88F800401170002449E7B9F1000F26
:1091500050D009F1FF34E4B284E7B98A01F0040188
:1091600089B200293FF440AF3B6A03929847039AC3
:1091700000283FF43DAFAB79FC680021D15438E7BB
:109180007B8A43453CD908F101081FFA88F830E78B
:109190003B8A43453BD208F1FF381FFA88F828E79D
:1091A00025238DE8180042483C703C2318224121B9
:1091B00003F098FA3046FAE6002B3FF40CAF3D4A34
:1091C0003D4E1188394A03F11900013B400080B23D
:1091D00026F81310012388F80030157000F062FBA8
:1091E000364B20461D70E2E6002A3FF755AF04F1EA
:1091F000FF3B4DE74C46F3E64FF000094B4651E785
:10920000BB8ADA077FF5F5AEB7F81080F1E6BB8AC6
:10921000D9077FF5EEAEB7F81280EAE62849C85CB8
:10922000C0EB090009F1010EC0B201214FF0340B6F
:1092300002F803E0FEF7E6FEB6681D4801944023FD
:109240000B223F210124CDF800B003F04BFA40235C
:109250000B223F211648CDF800B0019403F0C4FA68
:109260002146134803F006FE304608F0C9FDA0EB86
:10927000800000F15F0109B20F220D4803F0F6FDF6
:10928000304608F0BDFD31460246094803F088FF2C
:10929000074803F09BFFE968A879FFF745FAAB7927
:1092A0009EE600BF30A0FF1FDC9FFF1FF09FFF1F47
:1092B000789FFF1FE49EFF1F209EFF1FF39FFF1F4D
:1092C000709FFF1F2DE9F047DFF808926D4B99F86A
:1092D00000601B68DFF800A282B0003601934FF0F7
:1092E000030018BF0126019F9AF8008004F028FEB1
:1092F0000546042004F024FE0446052004F020FE68
:10930000800040EA4404062004F01AFE2C4364B2B4
:109310005D4944EAC0000A7880F00F03DBB29A424C
:109320005A4A3CD01760002259480B7003788DF8D8
:1093300000808DF8012053B3564A12684EF6602122
:10934000BA1A8A4219D8022B59D0012B5FD0062BAA
:1093500048D0032B63D0042B69D0052B77D0072B83
:109360007DD0082B00F08380092B68D016B14A48C5
:1093700002F09EFF02B0BDE8F087484A484C002347
:109380000121237003701360938089F800103A461E
:1093900069464448FFF748FD3043C6B2E6E7126825
:1093A000BA1A1E2A6BD99AF80020934222D0394C5F
:1093B0003D488AF80030012B276082EA03020760EB
:1093C0009846B1D0042BAFD137480068381AB0F5B1
:1093D000C87FA9D9354C2068381A3228A4D927600B
:1093E0001A46A1E73A4669463148FFF71DFD30436A
:1093F000C6B2BBE7012B4FF00002E3D1E4E73A46E7
:1094000069462C48FFF710FD3043C6B2AEE73A4636
:1094100069462948FFF708FD3043C6B2A6E73A4639
:1094200069462648FFF700FD3043C6B29EE73A463C
:1094300069462348FFF7F8FC3043C6B296E73A4640
:1094400069462048FFF7F0FC3043C6B28EE73A4643
:1094500069461D48FFF7E8FC3043C6B286E73A4646
:1094600069461A48FFF7E0FC3043C6B27EE73A4649
:1094700069461748FFF7D8FC3043C6B276E70022AA
:1094800052E700BF30A0FF1FF49FFF1F609FFF1F28
:10949000F09FFF1FE89FFF1F789FFF1FE09FFF1FA8
:1094A000F29FFF1FF0320100F89FFF1F689FFF1F10
:1094B00020330100483201005C310100AC3F010063
:1094C0009C3F01004C310100B4310100E83F010034
:1094D0001C91FF1F888AFF1F649FFF1F28B110285F
:1094E000044BA8BF102018607047024B0120186081
:1094F000704700BFFC9FFF1F08B5002006F02AF947
:109500000028FAD108BD00BF10B504464FF44060F2
:1095100005F034F805F08CF80A4B1B7833B96CB1C0
:10952000102C094BA8BF10241C6010BD4FF4C05074
:1095300004F0FAFD04F02EFF002CF1D1024B0124BF
:109540001C6010BD469EFF1FFC9FFF1F70B50D469F
:109550001446064605F062F8284605F05FF82046F6
:1095600005F05CF8084B1B7813B1084B1B7803B966
:1095700070BD304604F0B6FE284604F0B3FE204627
:10958000BDE8704004F0AEBE469EFF1F629EFF1F06
:1095900038B5164D2B78044641F6FF72A0F5005001
:1095A000824203F1FF33A8BF02461B0202F50052BC
:1095B00003F47063100443F4604343F00E0300F4BB
:1095C000FE005204184302F0FE42104305F0F8FF7B
:1095D0002868013860F01F00C4F3C61204F07F0150
:1095E000C0B2BDE83840FFF7B1BF00BFFC9FFF1F0E
:1095F00070B5104E3378013B1B0203F470630446D0
:1096000043F430430806220400F0FE4043F00B030D
:10961000034302F4FE0018430D4605F0D1FF306805
:10962000013860F04F002A462146C0B2BDE87040C4
:10963000FFF78CBFFC9FFF1F08B564210720FFF7D1
:10964000D7FF7F210B20BDE80840FFF7D1BF00BF47
:1096500070B5104E3378013B1B0203F4706304466F
:1096600043F410430806220400F0FE4043F00903CF
:10967000034302F4FE0018430D4605F0A1FF3068D5
:10968000013860F06F002A462146C0B2BDE8704044
:10969000FFF75CBFFC9FFF1F38B50E4D2B78013BD9
:1096A0001B0203F47063044643F41043000443F0C8
:1096B000090300F4FE00184305F082FF2868013812
:1096C00060F06F002146C0B20022BDE83840FFF7CD
:1096D0003DBF00BFFC9FFF1F10B500217B20FFF79F
:1096E00087FF0024E0B2FFF7D7FF0134022004F027
:1096F0005DFC802CF6D110BD38B50C46054604F053
:109700008DFF204604F08AFF074B1B7813B1074BEF
:109710001B7803B938BD284604F0E4FD2046BDE8B7
:10972000384004F0DFBD00BF469EFF1F629EFF1F52
:1097300038B50D4D2B78013B1B0203F470630446D2
:1097400043F45043000443F00D0300F4FE001843BB
:1097500005F036FF2868013860F02F002146C0B2BE
:10976000BDE83840FFF7C8BFFC9FFF1F38B50E4D5E
:109770002B78013B01381B02C4B203F47063200450
:1097800043F4404343F00C0300F4FE00184305F09B
:1097900017FF2868013860F03F002146C0B2BDE8DD
:1097A0003840FFF7A9BF00BFFC9FFF1F38B5044634
:1097B0000D46F02004F032FF35B1254414F8010BBA
:1097C00004F02CFFAC42F9D1F720BDE8384004F09A
:1097D00025BF00BF00B50B4B83B0024699881868BF
:1097E0000090032AADF8041002D903B05DF804FB21
:1097F000684606218DF80520FFF7D8FF03B05DF815
:1098000004FB00BF2840010000B50B4B024683B0AB
:10981000186899880090131F4C2BADF8041002D9DA
:1098200003B05DF804FB684606218DF80520FFF7BC
:10983000BDFF03B05DF804FB30400100030203F4F8
:10984000FE43C0F3C6101843704700BF037840784A
:10985000DB0103F47E5300F07F001843704700BF24
:1098600082B002AA114642F8040D002012F8013B12
:1098700003F07F03914243EA0020F7D102B0704722
:10988000003210B403884FF0010404FA01F418BF49
:10989000012202FA01F123EA04020A43028010BC09
:1098A000704700BF70B5CEB20C46054603F010FFFE
:1098B000864203D03146284603F024FF013528466E
:1098C00003F006FF240A844205D021462846BDE85D
:1098D000704003F017BF70BD38B5054603F0F8FEC1
:1098E0004FF0000460F30704681C03F0F1FE60F31E
:1098F0000F24A0B238BD00BFF8B504460020FFF722
:10990000EBFF002C00F083814FF4AF610220FFF7E2
:10991000C9FF04204FF47A61FFF7C4FF0B2004F065
:109920000FFB002840F079874FF496610620FFF77F
:10993000B9FF4FF4FA610820FFF7B4FF4FF4FA6162
:109940000A20FFF7AFFF40F6B8310C20FFF7AAFF5F
:109950004FF42F612220FFF7A5FF40F6AC512420E1
:10996000FFF7A0FF7D212A20FFF79CFF0C210E208E
:10997000FFF798FF01211020FFF794FF022112202A
:10998000FFF790FF00211420FFF78CFF0021162025
:10999000FFF788FF02211820FFF784FF01211A201A
:1099A000FFF780FF01211C20FFF77CFF04211E2010
:1099B000FFF778FF14212020FFF774FF01212620F4
:1099C000FFF770FF03212820FFF76CFF04212C20F4
:1099D000FFF768FF14212E20FFF764FF00213020DD
:1099E000FFF760FF0C213220FFF75CFF00213420DD
:1099F000FFF758FF00213620FFF754FF00213820E1
:109A0000FFF750FF00213A20FFF74CFF00213C20D8
:109A1000FFF748FF00213E20FFF744FF00214020D0
:109A2000FFF740FF00214220FFF73CFF1F214420A9
:109A3000FFF738FF13214620FFF734FF0E2148209F
:109A4000FFF730FF11214A20FFF72CFF0A214C209D
:109A5000FFF728FF00214E20FFF724FF06215020AA
:109A6000FFF720FF02215220FFF71CFF0C2154209A
:109A7000FFF718FF00215620FFF714FF00215820A0
:109A8000FFF710FF01215A20FFF70CFF08215C208F
:109A9000FFF708FF0A215E20FFF704FF0021602086
:109AA000FFF700FF04216220FFF7FCFE0121642084
:109AB000FFF7F8FE00216620FFF7F4FE0B21682077
:109AC000FFF7F0FE7F216A20FFF7ECFE00216C20FB
:109AD000FFF7E8FE00216E20FFF7E4FE0021702072
:109AE000FFF7E0FE00217220FFF7DCFE002174206A
:109AF000FFF7D8FE1F217620FFF7D4FE1321782030
:109B0000FFF7D0FE0E217A20FFF7CCFE11217C203A
:109B1000FFF7C8FE0A217E20FFF7C4FE1F21802028
:109B2000FFF7C0FE13218220FFF7BCFE0E21842028
:109B3000FFF7B8FE11218620FFF7B4FE0A21882026
:109B4000FFF7B0FE00218A20FFF7ACFE00218C2039
:109B5000FFF7A8FE00219620FFF7A4FE0021982021
:109B6000FFF7A0FE00219A20FFF79CFE05219C2014
:109B7000FFF798FE06219E20FFF794FE0021A0200B
:109B8000FFF790FE7F21A220FFF78CFE40F2A46138
:109B9000A420FFF787FE4FF4E161A620FFF782FEC5
:109BA0000021A820FFF77EFE0021AA20FFF77AFE01
:109BB0000221AC20FFF776FE0121AE20FFF772FEF6
:109BC0000121B020FFF76EFE0B21B220FFF76AFEE5
:109BD0006421B420FFF766FE6421B620FFF762FE21
:109BE0000321B820FFF75EFE2C210020FFF75AFE6C
:109BF0000220FFF771FEB0F5805F034616D34FF4E5
:109C0000AF610220FFF74EFE4FF4AF630EE04FF658
:109C1000FF7398423FF478AE2C2840F00A86022069
:109C2000FFF75AFEB0F5805F0346E8D2D24A04201F
:109C30001380FFF751FEB0F5805F034680F0568435
:109C4000CE4A06201380FFF747FEA0F52F739BB284
:109C5000B3F57A6F024606D940F628210620FFF7B1
:109C600021FE40F62822C64B08201A80FFF734FE5A
:109C7000A0F52F739BB2B3F57A6F024606D940F672
:109C8000E4410820FFF70EFE40F6E442BD4B0A20F7
:109C90001A80FFF721FEA0F5FA739BB240F6AC5193
:109CA0008B42024606D94FF4FA610A20FFF7FAFD0B
:109CB0004FF4FA62B44B0C201A80FFF70DFEA0F5AA
:109CC000FA739BB240F6AC518B42024606D940F67D
:109CD000B8310C20FFF7E6FD40F6B832AB4B0E2052
:109CE0001A80FFF7F9FD1828034600F2C584A84A38
:109CF00010201380FFF7F0FD431E9BB20F2B02468E
:109D000004D901211020FFF7CDFD0122A14B122023
:109D10001A80FFF7E1FD0A28034600F2A6849E4A56
:109D200014201380FFF7D8FD0128034604D9002131
:109D30001420FFF7B7FD0023984A16201380FFF781
:109D4000CBFD7F28034600F28984954A18201380B2
:109D5000FFF7C2FD0528034600F27984914A1A20D4
:109D60001380FFF7B9FD0C28034600F2BD848E4A2C
:109D70001C201380FFF7B0FD0428034600F2AD84D9
:109D80008A4A1E201380FFF7A7FD0928034600F228
:109D90009D84874A20201380FFF79EFD46280346B6
:109DA00000F28D84834A22201380FFF795FDA0F5F1
:109DB000FA739BB240F6AC518B42024606D94FF47F
:109DC0002F612220FFF76EFD4FF42F627A4B242083
:109DD0001A80FFF781FDA0F5FA739BB240F6AC54F0
:109DE000A342024604D921462420FFF75BFD224608
:109DF000724B26201A80FFF76FFD7F28034600F282
:109E000057846F4A28201380FFF766FD0628034613
:109E100000F247846B4A2A201380FFF75DFDA0F112
:109E200032039BB2B3F5967F024604D97D212A20E6
:109E3000FFF738FD7D22644B2C201A80FFF74CFD84
:109E40000C28034600F22684604A2E201380FFF778
:109E500043FD1E28034600F216845D4A302013801D
:109E6000FFF73AFD0928034600F2D084594A322010
:109E70001380FFF731FD1F28034600F2C084564AC5
:109E800034201380FFF728FD7F28034600F2B084BA
:109E9000524C36202380FFF71FFD7F28034600F237
:109EA000A08438206380FFF717FD7F28034600F267
:109EB00091843A20A380FFF70FFD7F28034600F22C
:109EC00082843C20E380FFF707FD7F28034600F2F1
:109ED00073843E202381FFF7FFFC7F28034600F2B6
:109EE000648440206381FFF7F7FC7F28034600F27B
:109EF00055844220A381FFF7EFFC394D2880442090
:109F0000FFF7EAFC3028034600F24184354A462038
:109F10001380FFF7E1FC3028034600F23184324C15
:109F200048202380FFF7D8FC3028034600F2218424
:109F30004A206380FFF7D0FC3028034600F21284E9
:109F40004C20A380FFF7C8FC3028034600F2DF83D3
:109F50004E20E380FFF7C0FC0128034604D900210E
:109F60004E20FFF79FFC0023204A50201380FFF76C
:109F7000B3FC431E3CE000BF489DFF1F129FFF1F24
:109F8000029DFF1FE09EFF1FAC9EFF1FC89CFF1F8E
:109F9000969CFF1F649EFF1F969EFF1F3E9DFF1F06
:109FA0009C9CFF1F4E9DFF1FE89CFF1FE09CFF1F16
:109FB000D09CFF1FF29EFF1F609EFF1F5C9EFF1F35
:109FC000E49EFF1FBA9EFF1F0A9FFF1FB69CFF1F44
:109FD000349DFF1F209FFF1FE29EFF1F209EFF1F3B
:109FE000149FFF1FC09CFF1FBC9EFF1FDE9CFF1F16
:109FF0009BB20B2B024604D906215020FFF752FCDE
:10A000000622CF4B52201A80FFF766FC0428034635
:10A0100000F27783CB4A54201380FFF75DFC431E88
:10A020009BB21D2B024604D90C215420FFF73AFCA9
:10A030000C22C54B56201A80FFF74EFC0128034620
:10A0400004D900215620FFF72DFC0023BF4A5820D9
:10A050001380FFF741FC7F28034600F24C83BC4A83
:10A060005A201380FFF738FC431E9BB2092B02468F
:10A0700004D901215A20FFF715FC0122B54B5C20C1
:10A080001A80FFF729FC431E9BB2102B024604D90D
:10A0900008215C20FFF706FC0822AF4B5E201A80E7
:10A0A000FFF71AFC431E9BB21D2B024604D90A215E
:10A0B0005E20FFF7F7FB0A22A84B60201A80FFF70B
:10A0C0000BFC0228034600F2A482A54A64201380F8
:10A0D000FFF702FC0128034604D901216420FFF7A1
:10A0E000E1FB01239F4A62201380FFF7F5FBC31EAB
:10A0F0009BB2012B024604D904216220FFF7D2FB58
:10A100000422994B66201A80FFF7E6FB7F2803465E
:10A1100000F27982954A68201380FFF7DDFB7F28E3
:10A12000034600F26A82924A6A201380FFF7D4FB4A
:10A130007F28034600F25B828E4A6C201380FFF773
:10A14000CBFB0328034600F24C828B4A6E2013801F
:10A15000FFF7C2FB1928034600F23D82874A7020B0
:10A160001380FFF7B9FB0228034600F22E82844ACF
:10A1700072201380FFF7B0FB0628034600F21F820F
:10A18000804A74201380FFF7A7FB0728034600F2DC
:10A1900010827D4A8A201380FFF79EFB0A2803461F
:10A1A00000F20182794A8C201380FFF795FB042886
:10A1B000034600F2F281764A98201380FFF78CFB69
:10A1C0000128034604D900219820FFF76BFB0023E8
:10A1D000704A9A201380FFF77FFB0128034604D9B9
:10A1E00000219A20FFF75EFB00236B4A9620138024
:10A1F000FFF772FB0B28034600F2C981674A9C20D7
:10A200001380FFF769FB831E9BB2032B024604D920
:10A2100005219C20FFF746FB0522614B76201A8022
:10A22000FFF75AFB3028034600F2AB815D4A7820E5
:10A230001380FFF751FB3028034600F29C815A4CF3
:10A240007A202380FFF748FB3028034600F28D81F7
:10A250007C206380FFF740FB3028034600F27F81BB
:10A260007E20A380FFF738FB3028034600F271817F
:10A270008020E380FFF730FB3028034600F2638143
:10A280004A4A82201380FFF727FB3028034600F25A
:10A290005481474C84202380FFF71EFB302803465F
:10A2A00000F2458186206380FFF716FB30280346C5
:10A2B00000F237818820A380FFF70EFB3028034689
:10A2C00000F22981A020E380FFF706FB0128034666
:10A2D00004D90021A020FFF7E5FA0023354A9E208B
:10A2E0001380FFF7F9FAC31E9BB20C2B024604D968
:10A2F00006219E20FFF7D6FA06222F4BA2201A80B5
:10A30000FFF7EAFA431E9BB27E2B024604D97F2157
:10A31000A220FFF7C7FA7F22284BA4201A80FFF75C
:10A32000DBFAA0F5AF639BB2B3F5167F024647D9BF
:10A3300040F2A461A420FFF7B5FA40F2A4623FE026
:10A340002089FF1F3489FF1FB089FF1F229DFF1F37
:10A35000A69EFF1F909CFF1FB489FF1F2C89FF1F23
:10A36000589EFF1FB49EFF1FF09CFF1FF49EFF1F0F
:10A37000209DFF1FD49CFF1F849CFF1F489FFF1F31
:10A38000409EFF1F1C9FFF1FD89EFF1F669EFF1F42
:10A39000509EFF1FD29CFF1F2C9DFF1FA09EFF1FE2
:10A3A000B89CFF1FCA9CFF1F309EFF1FCC9CFF1F45
:10A3B000389EFF1FC49EFF1F9C89FF1FE69EFF1F44
:10A3C000D64BA6201A80FFF787FAA0F5AF639BB2A1
:10A3D000B3F5167F024606D94FF4E161A620FFF7D8
:10A3E00061FA4FF4E162CE4BA8201A80FFF774FAAD
:10A3F0000628034600F28980CA4AAA201380FFF784
:10A400006BFA032803467AD8C74AAC201380FFF7BB
:10A4100063FA0328034600F21481C44AB020138073
:10A42000FFF75AFA0328034600F20581C04AAE201E
:10A430001380FFF751FA7F28034600F2F680BD4AE9
:10A44000B2201380FFF748FA7F28034600F2E78026
:10A45000B94AB4201380FFF73FFA431E9BB2C62BC4
:10A46000024604D96421B420FFF71CFA6422B34BDE
:10A47000B6201A80FFF730FA431E9BB2C62B024665
:10A4800004D96421B620FFF70DFA6422AC4BB82042
:10A490001A80FFF721FA082822D82B88DFF8C0E2BB
:10A4A000A84FA94AA94DAA4EAA4CAB4903F0010CEA
:10A4B000AEF800C0C3F3400EA7F800E0C3F3800776
:10A4C0001780C3F3C007A54A2F70C3F30017C3F367
:10A4D0004015C3F38013378025800B801080F8BDB2
:10A4E000B8200321FFF7DEF90320D6E74FF47A61A5
:10A4F0000420FFF7D7F94FF47A63FFF7A1BB0021DF
:10A50000AA20FFF7CFF900237EE70021A820FFF75C
:10A51000C9F9002370E70A218820FFF7C3F90A234D
:10A52000D0E611218620FFF7BDF91123C2E60E21E6
:10A530008420FFF7B7F90E23B4E613218220FFF73A
:10A54000B1F91323A5E61F218020FFF7ABF91F23E4
:10A5500096E60A217E20FFF7A5F90A2388E6112155
:10A560007C20FFF79FF911237AE60E217A20FFF76E
:10A5700099F90E236CE613217820FFF793F9132342
:10A580005DE61F217620FFF78DF91F234EE600219F
:10A590009620FFF787F9002330E600218C20FFF793
:10A5A00081F9002307E600218A20FFF77BF90023C9
:10A5B000F8E500217420FFF775F90023E9E5002193
:10A5C0007220FFF76FF90023DAE500217020FFF712
:10A5D00069F90023CBE500216E20FFF763F9002322
:10A5E000BCE500216C20FFF75DF90023ADE57F217C
:10A5F0006A20FFF757F97F239EE50B216820FFF7BC
:10A6000051F90B238FE500216620FFF74BF900235A
:10A6100080E500216020FFF745F9002355E50B2177
:10A62000B220FFF73FF90B2312E70121AE20FFF71D
:10A6300039F9012303E70121B020FFF733F90123A2
:10A64000F4E60221AC20FFF72DF90223E5E6022112
:10A650001820FFF727F90223FFF780BB00211620FF
:10A66000FFF720F90023FFF770BB02211220FFF74C
:10A6700019F90223FFF753BB0C210E20FFF712F943
:10A680000C23FFF734BB14212E20FFF70BF9142302
:10A69000FFF7E3BB04212C20FFF704F90423FFF7A5
:10A6A000D3BB03212820FFF7FDF80323FFF7B2BB3C
:10A6B00001212620FFF7F6F80123FFF7A2BB1421A2
:10A6C0002020FFF7EFF81423FFF76CBB04211E20B6
:10A6D000FFF7E8F80423FFF75CBB01211C20FFF71C
:10A6E000E1F80123FFF74CBB01211A20FFF7DAF84C
:10A6F0000123FFF73CBB00215820FFF7D3F80023CC
:10A70000ADE402215220FFF7CDF8022382E40A21B2
:10A710004C20FFF7C7F80A231AE400BF4C9DFF1F27
:10A72000CC9EFF1F929CFF1F069DFF1FB69EFF1F22
:10A73000449EFF1FDC9CFF1FFA9CFF1F089FFF1F0A
:10A74000349FFF1F009DFF1F369DFF1F629EFF1F4E
:10A750005A9EFF1FB89EFF1F6A9EFF1F989CFF1FF7
:10A76000A29EFF1F11214A20FFF79CF81123FFF73B
:10A77000E7BB0E214820FFF795F80E23FFF7D8BB63
:10A7800013214620FFF78EF81323FFF7C8BB1F21C4
:10A790004420FFF787F81F23FFF7B8BB00214020B4
:10A7A000FFF780F80023FFF7A4BB00213E20FFF74E
:10A7B00079F80023FFF795BB00213C20FFF772F8E2
:10A7C0000023FFF786BB00213A20FFF76BF8002338
:10A7D000FFF777BB00213820FFF764F80023FFF76D
:10A7E00068BB00213620FFF75DF80023FFF759BB57
:10A7F00000213420FFF756F80023FFF749BB0C2156
:10A800003220FFF74FF80C23FFF739BB002130202F
:10A81000FFF748F80023FFF729BB40F62821062060
:10A82000FFF740F840F6E4410820FFF73BF8FFF758
:10A8300085B817287FF668A819287FF6D7A81B289F
:10A840007FF6F4A81C283FF409A91E287FF60EA95C
:10A850001F283FF413A920283FF42CA921283FF4F6
:10A8600035A922283FF43AA923283FF443A92428F4
:10A870003FF474A925283FF479A926283FF47AA942
:10A8800027283FF47FA928283FF48AA929283FF4E4
:10A890008FA92A283FF49CA92B287FF4A5A9FFF7AC
:10A8A0009FB900BFF8B5CB2006F00AFD204B214A26
:10A8B000054603CB1368C5F803001A0CBA20C5F887
:10A8C00007102B80AA70FEF7B9FF2E46002426F849
:10A8D0000B0FA0B2FFF700F8FEF7B0FF0234BA2C5E
:10A8E00026F8020FF5D16C1E05F1C6064FF0FF30B9
:10A8F00014F8013F082758400F4B40F300017A1E1F
:10A900000B4012F0FF0783EA5000F5D1B442EFD1BB
:10A91000C043FEF7A5FF3A46C5F8C700CB2128463D
:10A9200004F09CFE2846BDE8F84006F0D1BC00BF0C
:10A930003C400100384001002083B8EDF0B50E4BDB
:10A940000E4C054693E8070085B024682E88AD7844
:10A9500001AB83E80700270C184600220B21ADF855
:10A9600004408DF80670ADF80C608DF80E5004F0C0
:10A9700075FE05B0F0BD00BF484001003840010041
:10A98000F0B5124B124D1E68124F0FCD87B06C46BA
:10A990000FC495E8030044F8040B38683B79CDF800
:10A9A0000D00320C2C2021808DF802208DF8113002
:10A9B000ADF80060FEF742FF0022ADF80B00122157
:10A9C000684604F04BFE07B0F0BD00BF3840010000
:10A9D00054400100BC340100002004F0BBBE00BFA5
:10A9E00002F02EBE70B5124C82B000254023064600
:10A9F00029462046009301958023202201F072FE13
:10AA000020222946204602F031FA2046012102F098
:10AA100037FA304607F0F4F931460246204602F094
:10AA2000BFFB204602B0BDE8704001F041BC00BF52
:10AA3000789FFF1FF0B5CA2983B075D90546441E1B
:10AA400000F1C6064FF0FF3014F8012F08275040E0
:10AA5000404A40F300017B1E0A4013F0FF0782EAE0
:10AA60005000F5D1B442EFD1C043FEF7F9FE0146E4
:10AA7000D5F8C7000190019A914202D0B2F17F2F20
:10AA80000BD105F10B00FEF7E1FEBA280BD03248DE
:10AA9000FFF7A8FF002003B0F0BD3048FFF7A2FF8A
:10AAA000384603B0F0BD05F10D00FEF7CFFE2C28AF
:10AAB00040D1002440F6AC5613E004281AD00628F2
:10AAC00021D008281FD00A2828D00C2822D1A1F58F
:10AAD000FA7292B2B24201D8FEF7E4FE0234BA2C06
:10AAE0000ED004F10D002844FEF7B0FE022C014602
:10AAF000A0B2E2D1B1F5805FEED30234BA2CF0D12E
:10AB0000012003B0F0BDA1F52F7292B2B2F57A6FB9
:10AB1000E4D8E1E7222801D0242811D1A1F5FA7266
:10AB200092B2B242DAD8D7E70D48FFF75BFF0020B8
:10AB300003B0F0BD0B48FFF755FF002003B0F0BD98
:10AB40002A28C9D1A1F1320292B2B2F5967FC5D8B6
:10AB5000C2E700BF2083B8ED9840010084400100A7
:10AB60006C400100AC40010003290CD970B5461CB3
:10AB700082B005460C46304603222A4907F0AEF95A
:10AB800010B102B070BD70470B2C05D905222649C3
:10AB9000281D07F0A3F940B12448FFF723FF2448FC
:10ABA00002B0BDE87040FFF7C9BE05F109010322FC
:10ABB00001A807F0E3F901A803221E4907F08EF966
:10ABC000D8B103221C4901A807F088F908B301A8ED
:10ABD00003221A4907F082F9B0B91948FFF702FFBA
:10ABE000A11E89B23046FFF725FF0028C9D01548BD
:10ABF00002B0BDE87040FFF7F5BE1348FFF7F2FE64
:10AC0000FFF750FE1148F3E71148FFF7EBFE11483C
:10AC1000C6E71148FFF7E6FE02B0BDE87040FFF757
:10AC2000AFBE00BF38400100D4340100C440010071
:10AC3000D8400100DC400100044101001C4101003A
:10AC40002041010034410100E0400100F4400100D6
:10AC5000484101005C410100084101002DE9F04339
:10AC6000174D2B6883B081460F469046F3B1154EC1
:10AC700034880A1992B218461146328006F09EFEB8
:10AC800028603A464946204402F06CFDB8F1000FB6
:10AC900009D031882868FFF767FF286806F018FB9D
:10ACA00000232B60338003B0BDE8F083054E019391
:10ACB0000846318006F004FB019B28601C46E0E753
:10ACC00004A0FF1F00A0FF1F10B51F4C4FF4FA7027
:10ACD000FBF73AFD204601F0DFF90022114620463D
:10ACE00002F0C4F82046012102F0CAF820460021F3
:10ACF00002F0C0F80B221549204602F051FA204616
:10AD000002F064FA0F221249204602F049FA204666
:10AD100002F05CFA0F490722204602F041FA204671
:10AD200002F054FA204601F0C3FA0B4B0B4A1A60AA
:10AD30004FF4FA70FBF708FDFFF722FE0848BDE864
:10AD40001040FFF74FBE00BF789FFF1F604101001A
:10AD50006C4101007C41010038A2FF1F5DAC000086
:10AD6000844101000020704790F8392090F83800A5
:10AD7000101A704790F8383090F839209A4205D967
:10AD80005A1C034480F83820187E70474FF0FF307B
:10AD9000704700BF90F8383090F839209A4286BF4B
:10ADA0001B18187E4FF0FF30704700BF704700BF80
:10ADB00038B50546B0F85E0090B195F85D301446A0
:10ADC000C3F1210294420CD805F13B0018442246FD
:10ADD00002F0C8FC95F85D30234485F85D302046CC
:10ADE00038BD012014462871EEE700BFB0F85E3090
:10ADF0006BB190F85D30202B07D8C218013380F872
:10AE00005D30012082F83B10704701230371002060
:10AE1000704700BF0023426980F8383080F839302D
:10AE200080F85C3080F85D3080F85E3080F85F300C
:10AE300006CA30B40D68046943662A4383660A6013
:10AE4000A370426990F861301649146813441D7A62
:10AE50005B7B01EBC5051B026D6803F4E06343F007
:10AE600064032B6090F8623013449D7CDB7D01EB22
:10AE7000C5011B02496803F4E06343F064030B60FF
:10AE800021685368194205D0036927225A70036963
:10AE900004229A71036920225A71036980229A70F0
:10AEA00030BC7047B84C010043690CCB12681A42A1
:10AEB0000CD0094B99420AD9084B9942036994BFB7
:10AEC0001A220D225A70036904229A71704703698D
:10AED00027225A70F7E700BF7F1A06003F420F0093
:10AEE00010B50269D378DBB2D90604463DD51021EE
:10AEF0005806D17038D503F0040303F0FF02002B8D
:10AF000051D03D49626E00230B7084F85D30002AF9
:10AF10005BD0904794F85D30002B56D02369D02247
:10AF20009A70236994F83B201A712369012284F8EE
:10AF30005C200222DA7010BD304B84F860009C4225
:10AF40004AD02F4B9C4252D094F8391013791F29C4
:10AF5000DBB207D82848007820B16018013184F8A6
:10AF6000391003760223D37010BD5906C3D49178EB
:10AF700001F0100101F0FF000029DDD013F0010302
:10AF80001ED194F85C1094F85D00884281BF4B1C80
:10AF9000091984F85C3091F83B3013712369D02291
:10AFA0009A702269DEE7236984F83920C0229A70FA
:10AFB0002369114A1979012111700222DA7010BD3A
:10AFC000C023937022691379CCE70122002384F80F
:10AFD0005D2084F83B30A1E7626994F8613009494B
:10AFE00013440322187A02F043FD2269ACE7626938
:10AFF00094F861300449F3E708A0FF1F6491FF1F34
:10B00000D091FF1F69B0000075B000000369DB78C4
:10B0100003F0200373B190F860300133DBB2012BF1
:10B0200080F860301AD9426990F861301344187A78
:10B0300002F09ABD70B5426903F0FF0590F86130E7
:10B0400013440446187A02F08FFDA36E5BB184F8B6
:10B05000385094F83900BDE87040184790F85F30D8
:10B06000002BE0D0704770BD0148FFF7CFBF00BF95
:10B070006491FF1F0148FFF7C9BF00BFD091FF1FB8
:10B080002DE9F047374FDFF8E0903B68026982B066
:10B0900006460093DDF800800021A025D3789B06AA
:10B0A0005BD53B680193019BC8EB03030F2BF5D9DC
:10B0B00049B1102BF2D000209070336980229A7031
:10B0C00002B0BDE8F087726996F86130134405213B
:10B0D000187A02F043FF726996F861301344012137
:10B0E00093F812A0504602F039FF0924002150467F
:10B0F00002F020FF2B46013BFDD10121504602F01A
:10B1000019FF2B46013BFDD1013CEFD1706996F848
:10B11000611001444FF4A0720C7A4B7B09EBC4011F
:10B120001B02496803F4E06343F064030B6096F884
:10B1300062300344997CDB7D09EBC1011B02496845
:10B1400003F4E06343F064030B60013AFDD132691C
:10B15000D3789B064FF00101A3D4012002B0BDE8D3
:10B16000F08700BF30A0FF1FB84C0100F0B50369A5
:10B170001222DA700269937803F0200385B0044646
:10B180000D46002B5ED0B42393703C4922690B68B6
:10B190000093009E05E00B680193019B9B1B042B11
:10B1A00042D8D37803F0200303F0FF00002BF2D045
:10B1B00094F85D30002B31D04FF0000E4FF0020CB0
:10B1C00004EB0E0393F83B3013710B680393039F5A
:10B1D000206907E09B060DD50B680293029BDB1BE1
:10B1E000052B28D8C378DBB203F0020202F0FF0679
:10B1F000002AEFD080F803C02669F378DBB2DF06BF
:10B2000032462DD49F062BD5DB0731D40EF1010E2B
:10B2100094F85D305FFA8EFE7345D1D800201DBBD7
:10B22000002384F85E3004E09070236980229A70D5
:10B23000042005B0F0BD86702369802204209A7036
:10B2400005B0F0BD03F0FF06FFF71AFF10B90420A8
:10B2500005B0F0BD236984F85F60B0229A7094E76E
:10B260008023B3700420DAE726698023B370D7E720
:10B27000BEF1000F0CBF02200320F6E730A0FF1F35
:10B280002DE9F04106690025122780F8385080F832
:10B290003950F770D0F810C09CF802E00EF0200E84
:10B2A00088B00446884615461E46BEF1000F49D0B8
:10B2B000B4238CF80230784B21691A680092DDF8CB
:10B2C00000E006E01A6801920198CEEB0000042825
:10B2D00030D8C87800F0200000F0FF070028F1D037
:10B2E0004FEA480242F00102D2B20A711A68029291
:10B2F000DDF808E0206906E01A6803920399CEEBB6
:10B30000010105292AD8C17801F0020101F0FF07E7
:10B310000029F1D04FF0020C80F803C02269D178E7
:10B3200011F0110722D12DBB002E0CBFA0238023CA
:10B33000937003E08F70236980229A70384608B0BA
:10B34000BDE8F0810EF0FF07FFF79AFE0028F5D068
:10B35000236984F85F70B0229A70ACE78770236924
:10B36000802238469A7008B0BDE8F081802393703F
:10B370000027E3E7012D75D0A021917021690A799A
:10B38000BE4667464FF0A80C1A680492049805E080
:10B390001A680592059A121A052A4AD8CA7802F044
:10B3A000020202F0FF08002AF2D0CF702169CA78A9
:10B3B000D2B212F0100F08465AD1920658D5013D6C
:10B3C000EDB2012D49D0BEF11F0F3BD90A79012DF5
:10B3D000DAD11A680692069D05E01A680792079A64
:10B3E000521B052A46D8C27802F0020202F0FF0181
:10B3F000002AF2D00223C3702269D378DBB2D906C7
:10B400003AD49B0634D5B023BEF11F0F93703FD8BA
:10B41000226904EB0E0312791A760EF1010E5FFA1F
:10B420008EFE16B1236980229A7084F839E077463F
:10B4300084E781F80280236980229A70774684F835
:10B4400039E07BE704EB0E0291F8048082F8188063
:10B450000EF1010E5FFA8EFEB9E781F802C0216994
:10B460000846B0E7A82191702069BE460279B0E78E
:10B47000774663E78170DEE71021A023D170013B9E
:10B48000FDD12269937803F0F7037746937055E76F
:10B4900023691B79C5E700BF30A0FF1F0148FFF7F4
:10B4A0001FBD00BF6491FF1F0148FFF719BD00BF1A
:10B4B000D091FF1F704700BF38B5144C03780122AC
:10B4C0005B000546204684F83B3084F85E2084F813
:10B4D0005D20FFF78BFC20460021FFF747FE0B4C59
:10B4E0002978012320461A46FFF7CAFE0128F6D123
:10B4F00094F8383094F839209A4205D9E21801338B
:10B5000084F83830107E38BDFF2038BD6491FF1FAD
:10B5100038B51B4C037801225B000546204684F8B1
:10B520003B3084F85E2084F85D20FFF75FFC204606
:10B530000021FFF71BFE124C29782046012302222E
:10B54000FFF79EFE0228F6D194F8382094F83910BF
:10B550008A420FD2531CDBB2A018994284F83830CB
:10B56000007E0AD9234402321B7E84F8382040EA48
:10B57000032038BD4FF6FF7038BD40F47F4038BD22
:10B580006491FF1F0C2901D9002070470231490046
:10B5900001F0FE01FFF7BCBF70B50C4C03781646F6
:10B5A00001255B00204684F83B3084F85E5084F827
:10B5B0005D50FFF71BFC31462046FFF717FC29467C
:10B5C0002046BDE87040FFF7D1BD00BF6491FF1F6A
:10B5D000F8B505460F461646412421463A46284608
:10B5E000FFF7DAFF611C0234C9B232462846E4B2E2
:10B5F000FFF7D2FF592CF0D1F8BD00BF38B5044693
:10B600000D463548FFF706FC632280212046257051
:10B61000FFF7C2FF012002F0C9FC204600225E2194
:10B62000FFF7BAFF20465D21FFF746FF242801D02F
:10B63000002038BD204606220C21FFF7C9FF204616
:10B6400001222B21FFF7A8FF204601222C21FFF722
:10B65000A3FF20460E222D21FFF79EFF2046002249
:10B660002E21FFF799FF204601222F21FFF794FF9B
:10B67000204605223021FFF78FFF2046012231218D
:10B68000FFF78AFF204600223221FFF785FF204680
:10B6900000223321FFF780FF204600223421FFF7EC
:10B6A0007BFF204600223521FFF776FF204600224F
:10B6B0005B21FFF771FF204610225C21FFF76CFF32
:10B6C000204620225D21FFF767FF20468F225E2162
:10B6D000FFF762FF012038BD6491FF1F10B4047FA3
:10B6E0004160022CC26002D010BC01F0D7BB83685D
:10B6F00010BC184790E80C00F0B41C685968256825
:10B70000164F174E29432160164D17491760D66012
:10B7100015611160417A154A5C180A3194F8244089
:10B7200053F8215002EBC40149680D60017A5C189E
:10B7300003EB8101247ECD6902EBC40149680D60F1
:10B74000817A581803EB810390F83000596B02EBB3
:10B75000C002F0BC53681960704700BF01401F0071
:10B76000011000380110007800001F80B84C010063
:10B77000704700BFF0B50C1EBDF8146034DBB0F9A3
:10B7800006701919B942C4BF3B1B1BB2002BA64659
:10B790001CDD002A1146B8BFD11D02F00705CC10F0
:10B7A000826A012007FB04E1A840012E0A44C0B2CE
:10B7B0001ED00CD3022E09D1013B12FA83F3013AB9
:10B7C00012F8011F41409A421170F9D1F0BDC043F7
:10B7D000013B12FA83F3C0B2013A12F8011F014093
:10B7E00093421170F9D1F0BD23441BB20024C6E787
:10B7F000013B12FA83F3013A12F8011F01439A4206
:10B800001170F9D1F0BD00BFF8B50D1E0EDB144666
:10B810001F46064601F03AFBA84207DD002C05DB77
:10B82000304601F037FBA04201DCF8BDF8BD3046E0
:10B8300001F02AFB022853D003284BD0012806D15F
:10B840006540F3886C406540013B5D1B2DB2012FC4
:10B8500003D02AD3022F14D0F8BD002C2246B6F90B
:10B860000630B06AB8BFE21D42F3CF0202FB0355B7
:10B8700004F00704435D012101FA04F41C4344551C
:10B88000F8BD002C2246B6F90630B06AB8BFE21DFA
:10B8900042F3CF0202FB035504F00704435D01218C
:10B8A00001FA04F45C404455F8BD002C2246B6F978
:10B8B0000630B06AB8BFE21D42F3CF0202FB035567
:10B8C00004F00704435D012101FA04F423EA0404AF
:10B8D0004455F8BD3389013B591B25460CB2B6E7E8
:10B8E000F18832890139013A4D1B141B2DB224B263
:10B8F000ADE700BF2DE9F041079E9DF91880089D36
:10B9000004461F4600F0C0FF0D4B0E480E4984F858
:10B910003380FF22002F08BF1F4684F82F2000230A
:10B9200084F8302084F8312084F832202060A66525
:10B93000E565676261652362A3622046BDE8F08128
:10B940006491FF1F104201000110013810B5044638
:10B95000806A034B236008B105F0BAFC204610BD95
:10B9600010420100F8B5436ADBB190F82C200125A4
:10B97000AA4083F83B2083F85E5083F85D5004466C
:10B98000406A03680E461B6800219847606A036896
:10B9900031461B6898472946606ABDE8F840FFF7C2
:10B9A000E5BBC26BC56C1368046A23EA0503136028
:10B9B0004CB122684FF00043D3625163D36A002B2D
:10B9C000FCDA936BF8BD836B466B0825802410E08E
:10B9D0003768426C3A4332601F68826C3A431A609F
:10B9E0001A68876C013D22EA07024FEA54041A6084
:10B9F00007D02142ECD13268476C22EA070232605C
:10BA0000EAE7F8BD70B50446406A0D4600282BD021
:10BA1000A16DFFF749FA002D20460CBFA621A721F2
:10BA2000FFF7A0FF606A20B1E16DBDE87040FFF74D
:10BA30003BBA216C226D0868236A02430A6093B105
:10BA4000DA7A82B1D00703D5224A99691160DA7A8D
:10BA5000910703D5204AD9691160DA7A520702D5D5
:10BA60001E4A1B6A136070BD236A002B2BD0D97A43
:10BA7000626DE1B172B6D97ACE0706D51848D96899
:10BA80000668314099610160D97A880706D5154862
:10BA9000196906683140D9610160D97A4E0705D528
:10BAA00011485969066831401962016062B61B6825
:10BAB000D968914207D00D4818600D49DA6042F00C
:10BAC000804018611960226C216D136823EA01031C
:10BAD0001360A0E700E100E004E100E008E100E01D
:10BAE00080E100E084E100E088E100E001403F0007
:10BAF00000003F80436A2DE9F04105460E4690461E
:10BB0000002B3ED090F82C100124A14083F83B106C
:10BB100083F85E4083F85D40406A036800211B683B
:10BB200008F1FF379847FFB2B8F1000F23D0374430
:10BB3000A046013E686A16F8011F03681B68984713
:10BB40000134B742E4B216D0202CF3D10121686A47
:10BB5000FFF70CFB95F82C206B6A520083F83B2012
:10BB600083F85E8083F85D80686A036800211B6843
:10BB700098470124DEE7686A0121BDE8F041FFF73C
:10BB8000F5BAC26BC16C136823EA010306EB080423
:10BB900013604FF00048A6420ED02B6A16F801EB56
:10BBA00063B11A68C2F82C80C2F834E0D36A002B63
:10BBB000FCDAA642936BF0D1BDE8F081AB6BD5F80F
:10BBC00034C008208021DCF800206F6C1EEA010FD1
:10BBD00014BF3A43BA43CCF800201A68AF6C3A431A
:10BBE0001A601A68AF6C013822EA07024FEA510165
:10BBF0001A60E8D1CFE700BF70B50446406A0D4631
:10BC0000002828D0A16DFFF74FF920462946FFF7FD
:10BC1000A9FE606A20B1E16DBDE87040FFF744B94C
:10BC2000216C226D0868236A02430A6093B1DA7AB4
:10BC300082B1D00703D5234A99691160DA7A910756
:10BC400003D5214AD9691160DA7A520702D51F4A11
:10BC50001B6A136070BD236A002B2BD0D97A626DEA
:10BC6000E1B172B6D97ACE0706D51948D968066807
:10BC7000314099610160D97A880706D5154819695C
:10BC800006683140D9610160D97A4E0705D512485E
:10BC90005969066831401962016062B61B68D9684B
:10BCA000914207D00D4818600D49DA6042F080409B
:10BCB00018611960226C216D136823EA0103136077
:10BCC000A3E700BF00E100E004E100E008E100E0DC
:10BCD00080E100E084E100E088E100E001403F0015
:10BCE00000003F802DE9F041044686B0806A9DF84F
:10BCF00030801E460F461546B4F90830002800F083
:10BD00004281DA1D48BF03F10E02B4F90630D210A9
:10BD100003FB02F2002105F0FFFDB4F90820202A00
:10BD200000F39280B4F90610A34B0120203A733936
:10BD300002EBD27201EBD1714FF0200E0290732012
:10BD40008DE8014042F34F0241F34F01204600F0DD
:10BD500051FE606A84F82D70002800F04D81002D9E
:10BD600040F08A80B4F90830202B14BF3D253C25D3
:10BD700084F82C50B8F1000F40F0858006B394F998
:10BD80003300002818DBC0B2012102F0E7F80121DE
:10BD900094F8330002F0CEF8012002F007F90021F8
:10BDA00094F8330002F0C6F80A2002F0FFF80121EF
:10BDB00094F8330002F0BEF8606A002800F0828038
:10BDC000A16DFFF771F804227C492046FFF792FE2F
:10BDD000217A0139C9B22046FFF7C4FD784904220F
:10BDE0002046FFF787FE94F92D30012B14BF142154
:10BDF00010212046FFF7B6FD042272492046FFF7C6
:10BE000079FEB4F90630802B00F09280602B00F0B0
:10BE1000A680D9212046FFF7A5FD94F92D30012BEE
:10BE200014BFF12122212046FFF79CFD2046062267
:10BE30006549FFF75FFE606A50B3E16DFFF734F8C4
:10BE4000012006B0BDE8F081B4F906105F4B012077
:10BE5000403A52394FF0400E029002EBD27252201B
:10BE600001EBD1718DE8014042F34F0241F34F01E4
:10BE7000204600F0BFFD6CE76DB284F82C50B8F19D
:10BE8000000F3FF47BAFFEF7C5FF002E94D076E79E
:10BE9000216C226D0868236A02430A6073B1DA7A62
:10BEA00062B1D00703D54A4A99691160DA7A9107DD
:10BEB0007CD4520702D5474A1B6A1360012006B0A2
:10BEC000BDE8F081236A002B2BD0D97A626DE1B1F5
:10BED00072B6D97ACF0706D53F48D9680568294098
:10BEE00099610160D97A8E0706D53C4819690568C1
:10BEF0002940D9610160D97A4D0705D5384859697B
:10BF0000056829401962016062B61B68D9689142D0
:10BF100007D0344818603449DA6042F08040186134
:10BF20001960226C216D136823EA010313604AE74C
:10BF3000B4F90830202B00F08680402B7FF469AFE5
:10BF40002A4920460322FFF7D5FD94F92D30012B15
:10BF500014BFCF219F212046FFF704FD59E7B4F914
:10BF60000830102B7FF455AF214920460322FFF7FC
:10BF7000C1FD94F92D30012B14BFAF2110212046B3
:10BF8000FFF7F0FC45E7DA1D48BF03F10E02B4F9F4
:10BF90000630D21003FB02F21046059205F090F92C
:10BFA000A06200283FF44DAF059AB3E6114AD96963
:10BFB0001160DA7A7DE700BF684201004844010061
:10BFC0004C44010050440100544401005C44010011
:10BFD00000E100E008E100E080E100E084E100E051
:10BFE00088E100E001403F0000003F806442010022
:10BFF0001C47010004E100E0012194F83100244FC6
:10C0000001F0ACFF94F83200012101F0A7FF94F990
:10C01000312094F9323057F83220E26357F8333048
:10C02000206A23640125E56425651A682A431A609D
:10C0300078B1B8F1000F3FF428AFFFF75BFB002E9B
:10C040003FF4BAAE9BE6042212492046FFF752FDA8
:10C05000DFE6294694F82F0001F080FF294694F886
:10C06000300001F07BFF94F92F2094F9303057F81D
:10C070003220626357F833306564A5641A68A3639D
:10C0800022F001021A60002E3FF496AE77E600BF60
:10C09000B84C010060420100B0F90820D31D48BF30
:10C0A00002F10E03B0F90620806ADB1002FB03F2F6
:10C0B000002105F031BC00BFF0B50029BDF81450D7
:10C0C0002EDBB0F90660B1422ADA002A59DBB0F95A
:10C0D000087014461C44BC42C4BFBB1A1BB2002BE0
:10C0E0001EDDD2B2D408D0F828E016FB041112F0FD
:10C0F0000702DBB20EEB010421D0C2F10807FAB24D
:10C10000374F9342BF5C0CD2C3EB020CFF2646FABA
:10C110000CF6012D07EA06073FD005D3022D36D0D5
:10C12000F0BD012D39D030D21EF8016026EA070794
:10C130000EF801709342F3D3B0F906100C449A1A2A
:10C14000D2B2072A10D9022D36D0002D14BFFF26F7
:10C15000002613462670083BB0F90610DBB2072B09
:10C160000C44F7D802F00702002AD9D01D4B012D4C
:10C170009B5C1DD017D3022DD2D12278534023705F
:10C18000F0BD13441BB20022A1E7022D25D11EF8F9
:10C19000016077400EF80170CCE71EF8016037436C
:10C1A0000EF80170C6E7227822EA03032370F0BD7F
:10C1B000227813432370F0BD11462378DB432370AC
:10C1C0000839B0F90630C9B207291C44F5D812F075
:10C1D0000702A5D0034B9B5CCFE73444AFE700BF19
:10C1E00000420100F041010070B4C47DBDF80C5064
:10C1F000022C18D0032C1FD0012C0BD0002A03DBFB
:10C20000B0F90840944201DC70BC7047039570BCE3
:10C21000FFF7B0BAC4880395013CA41A0A4621B2BC
:10C2200070BCFFF749BF0689C488013E641AB21A80
:10C23000E41A12B221B2E1E704890395E41A641A00
:10C24000114622B270BCFFF737BF00BF70B4C57D86
:10C25000BDF80C60022D1AD0032D12D0012D03D091
:10C26000039670BCFFF728BFC488E41AA41A0A46D4
:10C2700021B2002A03DBB0F90840944213DC70BC01
:10C2800070470489013C641A114622B2F1E7C48860
:10C2900005890396013CAD1AED1A621A11B22AB251
:10C2A00070BCFFF709BF039670BCFFF763BA00BF0D
:10C2B0002DE9F8430446406A002863D0A16DFEF7DB
:10C2C000F3FD052274492046FFF714FCA1790139DA
:10C2D000C9B22046FFF746FBB4F90820E588A66AF4
:10C2E000D31D48BF02F10E03DB10626A15FB03F594
:10C2F0001FFA85F8002A7BD094F82C300125AB403A
:10C3000082F83B3082F85E5082F85D50606A0368C4
:10C3100040211B6808F1FF379847BFB2B8F1000F02
:10C3200023D03744A846013E606A16F8011F03680F
:10C330001B6898470135B742EDB216D0202DF3D1D6
:10C340000121606AFEF712FF94F82C20636A520004
:10C3500083F83B2083F85E8083F85D80606A036821
:10C3600040211B6898470125DEE70121606AFEF73E
:10C37000FDFE606A002800F08D80E16DBDE8F843A5
:10C38000FEF792BD236A002B2BD0D97A626DE1B102
:10C3900072B6D97ACE0706D54048D96805682940D3
:10C3A00099610160D97A8D0706D53D4819690568FC
:10C3B0002940D9610160D97A480705D539485969BA
:10C3C000056829401962016062B61B68D96891420C
:10C3D00007D0354818603549DA6042F0804018616E
:10C3E0001960226C216D136823EA0103136068E76A
:10C3F000E26BE36C1168276A0B4306EB08091360D4
:10C400004FF0004E4E450DD016F801CB2FB33A68D1
:10C41000C2F82CE0C2F834C0D36A002BFCDA4E45D7
:10C42000936BF1D1226C236D11680B43136097B1AC
:10C43000FB7A83B1D90703D51D4BBA691A60FB7A21
:10C440009A0703D51B4BFA691A60FB7A5B0702D582
:10C45000194B3A6A1A60BDE8F883A36BD4F83480AC
:10C4600008208021D8F80020656C1CEA010F14BF59
:10C470002A43AA43C8F800201A68A56C2A431A6008
:10C480001A68A56C013822EA05024FEA51011A60C8
:10C49000E8D1B7E7276AC5E7F841010080E100E08D
:10C4A00084E100E088E100E001403F0000003F80BF
:10C4B00000E100E004E100E008E100E02DE9F04FD8
:10C4C00085B09946BDF93870BDF83CA0BB1AC1EBE8
:10C4D000090B002BB8BF5B42BBF1000FB8BFCBF11B
:10C4E000000B5B450D4616460093804648DC4D45E3
:10C4F0003A4633464CDC194613460A46C5EB090159
:10C500009B1A89B2002B0CB2B8BF5B4204EBD47407
:10C51000BE42ACBF4FF0FF3201224D450391029263
:10C520004FEA640429DC9BB201930DE0D8F8007057
:10C53000BF69B847019BE41AA3B21CB20135002CB5
:10C540002DB211DBA94518DB009B5B452A465346FB
:10C5500031464046EADCD8F8002053469769294620
:10C5600032464046B847E5E7029A1644039AA94581
:10C5700002EB030436B224B2E6DA05B0BDE8F08F70
:10C580004A462B46B94635464D4517461E46B2DD4E
:10C59000304629463E464D4607468946AEE700BF2F
:10C5A00010B404682469A44610BC604730B4046821
:10C5B000BDF808500295A46BA44630BC604700BF8C
:10C5C00030B40468BDF808500295E46BA44630BC52
:10C5D000604700BF70B40468BDF90C60BDF810502E
:10C5E00003960495246CA44670BC6047704700BF56
:10C5F00010B582B0B0F90C200191016800920022C0
:10C600000C6CB0F90A301146A04702B010BD00BF53
:10C61000704700BF01F003010129C17506D003294D
:10C6200004D0C28803894281838170470289C3880C
:10C6300042818381704700BF2DE9F0410568134EA8
:10C640006F6986B0B7420446BDF8308010D1013B17
:10C6500013441BB20093CDF804800B46AD6A20460C
:10C66000A8472368DB6AB3420AD106B0BDE8F0816F
:10C67000059304920391B84703A925680EC9E6E71C
:10C68000204606B0BDE8F041184700BFEDC50000E8
:10C690002DE9F0410568124E6F6986B0B742044635
:10C6A000BDF830800FD1013BCDF804800B440092DF
:10C6B0001BB2AD6A2046A8472368DB6AB3420AD1A1
:10C6C00006B0BDE8F081059304920391B84703A931
:10C6D00025680EC9E7E7204606B0BDE8F0411847D7
:10C6E000EDC500002DE9F04F0568DFF858B06F691F
:10C6F00085B05F450646BDF93890BDF83CA00C46B4
:10C70000904615D11F19BC420CDACDF800A0214685
:10C7100001342D6A4B464246304624B2A847BC42FB
:10C720003568F2DBEB6A5B4507D105B0BDE8F08FF9
:10C730000393B8473568039BE4E7304605B0BDE88E
:10C74000F04F1847EDC500002DE9F04387B099423E
:10C750000546BDF93840BDF83C6025D0A24212D054
:10C760000768DFF88080D7F81490C14532D18DE892
:10C7700050002846BC6AA0472B68DB6A434524D199
:10C7800007B0BDE8F083994202DD0846194603462A
:10C7900028680E96C46B01335B1A1BB22846A44668
:10C7A00007B0BDE8F0436047A24202DD13462246CF
:10C7B0001C4628680E96631C846B9B1A1BB2284685
:10C7C000A44607B0BDE8F0436047284607B0BDE87F
:10C7D000F0431847059304920391C84703A92F68B3
:10C7E0000EC9C4E7EDC500002DE9F04FD0F800E018
:10C7F000DFF89090DEF814B083B0CB450446BDF965
:10C800003080BDF834A00D4617461E4631D1CDF814
:10C8100000A0DEF824B0294633463A462046D847E1
:10C820002368CDF800A008F1FF323A44D3F824B0D1
:10C83000294612B233462046D8472368CDF800A0D7
:10C840002946D3F820B03A4643462046D8472068C8
:10C85000CDF800A0711E29444346056A09B23A4644
:10C860002046A8472368DB6A4B4506D103B0BDE8E4
:10C87000F08FD847D4F800E0C9E7204603B0BDE800
:10C88000F04F1847EDC50000F0B4002401264FF624
:10C89000FF75094F07600471C475C4810482447632
:10C8A000C4618675067685824582C1800281418198
:10C8B0008281F0BC704700BF284701002DE9F04F8E
:10C8C00085B00668BDF84450BDF93880CDF80080C9
:10C8D00004460195D6F848B00392BDF93C60BDF915
:10C8E000407089469A46D84723680195009742468A
:10C8F0005146D3F8488020463346C0472068039B02
:10C900000E930F95856C4B463A4631462046AC4611
:10C9100005B0BDE8F04F60472DE9F04F87B01746EE
:10C92000BDF9404000912546E91D059344BF2B46C3
:10C9300003F10E010268BDF8486053690294C91002
:10C9400003912B49BDF9444001968B42824645D163
:10C95000002C3CDD029B3C445E1EB6B24FF0000949
:10C9600023B2049301364D46029B002B28DD059B24
:10C97000002403EB090806E0EDB22B0604F10104E4
:10C9800011D4A6421CD0A1B211F0070F23B24FEA76
:10C990004505F1D1002BB8BF0733DB10013418F87F
:10C9A00003502B06EDD5009BD2F818B019443A4637
:10C9B00009B2019B5046D847A642DAF80020E2D1DE
:10C9C000039B01379944049B3FB2BB42CCD1D36A4D
:10C9D000074A934206D107B0BDE8F08F9847DAF8CE
:10C9E0000020B5E7504607B0BDE8F04F184700BF3C
:10C9F000EDC5000070B4BDF90C60BDF91050BDF874
:10CA0000144003960495059470BCFFF785BF00BFE2
:10CA10002DE9F04F93B090460591C1691090BDF893
:10CA200070000790BDF874909DF878A004930029D9
:10CA300000F0CD800A7A0AC9894604998A1AD2B2CE
:10CA400003EBC203BAF1010FDA780B9293F90520D8
:10CA50001E8893F802B00F9293F9064079D913B269
:10CA6000099323B20C93109B1A68A94B1193194692
:10CA700053698B4240F0A6800B9B002B55D01FFAC8
:10CA800088F300210D93C8462344DDF840900691B9
:10CA90000E930F460C46BBF1000F3FD0BDF81810A7
:10CAA0000C9B03971FFA8AF0CB1813FB00F304903A
:10CAB0000E9801440D98034409B21BB20A910893E1
:10CAC000002505E00135EBB264009B45E4B222D9B4
:10CAD000039B2B44590703D1731C18F806409EB2E0
:10CAE0002306EFD5099BBDF81000E91811FB00F1F2
:10CAF0000598BAF1010F0FFA8AF301441CD0079888
:10CB000001900093D26909B217464846089AB8477F
:10CB1000D9F80020D6E7039F5F44FFB2069B0B992C
:10CB200001330693DBB29942B5D8D36A119A934286
:10CB300043D113B0BDE8F08F0F9B191893690A9A7F
:10CB400029441F4609B2079B4846B847D9F8002038
:10CB5000B8E700230C93099385E70A9A0D9B0132ED
:10CB6000013B52B213F0FF030A920D936FD1DDF82F
:10CB70001890079BDDF83C80DDF820A04B4517D0CE
:10CB8000BAF1010F00F0C8800B9A109DCDF8049007
:10CB90000BEB8B014FEACB030A4400931146DEF8FE
:10CBA0001C405346424609B22846A047D5F800E04B
:10CBB000DEF82C30119A9342BBD0109813B0BDE828
:10CBC000F04F1847109D284698472A6854E7109A56
:10CBD0000598B2F90A308342ABDDB2F90C30434517
:10CBE000A7DD062313FB0A03002BA2DD08EBCA0313
:10CBF000002B9EDD537E2BB9049BAF2B02D9013352
:10CC0000DBB20493109BD3F800E0414B11931A461A
:10CC1000DEF81430934240F08E801FFA88F30E93B2
:10CC200008339BB2BDF81420059305230D93002310
:10CC30000A93CDF83C800FFA8AF3DDF84080CDF8F6
:10CC400018900B921FFA8AFBCDF820A099460A9AF9
:10CC5000BDF810000B9C0E9D0523194611FB002307
:10CC60002C481146C75C039702FB0B4214FA81F370
:10CC700012B21BB209920C932C462E461CE0089B64
:10CC80000999012B2AB24B4640462DD0079F0197A8
:10CC9000CDF80090DEF81CA0D047D8F800E0039B48
:10CCA0005B0801340393059BA4B25D445E44A34238
:10CCB000ADB2B6B23FF451AF039BD807DFD4079BA8
:10CCC000069A9342EBD0089B012B16D0069B01934A
:10CCD000CDF80090DEF81CA009994B4632B24046D0
:10CCE000D047D8F800E0DAE7DEF818A0079B0C99E7
:10CCF00022B2D047D8F800E0D1E7DEF818A00C99AE
:10CD00001346404622B2D047D8F800E0C7E700BF3C
:10CD1000EDC50000784701000B99109DCDF80090FB
:10CD20000531DEF8204009B2424608232846A047D4
:10CD3000D5F800E03CE7109C20469847D4F800E086
:10CD40006BE700BFF0B5C36985B004462BB30A2971
:10CD500068D00D294AD01A7A914247D3587A88422E
:10CD600044D35D688A1A05EBC205AA78002A50D020
:10CD7000E87800284DD0207E00283AD095F905E0CB
:10CD8000B4F90E00A67DB4F90A70724406FB0202E3
:10CD9000BA4262DCB4F9102030E00A2956D00D29DD
:10CDA00024D0027E002A4BD0B0F90E00A57DB4F944
:10CDB0000A60062212FB0502B2423EDD228AE381AE
:10CDC00002EBC50212B218462282A78A668A029531
:10CDD0000B468DE8C00001462046FFF719FEA37DF3
:10CDE000E28903EB430302EB4303E381012005B037
:10CDF000F0BDA67DB4F90E00B4F91020B4F814E02B
:10CE0000678A02960B468DE8804001462046FFF770
:10CE1000FFFD2979E389A27D012001FB0233E38133
:10CE200005B0F0BD0022C2819A7A817D038A01FBA0
:10CE300002330382012005B0F0BDB4F91020C4E72D
:10CE4000857DB4F91020B0F90E00BEE7028A817D1D
:10CE5000C38102EBC1030382C8E70020E0819B7A13
:10CE6000228A03FB062212B22282C7E7C181028214
:10CE7000704700BF002908BF01218175704700BFBE
:10CE800081824182704700BFC07D7047B0F90A00BF
:10CE9000704700BFB0F90C00704700BF10B4EFF34B
:10CEA000108272B6437F33B9017F012907D003296D
:10CEB0000FD00123437702B962B610BC7047124C01
:10CEC0002168A1B1114943610B6883610860586111
:10CED000EFE70F4C216881B10E4943610B68836114
:10CEE000086058610C4B4FF080511960E1E7074B27
:10CEF0004161816120601860DBE7064B416181611F
:10CF000020601860EEE700BF1CA0FF1F18A0FF1FE5
:10CF10000CA0FF1F10A0FF1F04ED00E070B5EFF3A1
:10CF2000108272B60C4C206880B10C4E002543690B
:10CF3000236073B19D6102B962B6457783689847F3
:10CF4000EFF3108272B620680028F0D102B962B601
:10CF500070BD3360EFE700BF0CA0FF1F10A0FF1FE4
:10CF6000FFF7DCBF184A30B41468002C27D00368E0
:10CF700021688B420ED2CB1A00218460C1602360ED
:10CF8000E06010600223037530BC704711688B426B
:10CF9000144608D3A2685B1A0360002AF6D18260A7
:10CFA000C460A060EEE7D268C2608460E060C568DB
:10CFB000CB1A0222A8602360027530BC70478460DF
:10CFC000C4601060DEE700BF14A0FF1FF8B5224E5A
:10CFD00034682CB32368002B3AD1204F1D4604E05F
:10CFE0003468ECB12368002B32D1A36803B1DD6053
:10CFF00020693360036825751B68BB4221D1037F1C
:10D000004560022BC46020D0FFF748FF6368002B07
:10D01000E6D023602046FFF7A5FF3468002CE1D15D
:10D02000EFF3108372B60E4A00211068116003B945
:10D0300062B628B18468FFF795FF20460028F9D131
:10D04000F8BD224600219847E0E783689847DDE76E
:10D05000013B2360E4E700BF14A0FF1FDDB6000022
:10D0600024A0FF1F024A136801331360FFF7AEBF0D
:10D0700030A0FF1F704700BF0368F0B4FBB100256C
:10D0800001249D60DC601B4C1A601C44241104F1D7
:10D0900044056A11032692009E60174F0679174BCC
:10D0A00047F8241002F1604202F5614205F01F05C5
:10D0B000012000FA05F5E6541560F0BC7047104CED
:10D0C000236843F40003236000BF0E4B0E4DA4F50C
:10D0D0008734A4F59E7401261E60234604609C6874
:10D0E000002CD0D01033AB420360F8D10023036092
:10D0F0001846E2E7008FFCBF3C92FF1F44E400E0CB
:10D100003C80044000700340407103400168A9B1B5
:10D110000B4BF0B40B441B110A4E0B4F0B4D46F852
:10D12000237003F1440202F01F0401235211A340B3
:10D13000002445F822308C600460F0BC704700BFCA
:10D14000008FFCBF3C92FF1F75D0000080E100E023
:10D15000024A034B012111601B6818470C71034000
:10D160003C92FF1F024A034B012111605B68184784
:10D170001C7103403C92FF1F024A034B01211160C6
:10D180009B6818472C7103403C92FF1F024A034BD7
:10D1900001211160DB6818473C7103403C92FF1F7E
:10D1A000F8B50E4671B17AB10746144600253B68C2
:10D1B00016F8011B1B6838469847013C0544F6D118
:10D1C0002846F8BD0846F8BD1046F8BD00B5064A29
:10D1D000036812885B6883B001A9ADF804200222BD
:10D1E000984703B05DF804FB784C0100F0B50746A2
:10D1F0008BB0002A33D0012A08BF0A2251B3212460
:10D2000000E0F4B2B1FBF2F502FB1511C8B2092936
:10D2100000F1300198BFC8B20AA988BF3730214455
:10D2200088BFC0B201F8240C661E2946002DE8D143
:10D2300033B1013CE4B20AAB23442D2203F8242C81
:10D240003B6801AA11195B683846C4F1220298476D
:10D250000BB0F0BD30228DF825202124E8E70368CB
:10D26000C9B21B6898470BB0F0BD00BF0029BABF18
:10D2700049422D2300230A22FFF7B8BF374A384915
:10D2800013681B06FCD40B6813F08003F8D172B648
:10D2900034490A78002A5FD0334A3448F0B4344C19
:10D2A000176806682568D4680C303E44143200685C
:10D2B0001268304F35442C4420440244C2F34E02DD
:10D2C0002D4E2E482E4D2F4C42F400423A603768C6
:10D2D00006682D682C4A24680C303E4400681268A9
:10D2E0002A4F35442C4420440244C2F34E02284EB7
:10D2F0002848294D294C42F400423A6037680668B4
:10D300002D68274A24680C303E4400681268254F77
:10D3100035442C4420440244C2F34E02224E23489A
:10D32000234D244C42F400423A60376806682D6869
:10D33000214A24680C303E440068126835442C446D
:10D3400020440244C2F34E021C4842F400420260F0
:10D350000B7062B6F0BC704762B6704724B00340F1
:10D3600024B00B4029A0FF1F38B003403CB003405D
:10D3700040B003402CB0034058B003405CB00340C1
:10D3800060B0034064B003406CB0034030B0034071
:10D3900038B00B403CB00B4040B00B4044B00B40A9
:10D3A0004CB00B402CB00B4058B00B405CB00B4065
:10D3B00060B00B4064B00B406CB00B4030B00B4021
:10D3C00030B42948294A2A4B2A4D6024E1210470AF
:10D3D00011701B78284C082B30D00A2B274828497D
:10D3E00037D00C2B0CBF35223D2212232A6023603C
:10D3F00002600B60234B24491B78244ABBB10123F4
:10D400000B601360224B23491B78234A012B26D93A
:10D41000042B0FD9082B1ED9102B94BF86238723EA
:10D420000B6013601D4B01221A7030BC70470B60FB
:10D430001360E7E784230B601360F3E700F58E20A9
:10D440000F490830012213232A60236002600B6019
:10D45000D0E73922F7E785230B601360E2E78023EA
:10D460000B601360DEE700BF00400740014007404B
:10D470004C92FF1F08B003400CB0034008B00B40B3
:10D480000CB00B402CA0FF1F20B0034020B00B407D
:10D490004D92FF1F24B0034024B00B4029A0FF1F72
:10D4A0000C2830B417D91023984228BF18461C46C0
:10D4B000104A114D1178181A8C42287018D00F4953
:10D4C00013700B7823B10E490E4A00230B601360D2
:10D4D00030BCFFF775BF0A2802D90C231C46E7E7CA
:10D4E000082802D90A231C46E2E708231C46DFE786
:10D4F00030BC70474C92FF1F28A0FF1F29A0FF1FC0
:10D5000024B0034024B00B4028282FD8334B2DE9FA
:10D51000F0411E5CFF2E2BD0314B1B78002B2AD103
:10D5200032062CD472B62F4D2F4C2F460123266085
:10D530002B7062B672B623681B060CD43B781BB9FD
:10D54000F4E72B78002BF1D062B602F073FB72B6D1
:10D5500023681806F5D5254B1B6800222A7062B691
:10D56000234A107843FA00F0BDE8F08100207047AC
:10D570000020BDE8F081FFF781FE3206D2D572B6F9
:10D580001C4DDFF87C801C4C06F04007FFB206F013
:10D590003F06D8F80030DFB123F01003C8F80030A0
:10D5A00001232660134A2B7062B672B623681906EF
:10D5B0000CD413781BB9ECE72B78002BE9D062B6BA
:10D5C00002F038FB72B623681B06F5D50B4BC3E798
:10D5D00043F01003C8F80030E2E700BF7C4C0100C4
:10D5E00029A0FF1F2BA0FF1F00B0034010B0034075
:10D5F00028A0FF1F2AA0FF1F00B00B4010B00B4057
:10D600000CB00B400A4A0B49136843F48053136073
:10D610000B7843B9084BC0221A70084B80F30C00FA
:10D6200000B218807047044B80221A70F5E700BFE3
:10D630002C8004402CA0FF1F21C00C4000C00C40D7
:10D64000F0B51B4B1B4E596818689A68DB6885B0AB
:10D650006C460FC4337899071DD5174A174C1378B9
:10D66000174913F0700318BF1370164A164B802722
:10D67000177000263320032226706D4608701A703A
:10D6800072B6043C45F001052046A84762B62378EF
:10D6900013F0700309D10D4B064901E0013B02D0A4
:10D6A0000A78D207FAD505B0F0BD237005B0F0BDF9
:10D6B000A84C0100010002400000024004000240AA
:10D6C0000B000240070002400A000240410D030027
:10D6D000B0F5006F0AD210B5094B1B78DB07044682
:10D6E00006D504F1A0500078C0B210BD00207047EC
:10D6F000FFF7A6FF04F1A0500078C0B210BD00BF34
:10D7000001000240B0F5006F17D238B50F4B1B78FF
:10D71000DA070D46044611D504F1A0500378AB4258
:10D720000AD00B4A137813F0700318BF1370074A1E
:10D7300005701378DB07FCD538BD7047FFF780FF15
:10D7400004F1A0500378AB42EBD1F5E701000240B1
:10D750000000024008B5F4F7F1FAF4F759FF02F0BF
:10D7600069FAFAE7844641EA000313F003036DD136
:10D77000403A41D351F8043B40F8043B51F8043B94
:10D7800040F8043B51F8043B40F8043B51F8043B9B
:10D7900040F8043B51F8043B40F8043B51F8043B8B
:10D7A00040F8043B51F8043B40F8043B51F8043B7B
:10D7B00040F8043B51F8043B40F8043B51F8043B6B
:10D7C00040F8043B51F8043B40F8043B51F8043B5B
:10D7D00040F8043B51F8043B40F8043B51F8043B4B
:10D7E00040F8043B51F8043B40F8043B51F8043B3B
:10D7F00040F8043B403ABDD2303211D351F8043BDB
:10D8000040F8043B51F8043B40F8043B51F8043B1A
:10D8100040F8043B51F8043B40F8043B103AEDD289
:10D820000C3205D351F8043B40F8043B043AF9D2DA
:10D83000043208D0D2071CBF11F8013B00F8013BAD
:10D8400001D30B8803806046704700BF082A13D3BA
:10D850008B078DD010F003038AD0C3F10403D21AD2
:10D86000DB071CBF11F8013B00F8013B80D331F806
:10D87000023B20F8023B7BE7043AD9D3013A11F886
:10D88000013B00F8013BF9D20B7803704B784370F1
:10D890008B7883706046704708B5104C08E02368A9
:10D8A00059050DD423681A050FD42368DB0411D45D
:10D8B00023685803F3D501F065F823685905F1D5BD
:10D8C00002F01CFA23681A05EFD500F07FFD2368EB
:10D8D000DB04EDD500F0C8FEEAE700BF3480044069
:10D8E00008B5FFF7D9FF00BF014B10221A8070471F
:10D8F00000200540704700BF094908B50B6830B1EA
:10D900006A461844A2F58052904202D20860184636
:10D9100008BD03F0A7FC0C2303604FF0FF3008BDE7
:10D920005092FF1FFEE700BFEFF3138070B9EFF3D3
:10D9300010836BB9EFF305825AB94FF48070EFF39F
:10D9400011832BB1984228BF184670474FF0FF3023
:10D9500070470F2A01D81846F1E7014BD05CEEE77B
:10D96000F0E300E0F0B44D1E2E46002400E0013448
:10D97000B0FBF2F302FB1300092800F130078ABF65
:10D980003730F8B2C0B206F8010F1846002BEED1BE
:10D990000A1953704CB1107815F8016F28700133D3
:10D9A000E01A834202F80169F5DB0846F0BC7047D3
:10D9B000704700BF10B40F4B53F8302092F88042EC
:10D9C0002CB1012369B182F8803010BC704703EBA1
:10D9D000C0035B681A6841B922F002021A6010BCE9
:10D9E000704782F8003110BC704742F003021A60A1
:10D9F00010BC7047B84C01001C4A02EBC00301295F
:10DA00005B6811D004291BD052F83000002280F846
:10DA1000802229B1022920D0032922D01A60704720
:10DA20004FF480721A60704752F830004FF4A272BF
:10DA300080F880121A601A6822F020021A6070477B
:10DA400052F830104FF4A272012081F880021A605F
:10DA50001A6842F020021A60704740F203121A60FE
:10DA600070474FF481721A60704700BFB84C0100D4
:10DA7000212848D8F8B5042A44D8DFE802F0484BFA
:10DA80004E0345004FF410262B4B03EBC0030D460D
:10DA90005C68216811F4E06148D0284B284A294984
:10DAA000C3F89C2104F140422748C3F8A411A2F511
:10DAB0009221264FC3F8A0017C292548C3F8A871FC
:10DAC000C3F8AC012CD9A2F594237C2B2AD9A2F55A
:10DAD00096237C2B28D9A2F598237C2B29D9A2F553
:10DAE0009A227C2A27D81B4872B6236823F4702315
:10DAF00043F08072C4F384011643236040F8215040
:10DB0000266062B6F8BD70474FF43026BCE74FF48C
:10DB10000026B9E74FF44026B6E74FF42026B3E7D6
:10DB20000D48E1E70D48DFE70D48DDE7FFF764FF4B
:10DB3000B3E70C48D8E7F8BDB84C01000082FF1FDE
:10DB4000F188FF1F9988FF1FC588FF1F6D88FF1F81
:10DB50004188FF1F2C93FF1F5492FF1F8C92FF1FC1
:10DB6000DC92FF1F0C93FF1F1A4B03EBC00010B495
:10DB7000426802F14043A3F592217C2923D9A3F501
:10DB800094217C290DD9A3F596217C291FD9A3F5D1
:10DB900098217C2919D9A3F59A237C2B11D80E4CF6
:10DBA00000E00E4C72B613680D4823F08773C2F381
:10DBB000840123F4803343F08073136044F8210020
:10DBC00062B610BC7047074CECE7074CEAE7074C1D
:10DBD000E8E700BFB84C01002C93FF1F8C92FF1F99
:10DBE000B1D900005492FF1F0C93FF1FDC92FF1F5E
:10DBF00030B4054B054D064C002210211A602A60F6
:10DC00002060196030BC704714D0034004D003403A
:10DC100000D00340282838B52ED0002904464FDD17
:10DC20005F4B1B78012505FA03F28A4202D82128AE
:10DC300037D938BD0338C2B2012A3AD9202C4AD08C
:10DC4000192C48D0574A126802FB011222FA03F33A
:10DC50001D2800F29B80DFE800F0928B847D99996B
:10DC6000766F99999999999999999968615A53995F
:10DC70004C99999999999945494B1B780B2B08D93F
:10DC80000C2B1CBF0C3B19410846BDE83840FFF780
:10DC9000B9BCC3F10C0399400846BDE83840FFF712
:10DCA000B1BC2946FFF786FE2946BDE83840FFF79C
:10DCB000A3BE3D4A126802FB011222FA03F3C7E732
:10DCC0002128B6D80021FFF775FE20460121BDE8C6
:10DCD0003840FFF791BE354A126802FB011222FA62
:10DCE00003F3B5E73249334A0B604FF451731360C5
:10DCF00038BD3149314A0B604FF45173136038BD60
:10DD00002F49304A0B6040F24443136038BD2E491E
:10DD10002E4A0B6040F24443136038BD2C492D4A13
:10DD20000B6040F24443136038BD2B492B4A0B6013
:10DD300040F24443136038BD29492A4A0B6040F23F
:10DD40004443136038BD2849284A0B6040F24443DD
:10DD5000136038BD2649274A0B6040F244431360E4
:10DD600038BD2549254A0B6040F24443136038BD55
:10DD70002349244A0B604FF45173136038BD224984
:10DD8000224A0B604FF45173136038BD212C3FF6CB
:10DD900050AF7F29D4BF00210121204693E700BF67
:10DDA0003493FF1F088003400890034008800B4015
:10DDB00010800B4048A0044018800B404CA0044049
:10DDC0001880034008B004401080034004B00440B1
:10DDD0004080034018C004403880034014C0044011
:10DDE0002880034010B00440208003400CB0044061
:10DDF0003080034010C00440488003401CC00440F1
:10DE00001890034034900440109003403090044038
:10DE100038B1102828BF1020044AC3B210781370FC
:10DE20007047024A01231078137070473493FF1F24
:10DE30002DE9F8430E4680463249334D304603F013
:10DE400097F947F6122300281ABF1D464FF0020922
:10DE50004FF00109002425FA04F002F093FF4FF07F
:10DE60005E51074602F0E6FF0146304603F094F9A2
:10DE700030B90134072CEED1E80902F083FF0746E0
:10DE80003146384603F08AF84FF07C5102F0C8FE64
:10DE900003F0BCF94FF6FF729042A8F1030328BFCC
:10DEA0001046012B29D9B8F1170F17D8174B23FAB1
:10DEB00008F303F0010383F0010223B9B8F1190F4D
:10DEC0000FD0BDE8F883124B124D13491A6044EA93
:10DED000C9042A6008601C60BDE8F883B8F1200F0F
:10DEE000ECD10E4B0E4D0F49002244EAC9041A60D2
:10DEF0002A6008601C60BDE8F8830B4B0B4D0C4991
:10DF0000F2E700BF001BB740006CDC026006F000C7
:10DF100000800340048003400880034000800B40E1
:10DF200004800B4008800B400090034004900340A5
:10DF300008900340212801D8FFF73CBD704700BF7F
:10DF4000212806D8044B53F8303093F80002C0B2B1
:10DF500070470020704700BFB84C0100212801D84D
:10DF6000FFF74ABD704700BF72B60C490C4B0D4A13
:10DF70001B680868126862B6520102D5322B88BF4E
:10DF800001300949C3F5BB334FF47A72FF33A1FB6B
:10DF9000031302FB00F000EB9310704730A0FF1F4B
:10DFA00018E000E004ED00E0ABAAAAAA2DE9F843CE
:10DFB000054672B6204F214B214A1B683C68126807
:10DFC00062B6520102D5322B88BF013495B3C3F536
:10DFD000BB331C4EDFF86490DFF86480FF334FF4EE
:10DFE0007A72A6FB031302FB04F404EB931472B6DB
:10DFF000D9F800103A68D8F800E062B6C1F5BB3332
:10E00000FF33A6FB03031EF0806FC4EB93134FF4A2
:10E010007A7002D0322988BF013200FB0233B3F597
:10E020007A7F04D3013D05D004F57A74DFE701F06F
:10E0300001FEDCE7BDE8F88330A0FF1F18E000E038
:10E0400004ED00E0ABAAAAAAF8B52D4B2D49DFF8E4
:10E05000D0E0DFF8D0C02C4E2C4D2D4C2D4A2E4F49
:10E060004FF4000018604FF0807018604FF000709F
:10E0700018604FF0806018604FF00060186000205A
:10E08000086028234BF6FF71CCF80010CEF8003062
:10E09000336013602B6023603B60B362936209229C
:10E0A00045F8242CC4F8D80F05F57F65C7F8D41FB0
:10E0B00007F5FF2707F5FA67C6F8F83F2B6006F566
:10E0C000FF26C4F8D42F05F5FD2504F5FF2438609C
:10E0D00006F2F4761148316005F5FF6504F5FD643C
:10E0E0002B6023600260FFF76BF91920FFF75EFFDA
:10E0F00001F08EF940F21310BDE8F840FFF756BF6B
:10E1000008E100E0048003401480034024800340C1
:10E110002C8003401C8003403480034000800B406F
:10E120000C800340088003402B4A2C491368F0B54B
:10E1300043F4006313600A78294F2A4E2A4D2B4C72
:10E140002B490023092A3B7033702B7023700B700E
:10E150003DD01A2A21D0274B1B780A2B25D01F2B04
:10E1600030D01F2827D8002002460125224B234CFF
:10E170001A7023495D7004224FF0020E88273C2656
:10E18000402598729A704FF4004083F813E05A7556
:10E190001F74DE7025700860F0BD1A4B40F2133218
:10E1A0001A60144B1B780A2BD9D1174B4FF45172BC
:10E1B0001F281A60D7D9C0F34432C0F3471500F0C6
:10E1C0001F00D3E7114B4FF451721A60C9E7104B8F
:10E1D00040F213321A60BEE7348004403593FF1FCB
:10E1E000A4A0FF1F39A0FF1FACA0FF1FA5A0FF1F09
:10E1F00038A0FF1F3693FF1F00B006402FE400E059
:10E2000004E100E004D0044010B0044000D0044019
:10E210000CB0044009B140F08000174A13789842CE
:10E2200016D010B4154C246824050FD503F07F03D5
:10E230000A2B1CD01F2B11D0002900F07F0114BF26
:10E24000602344230A290DD01F2902D0107010BC6E
:10E2500070470B4943F440730B60F7E7084B002409
:10E260001C60E9E7074943F440730B60EEE7054B98
:10E2700000241C60E0E700BF3693FF1F3480044099
:10E2800000D0044010B00440124B1A7882420CD0E7
:10E2900011490968090507D5092A16D01A2A0AD092
:10E2A00009280DD01A2801D0187070470B4A40F287
:10E2B00013311160F8E7094A002109281160F1D1F2
:10E2C000074A40F213311160EEE7054A0021116060
:10E2D000E6E700BF3593FF1F3480044004D00440BC
:10E2E0000CB004402DE9F84F234B1B681A053BD5B1
:10E2F000224B1B680BB101221A70DFF89090204D61
:10E3000099F80040DFF888801E4E0134272C8ABF20
:10E310004FF0000A5FFA84FA54460746AB462B7862
:10E320009C4216D1FFF700FB40281FDC33791B0607
:10E33000F5D59BF800300133272B86BF002213460A
:10E34000DAB218F80330DBB2F3712A702B789C42F2
:10E35000E8D00D490B4BFFB20120BC2208F8047035
:10E36000087089F800A0DA70BDE8F88FFF28D6DDC4
:10E3700001F060FCD3E700BF34800440A8A0FF1F79
:10E38000A5A0FF1F00B0064038A0FF1FACA0FF1FD4
:10E390003CA0FF1F10B5044C237823B101F04AFCC8
:10E3A0002378002BFAD110BD38A0FF1F054A064B79
:10E3B00010781B78C0B2DBB2984238BF4030C01A28
:10E3C000704700BFA4A0FF1F39A0FF1FF0B4384B57
:10E3D0001A7912F0300F2CD072B6997D01F0FF023D
:10E3E00000293DD062B6334F334938780D78334E2B
:10E3F0001C46C0B2EDB2431C402BE17928BF00237C
:10E40000AB4202F1FF32C9B21CBFF154184612F000
:10E41000FF02F0D12A4B1B68C2B23A704BB1A8423E
:10E4200036BFC5F14005401B40192728C4BF012253
:10E430001A701F49CA78D2B2150616D452060DD5E5
:10E440001B4B1B795B0609D51E4B1F491B6800221D
:10E450000A7003B11A70164B3C22DA70F0BC704798
:10E460004022D9795A7462B6E3E70B791C06E5D5E8
:10E47000164B174E1C783378E4B2DBB29C420ED0B8
:10E48000144D01E0A3420AD00133282B28BF0023FA
:10E490000879E85CC0B2C871087D0728F2D9DBB200
:10E4A000034933700B79180644BF7C23CB70C5E752
:10E4B00000B00640A4A0FF1F39A0FF1F64A0FF1FEB
:10E4C00034A0FF1FA8A0FF1F38A0FF1FACA0FF1F94
:10E4D000A5A0FF1F3CA0FF1F2DE9F84F214B1B6893
:10E4E00007460BB101221A70DFF888901E4D99F88B
:10E4F0000040DFF884801D4E0134272C8ABF4FF086
:10E50000000A5FFA84FA5446AB462B78A34216D130
:10E51000FFF70AFA40281FDC33791B06F5D59BF874
:10E5200000300133272B86BF00221346DAB218F8D9
:10E530000330DBB2F3712A702B78A342E8D00C4988
:10E540000A4BFFB208F804700120AC22087089F869
:10E5500000A0DA70BDE8F88FFF28D6DD01F06AFB75
:10E56000D3E700BF24A1FF1F21A1FF1F00C0064069
:10E5700020A1FF1F28A1FF1FB8A0FF1F1C4BDFF821
:10E5800094C01A681B49F0B542F480521A4D1A60C3
:10E59000DFF884E0194F1A4E1A4C00238CF8003033
:10E5A0004FF451722B701F2840F213358EF8003053
:10E5B0003B70337025600A6012D819460124124A54
:10E5C000124D11701248547000212C27402693726E
:10E5D0004FF4003491701174D7702E700460F0BD48
:10E5E000C0F34431C0F3471400F01F03E7E700BF56
:10E5F000348004400CC00440B5A0FF1F21A1FF1FC0
:10E6000020A1FF1F08C0044000C0064031E400E024
:10E6100004E100E0B4A0FF1F28A1FF1F034B1B680B
:10E62000DB0401D5FFF758BF704700BF34800440BA
:10E6300010B5044C237823B101F0FCFA2378002BA9
:10E64000FAD110BD20A1FF1F054A064B10781B7898
:10E65000C0B2DBB2984238BF4030C01A704700BF2A
:10E66000B4A0FF1FB5A0FF1F30B42B4B1A7994063E
:10E670001FD52A48DA790378294901333F2B0978D5
:10E68000C8BF00238B42D2B203D0264CD9B2E25489
:10E690000170254A116861B1244A1278D2B29342BE
:10E6A00036BFC2F140029B1A9B18272BC4BF01231F
:10E6B0000B70194AD378DBB2180611D45A060DD55F
:10E6C000154B1B795B0609D5194B1A491B680022AB
:10E6D0000A7003B11A70104B2C22DA7030BC7047EC
:10E6E00011790906EAD5144910480C780178C9B2A5
:10E6F0008C420DD04A1C272A84BF00210A460F4DA8
:10E70000054C98BFD1B2AA5CD2B2E2710170D5E7D4
:10E710006C21D170D2E700BF00C00640B4A0FF1F3B
:10E72000B5A0FF1FE0A0FF1FB0A0FF1F21A1FF1F8A
:10E7300024A1FF1F20A1FF1F28A1FF1FB8A0FF1FBA
:10E7400021282FD8184B195CFF292BD0174B184ABA
:10E75000DFF870C003EBC000F0B54368DFF868E095
:10E76000144F154D154E00241C60DEF800300120BA
:10E7700043F020038840CEF8003014604FF4A073BB
:10E7800038602E60C2F800C0013BFDD113689B05C4
:10E79000FCD42023013BFDD1094B09B233F8110011
:10E7A00080B2F0BD00207047C84D0100B84C010098
:10E7B000005004400850044004500440000002038C
:10E7C0000051044080014A0038800440431E032B5E
:10E7D00014D872B60A4951F8230068B170B4094CD4
:10E7E000058834F81320466841F82360521B24F84A
:10E7F000132062B670BC704762B670470020704745
:10E8000084A1FF1F4CA3FF1F013803280BD872B649
:10E81000074B53F8203043B100205B680130002BD8
:10E82000FBD162B67047002070471846F9E700BF79
:10E83000D8A1FF1F30B472B62B4A13781D0706D536
:10E840002A4B196A002936D0996A002941D0537899
:10E850001C0706D5254B196C00293ED0996C002960
:10E8600039D09378190705D5204B196E002936D079
:10E87000996E89B1D3781B0707D51C4BD3F880203C
:10E880007AB3D3F8882011213AB162B6184B00222E
:10E890001A7030BC00F04ABE0D21154C154D22787F
:10E8A00043F8315003EBC1030830013A586022703D
:10E8B00062B630BC704704220D4C0F4D217843F8EE
:10E8C000325003EBC20308304A1E5860227062B611
:10E8D000EFE70521E1E70921DFE70822ECE70C2259
:10E8E000EAE71022E8E700BFEC4D01000080FF1FBF
:10E8F00001A2FF1FC800400088004000431E032BF8
:10E900001DD81B4A400140F0100030B4104472B6CC
:10E91000184CE25C032A1BD8DFE802F0021215173C
:10E9200003220D88E25410F0080F14BFC823882377
:10E9300043EA054308310360416062B630BC70476A
:10E9400008300222EDE70522EBE708300422E8E771
:10E95000094A52F8230038B1084A52F823004160AE
:10E9600042F8231062B6E9E742F82310034AF7E7BA
:10E970000080FF1F10A2FF1FD8A1FF1FE8A1FF1FEB
:10E9800000BE70472DE9F04FDFF818B3DFF818A389
:10E9900087B044E0AD4F4FEA930807EBC809013E4A
:10E9A000D9F8042003F00803F6B2A2F1080003F03E
:10E9B000FF04002B40F0018157F838301B0C99B24E
:10E9C00022F8081C002B00F0EF80A14B22F8064C27
:10E9D00042F8044C53F82620002A00F0CF819D4DC8
:10E9E00055F8263058609C4C45F8260034F816300F
:10E9F000194424F8161000F079FD002800F0C281B7
:10EA0000964A974B19F0080F00F1080018BF1346FB
:10EA1000C9F8040047F8383008238BF800309BF819
:10EA20000040E4B265071CD58E4B1B78B3B18E490C
:10EA30000A7802F0FF0322B1013BDBB20B7003B98D
:10EA400000BE8A490A7802F0FF032AB1013BDBB21B
:10EA50000B70002B00F0688100F066FE04238BF839
:10EA6000003004F0080303F0FF02002B00F0C9801F
:10EA70009AF80030DBB21E098CD19A08DFF8CC91ED
:10EA800059F8321009EBC200C1F383010139406823
:10EA90000C2900F28580DFE801F07A7A8383838392
:10EAA00083834683838307000168714D4068714FFB
:10EAB000714E6860296088B240F281610024674B22
:10EAC00049F832304FF0010E88423C60C9F81040DE
:10EAD000C9F8184086F800E05C4A00F2E780B0F51B
:10EAE000D06F80F01B82B0F5817F00F0D98100F2F9
:10EAF0006981802800F02A82822840F0D781A98885
:10EB000001F07F01042900F2D1815C485C4A890050
:10EB100008441470547001788C0740F1608382F8C7
:10EB200000E0022173E1534F3A682AB3554B524E2D
:10EB3000554819883478057840298E4645F00208F2
:10EB400028BF4FF0400E002C84F001043470CEEB4F
:10EB500001010CBF8824C82409EBC80689B285F0DE
:10EB6000010544EA0E447260198049F83840724445
:10EB70000570002965D03A603D4B1A88B2F5A06F48
:10EB80000ED100219A785970404B1A7008E038492C
:10EB90003F4C0D68A54200F09880304949F832108A
:10EBA0003C4A0123137037E72C4A2D4B19F0080F0C
:10EBB00018BF134647F838302EE700F0B7FC364A46
:10EBC000364952F82630002B00F0E38058688C5DFF
:10EBD00042F8260003F10802C9F80420032C05D8E6
:10EBE000DFE804F02C02292602228A551A8819F03F
:10EBF000080F0CBF8823C82343EA024347F8383084
:10EC00000AE7E00700F19380210600F1D180A20716
:10EC100006D5234A234913780220DBB2137008700B
:10EC2000E30602D51F4B10221A7007B0BDE8F08F23
:10EC300004228A55DAE705228A55D7E703228A5546
:10EC4000D4E7BEF1400F18BF002294E70080FF1FF9
:10EC500084A1FF1F30A1FF1F4CA3FF1FC80040006D
:10EC6000880040000CA2FF1F95A1FF1F80A2FF1F7C
:10EC7000F8A1FF1F2CA1FF1F94A1FF1FC020074078
:10EC800004A2FF1F40A1FF1F00A2FF1F9820074002
:10EC90002109000394200740D8A1FF1F10A2FF1FE5
:10ECA000882007408020074090200740B0F5106F73
:10ECB00000F07C8140F2A38040F62112904240F0A7
:10ECC0007B82A54A012313706AE74C68A3498C42F2
:10ECD0007FF463AF0178A9297FF45FAF41784529BC
:10ECE0007FF45BAF8178C2297FF457AFC1786B297D
:10ECF0007FF453AF9A489B4E0178347881F0010538
:10ED0000002C41F0020105700CBF8820C82084F05F
:10ED1000010449F8310009EBC10193483470002522
:10ED200005244D60047038E700F064FF94E68F4BD3
:10ED300089488B491A614FF0020E80F800E08C4F31
:10ED40000A708C49196099608B4E8C4D8C4C9A617D
:10ED50000D213970FF213170DFF84CE229702270EB
:10ED6000884D894A8EF800109F27012406F8047CFC
:10ED70005D600470DA6007B0BDE8F08F43F82600EC
:10ED8000824D30E6824A47F8380013780133137019
:10ED900042E68B5D032B00F2BA8001A252F823F009
:10EDA00019EA000019EA0000F9ED0000F3ED000097
:10EDB0006F49724B80220D2008701A70A2077FF5F0
:10EDC0002FAF26E740F20232904240F0ED81AA8850
:10EDD00002F07F02042A69D86D88002D66D164494B
:10EDE000CDF804E0920011440A7842F002020A7061
:10EDF000C1E101238B550FE600238B550CE6B0F5DE
:10EE0000086F53D16349644A097811707146ED88DF
:10EE10008D4280F0E88252480478402DAE4644F09E
:10EE2000020C28BF4FF0400E02EB0E0309EBCC01A1
:10EE3000029301234A604FEA0E48CEEB050101938D
:10EE40000025C82242EA080384F0010249F83C3058
:10EE500035700270DFF814C1424BDFF8048149BB02
:10EE6000BEF1400F7FF42DAF42F0020C09EBCC0352
:10EE7000029ADFF8F8E05A608DBB0D0445F0880572
:10EE80009DF804304EF83C500A4433700470134629
:10EE900040297FF416AF0021404A3B60118010E703
:10EEA000AA8802F07F02042A40F28B81304A0F23A5
:10EEB000137006E74029D7D942F002020CEBC200DA
:10EEC000029E4660BDB19DF8045035481D70334622
:10EED000403988F8004040334CF83200DCE79DF8B8
:10EEE000043033700D04029B047045F0C8050B44D8
:10EEF0004EF83C50CCE79DF804501D70029B1D4815
:10EF000088F80040403940334CF83200C4E719F02B
:10EF1000080F0CBF022303238B557DE521494A6866
:10EF2000002AC3D06C88B5F804E003E00C314A68CD
:10EF3000002ABBD00B88A342F8D14B887345F5D18A
:10EF4000240A032C0CBF1178098960E7124A0221B8
:10EF5000147054705BE700BF942007400100040068
:10EF600000A2FF1F94A1FF1F95A1FF1F0080FF1F9C
:10EF7000C0200740880040008820074080200740CC
:10EF80009820074044A1FF1F98A1FF1F30A1FF1F39
:10EF900001A2FF1F0CA2FF1F04A2FF1F40A1FF1F21
:10EFA000C8004000F04D01008C200740B248116AB3
:10EFB000AC7804700C0600F19881D9F82820AF498C
:10EFC000100600F1DB81D9F83020AC49120600F1BF
:10EFD000D081D9F83820A949130600F1C581D9F8A4
:10EFE0004020A649150600F1BA81D9F84820A34966
:10EFF000140600F1AF81D9F85020A049100600F1A5
:10F00000A481D9F858209D49120600F19981D9F8B8
:10F0100060209A49130600F18E81D9F8682097493B
:10F02000150600F18381D9F870209449140600F187
:10F030007881D9F878209149100600F16D81D9F8CE
:10F0400080208E49120600F16181D9F888208B4911
:10F05000130600F15581D9F890208849150600F172
:10F060004981D9F898208549140600F1FF80844829
:10F07000844A854901908548854D864C0497002334
:10F080000596029580460F4616461D460394306845
:10F0900028B1446800F04AFA2046002CF9D1002338
:10F0A0003360029B38681A46002342F8253028B1A5
:10F0B000446800F03BFA2046002CF9D100223A6067
:10F0C000019A98F800301146002241F8042B039A67
:10F0D0000191023B4FF0000122F81510032B07D8D5
:10F0E000DFE803F05D025D024FF0010388F80030B5
:10F0F0000135042D06F1040607F1040708F10108A3
:10F10000C5D1654C654D2278654B049F059E002155
:10F11000100729701A7000F19280624962780A70B3
:10F120000021C9F83010C9F838101107DFF84C81F8
:10F130006ED4A2785C49DFF844810A70002112077E
:10F14000C9F85010C9F858104BD4E27857494B4CC5
:10F150000A7013074FF00001C9F87010C9F8781051
:10F1600000F1AE8033780193002283F00105C9F8E5
:10F170009020C9F898200021029188468E460A46C0
:10F180004B48047844F0020C09EBCC030393019B39
:10F19000002B039B5A600CBF8822C82252E64FF016
:10F1A000000388F80030A3E7B0F5A06F7FF47EAECF
:10F1B000012300250193DEE740F621229042F7D09B
:10F1C00074E66D88002D7FF471AE3A49CDF804E005
:10F1D000920011440A7822F002020A70CBE7022161
:10F1E00015E600F083F9002800F0EB800830324A81
:10F1F000C8F86400C8F8602000F078F9002800F032
:10F20000DA8008302D4AC9F86C00C9F868209CE7FC
:10F2100000F06CF9002800F0E0800830264AC8F8B9
:10F220004400C8F8402000F061F9002800F0CF80C9
:10F230000830224AC9F84C00C9F8482079E700F0A4
:10F2400055F9002800F0A58008301B4AC9F82400B1
:10F25000C9F8202000F04AF9002800F09480083016
:10F26000164AC9F82C00C9F8282056E7D1F89C00A6
:10F27000083800F05BF9FAE60CA2FF1F0080FF1FC0
:10F28000E8A1FF1F84A1FF1FD8A1FF1F10A2FF1F2D
:10F2900030A1FF1F4CA3FF1FEC4D010001A2FF1F77
:10F2A000C4200740C8200740CC200740D02007409A
:10F2B00000A2FF1FC020074088004000C800400097
:10F2C00000F014F9002870D008304F4AC4F88400C8
:10F2D000C4F8802000F00AF9002860D008304B4ABA
:10F2E000C9F88C00C9F888203CE7506A083800F05B
:10F2F0001DF962E6D1F89400083800F017F9B0E67D
:10F30000D1F88C00083800F011F9A4E6D1F8840097
:10F31000083800F00BF998E6C86F083800F006F9D5
:10F320008DE6486F083800F001F982E6C86E0838AB
:10F3300000F0FCF877E6486E083800F0F7F86CE665
:10F34000C86D083800F0F2F861E6486D083800F042
:10F35000EDF856E6C86C083800F0E8F84BE6486C63
:10F36000083800F0E3F840E6C86B083800F0DEF833
:10F3700035E6486B083800F0D9F82AE6C86A08383C
:10F3800000F0D4F81FE62A78C9F8280001322A7064
:10F39000C3E62A78C9F8200001322A705AE72A7891
:10F3A000C9F8880001322A70DCE62A78C4F88000A7
:10F3B00001322A708EE72A78C9F8680001322A7073
:10F3C000C3E62A78C8F8600001322A7014E72A7868
:10F3D000C9F8480001322A70ABE62A78C8F8400024
:10F3E00001322A701FE740298E4628BF4FF0400E99
:10F3F00002EB0E0302930123CEEB01014FEA0E480C
:10F4000000250193BCE600BF88004000C800400012
:10F41000F8B500F0F9FC294B29482A4C2A4F2B4D0E
:10F42000DFF8BCC0DFF8BCE0294E00221A605A6049
:10F430009A60DA601A615A619A61DA611A625A62F4
:10F440009A62DA621A635A639A63DA631A645A64D4
:10F450009A64DA641A655A659A65DA651A665A66B4
:10F460009A66DA661A675A679A67DA67C3F880207D
:10F470000168C3F8842041F480210160C3F30721AF
:10F480002170C3F30740134938701B0E2B70FF2304
:10F490008CF80030104D8EF8003010480B700123AE
:10F4A000337084F8642070264FF40074102207F83B
:10F4B0002C3C2E70046081F8F820F8BD0080FF1FFE
:10F4C000348004409C200740B0200740B42007400F
:10F4D000942007401020074049E400E008E100E0E4
:10F4E0008020074088200740704700BF72B60D4853
:10F4F0000268B2FA82F30F2B10DC4FF00041D940C2
:10F5000022EA0102026062B6074803EBC303DB0094
:10F51000C2180021C15010465160704762B60020E9
:10F52000704700BF3893FF1FBC83FF1F0D4B0E4A6F
:10F53000C31AA2FB03231B090F2B0CD80B4A12780A
:10F5400052B972B60A484FF00041026821FA03F33B
:10F550001A43026062B67047064A1278002AF0D059
:10F56000FFF768B9BC83FF1F398EE33801A2FF1F84
:10F570003893FF1F0CA2FF1F38B50E4B0E4C1B68B3
:10F58000218805468BB1B1F5917F05D20B4A4B1C02
:10F5900055549BB2238038BD00220848984700216B
:10F5A000064A55540123238038BDB1F5917FEDD330
:10F5B00038BD00BF38A2FF1F56A3FF1F5CA3FF1F6B
:10F5C0002DE9F843214E224F3168012380463B70DC
:10F5D000B1B1204D4B8801EB8302013300240F2B86
:10F5E000C2F808802C7004D84B8000233B70BDE823
:10F5F000F88340230B800320FFF780F93460F4E7A1
:10F60000DFF8549099F80030002BF0D0114D45F6FA
:10F61000215408E0013C12D02B7883B900F00AFB9A
:10F6200099F800307BB10320FFF7EEF80528F1D8F8
:10F63000FFF75CFF014630600028EBD0CAE70123EA
:10F640002B70BDE8F883BDE8F88300BF54A2FF1F0C
:10F6500028A2FF1F58A2FF1F0CA2FF1F1201F8B51E
:10F66000D5B2A1B3012943D04378044600781B06E4
:10F6700043EA004040F4704045F004068F1E3043DA
:10F68000FFF79EFF022F04F1020314D9053414F88A
:10F69000023C14F8032C14F8010C1B0443EA022367
:10F6A000334343EA0060033FFFF78AFF022F2346FC
:10F6B00004F10304EBD8022F23D0012F0DD045F421
:10F6C000774040F00500BDE8F840FFF779BF1448E7
:10F6D0002843BDE8F840FFF773BF187845F4770575
:10F6E00045F0060545EA0020BDE8F840FFF768BF91
:10F6F00003780C4845EA03452843BDE8F840FFF786
:10F700005FBF1A78587845F0774545F0070545EA18
:10F71000022545EA0040BDE8F840FFF751BF00BFB1
:10F7200006F0F70007F000F738B5084B1C7824B94D
:10F73000074D296809B14B8803B938BD9B000B8080
:10F740000320FFF7DBF82C6038BD00BF28A2FF1FA5
:10F7500054A2FF1F2DE9F041AD4E33680746002B40
:10F7600000F092801D885A88910803EB81010432D1
:10F77000AA428C6842D25A8004F00F064FEA14283D
:10F78000A449A6F1080208F00F00C4F30313062AE7
:10F7900000F101050B701AD9B31E012B5FFA88F036
:10F7A0004ED9052E48D0042E00F0A481731F022BE1
:10F7B0007FD90F2E0ED1F72842D8F02802D0964BD1
:10F7C0001B883BB1FFF7D8FE0020BDE8F08127B1D0
:10F7D000BD4202D00020BDE8F081082EC4F30333FF
:10F7E00000F08780092E11D00A2E40F094800A2B59
:10F7F000F0D18A4B8A4A1B68A02181E01846FFF7A6
:10F8000095FE0420FEF7E2FF3060B5E7092BE1D159
:10F81000270E00F07B81834B814A1B689021C4F343
:10F8200007461170EDB2FCB2002B00F09D8022461D
:10F8300031462846984797E0F02843D9F72841D029
:10F84000F1380E28C6D801A353F820F003FA0000BF
:10F85000E7F90000D5F90000D5F70000D5F7000062
:10F86000C7F90000D5F70000A7FA0000D5F700009F
:10F8700071FA00008BFA0000AFF90000D5F7000024
:10F8800097F900007BF90000674B1B78002BA1D093
:10F890000420FEF79BFF0346306000289AD00588BD
:10F8A000002D7FF460AFFFF741FE35602846BDE8CC
:10F8B000F081FFF761FEC4F30740FFF75DFE072EFE
:10F8C00002D1200EFFF758FE534B584A198858486A
:10F8D0001468584D524A017000270E0AF0201F800C
:10F8E0002E7010700CB301225348A0470120BDE8D0
:10F8F000F081082B7FF46EAF504B494A1B68802182
:10F90000C4F307461170EDB2240E6BB328462246AD
:10F910003146984728E00B2E11D10B2B7FF45AAFBC
:10F92000474B3F4A1B68B021EAE7464B1B68002B58
:10F9300000F0FB80404898470120BDE8F0810C2E84
:10F9400040F000810C2B7FF445AF3F4B344A1B68DD
:10F95000C0211170EDB2C4F30746002B00F0C8803F
:10F9600028463146240E98473849314A314B0D70AC
:10F9700016701C700120BDE8F081354B1B68002B10
:10F9800000F0D6809847C4F30746254BEDB2240E0D
:10F9900083F80080E8E72F4B1B68002BF2D12E4B39
:10F9A0001B68A3B1FE209847C4F30746EDE72B4B35
:10F9B0001B68002BE6D1284B1B6843B1FC209847FD
:10F9C000C4F30746E1E7264B1B68002BDAD1C4F3EA
:10F9D0000746DAE7234B1B68C4F30746002BD4D055
:10F9E00030469847D1E7204B1A68002AEFD0260C02
:10F9F000630C06F07F0003F47E531843F6B2904781
:10FA0000C3E71A4B1B68C4F30746002BE8D1BCE7D9
:10FA100060A2FF1F5AA3FF1F56A3FF1F3CA2FF1F98
:10FA200054A3FF1F70A2FF1F0CA2FF1F38A2FF1FCD
:10FA300058A3FF1F59A3FF1F5CA3FF1F68A2FF1F4E
:10FA40006CA2FF1F50A2FF1F2CA2FF1F5BA3FF1F72
:10FA500018A2FF1F1CA2FF1F20A2FF1F5CA2FF1FF6
:10FA60004CA2FF1F64A2FF1F34A2FF1F48A2FF1F6A
:10FA70003F4B1B68002B85D13E4B1B68002BA6D04B
:10FA8000FA209847C4F307467FE73B4B1B68002BDF
:10FA90007FF478AF374B1B68002B98D0FB2098473A
:10FAA000C4F3074671E7354B1B68002B7FF46AAF40
:10FAB000304B1B68002B8AD0F8209847C4F30746C8
:10FAC00063E70E2B7FF486AE2D4A2E4B1268E021A1
:10FAD0001970002A47D0260C610C06F07F0301F450
:10FAE0007E511943EDB2A1F5005128469047F6B278
:10FAF000240E39E7FFF740FDC4F30740FFF73CFD54
:10FB0000200EFFF739FD0020BDE8F0811E4B1D4A95
:10FB10001B6880211170EDB2C4F3074683B13146F2
:10FB200028463A4698473C461EE70120BDE8F0814A
:10FB3000104B1B68002B3FF44AAFFF20984746E765
:10FB40001C4611E70D2EBCD10D2B7FF443AE0F4B9D
:10FB50000C4A1B68D0211170EDB2C4F30746002B8C
:10FB60007FF4FEAEC4E7C4F30746EDB2240EFBE615
:10FB700044A2FF1F20A2FF1F24A2FF1F14A2FF1FE9
:10FB800030A2FF1F54A3FF1F68A2FF1F40A2FF1F48
:10FB900038B5164D2868E0B101884488A14213DDCC
:10FBA00003191B7A83B104F10803C2180C1B00234C
:10FBB00002E012F8011F21B10133A342F9D120461E
:10FBC00038BD1C46204638BDFFF7B0FC0020286039
:10FBD00038BD074B1B780BB9002038BD0220FEF75B
:10FBE000F5FD28600028D7D1F6E700BF7CA2FF1FF3
:10FBF0000CA2FF1F0D4B1B78BBB910B50C4C216834
:10FC000003F0FF024B883F2B07DC07330B4401F165
:10FC1000470003F8012F8342FBD140230B800120D2
:10FC2000FEF76CFE0023236010BD704774A2FF1F17
:10FC300078A2FF1F38B5224C237803B138BD0123C9
:10FC40002370FFF7A5FF70BB00F048F840BBFEF73C
:10FC5000ADFB10BBFEF7F8FCE0B900232370EFF317
:10FC60000583002BEAD1EFF3108172B6154B1868AB
:10FC7000E0B1154C2278CAB945691D600123237093
:10FC8000C5B1AA6101B962B6002545778368984776
:10FC90002570D3E700F020F8DFE700F01BF8D9E784
:10FCA00000F016F8D3E7FFF71FFCCDE70029C5D118
:10FCB00062B638BD054B1D600029E5D1E3E700BF02
:10FCC00081A2FF1F1CA0FF1F20A0FF1F18A0FF1F65
:10FCD000704700BF704700BF704700BF054A064B22
:10FCE00010781B78C0B2DBB2984238BF4030C01ADF
:10FCF000704700BF88A2FF1F89A2FF1FF0B4384BD6
:10FD00001A7912F0300F2CD072B6997D01F0FF02F3
:10FD100000293DD062B6334F334938780D78334EE1
:10FD20001C46C0B2EDB2431C402BE17928BF002332
:10FD3000AB4202F1FF32C9B21CBFF154184612F0B7
:10FD4000FF02F0D12A4B1B68C2B23A704BB1A842F5
:10FD500036BFC5F14005401B40192728C4BF01220A
:10FD60001A701F49CA78D2B2150616D452060DD59C
:10FD70001B4B1B795B0609D51E4B1F491B680022D4
:10FD80000A7003B11A70164B3C22DA70F0BC70474F
:10FD90004022D9795A7462B6E3E70B791C06E5D59F
:10FDA000164B174E1C783378E4B2DBB29C420ED06F
:10FDB000144D01E0A3420AD00133402B28BF002399
:10FDC0000879E85CC0B2C871087D0728F2D9DBB2B7
:10FDD000034933700B79180644BF7C23CB70C5E709
:10FDE00000A0064088A2FF1F89A2FF1FCCA2FF1F10
:10FDF00084A2FF1F10A3FF1F0CA3FF1F14A3FF1F4C
:10FE00000DA3FF1F8CA2FF1F70B584B072B6194BF3
:10FE1000194D1A48702241260F2480211A702E7025
:10FE20001A460470197013781B06FCD5144B186819
:10FE300062B6144B144C984298BF00EB800001A9A5
:10FE400098BF40000A22FDF78DFD01A9204600233E
:10FE500011F8012B01333AB10A2B20F8022FF7D108
:10FE60001623237004B070BD5B00DBB2237004B0B6
:10FE700070BD00BF000002400700024006000240C3
:10FE8000080002407F9698000494FF1FFFFFFFFFC9
:10FE90002DE9F043DFF8EC808BB006460F4600F00A
:10FEA00073F898F90030013304460D4637D03046D8
:10FEB000394600F0DFF9002831D02BA3D3E9002325
:10FEC0003046394600F026FE814668BB28A3D3E9B8
:10FED00000233046394600F0FFFD00B398F90030AA
:10FEE000254ACDF82090042400200021022BCDE9E2
:10FEF0000467CDE9026700940192CDE906012CD098
:10FF0000684600F0BDF940B3089B1BB101F0AAF9A7
:10FF1000089B0360DDE906010BB0BDE8F0832046D5
:10FF200029460BB0BDE8F083134A98F900300192DE
:10FF300003210022CDE90467CDE902670091089210
:10FF40002BB90E4B4FF06042CDE90623D8E70C49A0
:10FF50000020022BCDE90601D2D101F083F9222342
:10FF60000360D1E7AFF30080EF39FAFE422E8640FE
:10FF700051302DD5104987C05C4E0100FFFFEF477F
:10FF80000000F07F1A94FF1F2DE9F04FB04F21F0D1
:10FF90000042BA4283B00C464FEAD17605460DD9ED
:10FFA000AC4FBA4225D9C1F31303034340F0EF80AD
:10FFB0000EB10020014603B0BDE8F08FA64B9A4277
:10FFC00000F2CC80A54B9A4200F2DE808AA3D3E9EE
:10FFD000002300F05DF90022A14B00F09BFD0028FA
:10FFE00000F005812846214600229D4B00F050F983
:10FFF000E1E783A3D3E9002300F08CFD002840F063
:020000021000EC
:10000000CB802846214680A3D3E9002300F064FD7D
:100010000028CED1934B284603EBC60821467CA38B
:10002000D3E9002300F0E6FAD8E9002300F030F924
:1000300000F07AFD804600F077FA77A3D3E9002339
:1000400006460F4600F0D6FA02460B4628462146E1
:1000500000F01CF972A3D3E90023CDE9000130467A
:10006000394600F0C7FA82468B4652465B46DDE9C8
:10007000000100F00BF905460C462A4623462846A7
:10008000214600F0B7FA68A3D3E9002306460F46DD
:1000900000F0B0FA66A3D3E9002300F0F7F8324687
:1000A0003B4600F0A7FA64A3D3E9002300F0F0F880
:1000B00032463B4600F09EFA61A3D3E9002300F0EC
:1000C000E5F832463B4600F095FA5FA3D3E90023FA
:1000D00000F0DEF832463B4600F08CFA02460B4652
:1000E0002846214600F0D2F806460F46284621460B
:1000F00032463B46B8F1000F56D000F07BFA32464C
:1001000004460D463B4600204FF0804100F0BEF80B
:1001100002460B462046294600F096FB02460B4657
:100120005046594600F0B2F8DDE9002300F0AEF881
:100130000B4602464A49002000F0A8F86FF47F738E
:1001400098454FDA08F57A7801EB085100224FF014
:10015000B87300F04FFA03B0BDE8F08F424B9A42FB
:100160003FF658AF414BF4002344D3E9002300F09D
:100170008DF83F4BC6F101081C44CDE90001D4E9DC
:1001800000ABC6EB080870E74FF0000875E70246C1
:100190000B4600F07DF80EE717A3D3E900231046C5
:1001A000194600F027FA06E700F024FA00228046FC
:1001B00089464FF080433046394600F067F80246E2
:1001C0000B464046494600F03FFB2A46234600F0D6
:1001D0005DF802460B460020214900F057F803B0B5
:1001E000BDE8F08F01EB085103B0BDE8F08F804609
:1001F00043E700BFAFF300809C7500883CE4377E86
:10020000EF39FAFE422E864051302DD5104987C075
:10021000FE822B654715F73F0000E0FE422EE63FC9
:10022000763C7935EF39EA3DD0A4BE726937663E37
:10023000F16BD2C541BDBB3E2CDE25AF6A56113FE6
:1002400093BDBE166CC1663F3E5555555555C53FCD
:10025000412E8640FFFFEF7F422ED63FFFFF2F3E0D
:100260000000F03F604E0100B1A2F03F804E01005F
:10027000704E010041F0004101F58010C00F704741
:100280000020704781F0004102E000BF83F000438E
:1002900030B54FEA41044FEA430594EA050F08BF21
:1002A00090EA020F1FBF54EA000C55EA020C7FEAE5
:1002B000645C7FEA655C00F0E2804FEA5454D4EB62
:1002C0005555B8BF6D420CDD2C4480EA020281EA2C
:1002D000030382EA000083EA010180EA020281EA64
:1002E0000303362D88BF30BD11F0004F4FEA0131B6
:1002F0004FF4801C4CEA113102D0404261EB4101C5
:1003000013F0004F4FEA03334CEA133302D052424A
:1003100063EB430394EA050F00F0A780A4F1010406
:10032000D5F1200E0DDB02FA0EFC22FA05F2801840
:1003300041F1000103FA0EF2801843FA05F3594126
:100340000EE0A5F120050EF1200E012A03FA0EFCA5
:1003500028BF4CF0020C43FA05F3C01851EBE371CF
:1003600001F0004507D54FF0000EDCF1000C7EEBEC
:1003700000006EEB0101B1F5801F1BD3B1F5001F2A
:100380000CD349085FEA30004FEA3C0C04F1010449
:100390004FEA445212F5800F80F09A80BCF1004F72
:1003A00008BF5FEA500C50F1000041EB045141EAF4
:1003B000050130BD5FEA4C0C404141EB010111F4F5
:1003C000801FA4F10104E9D191F0000F04BF0146A0
:1003D0000020B1FA81F308BF2033A3F10B03B3F17E
:1003E00020020CDA0C3208DD02F1140CC2F10C020E
:1003F00001FA0CF021FA02F10CE002F11402D8BF6C
:10040000C2F1200C01FA02F120FA0CFCDCBF41EA37
:100410000C019040E41AA2BF01EB0451294330BD06
:100420006FEA04041F3C1CDA0C340EDC04F11404E3
:10043000C4F1200220FA04F001FA02F340EA0300BA
:1004400021FA04F345EA030130BDC4F10C04C4F100
:10045000200220FA02F001FA04F340EA03002946E0
:1004600030BD21FA04F0294630BD94F0000F83F42A
:10047000801306BF81F480110134013D4EE77FEA0D
:10048000645C18BF7FEA655C29D094EA050F08BF59
:1004900090EA020F05D054EA000C04BF194610463A
:1004A00030BD91EA030F1EBF0021002030BD5FEA7E
:1004B000545C05D14000494128BF41F0004130BDA6
:1004C00014F580043CBF01F5801130BD01F00045FA
:1004D00045F0FE4141F470014FF0000030BD7FEA6D
:1004E000645C1ABF194610467FEA655C1CBF0B4668
:1004F000024650EA013406BF52EA033591EA030F7F
:1005000041F4002130BD00BF90F0000F04BF002176
:10051000704730B54FF4806404F132044FF00005A9
:100520004FF0000150E700BF90F0000F04BF002122
:10053000704730B54FF4806404F1320410F0004588
:1005400048BF40424FF000013EE700BF42004FEA83
:10055000E2014FEA31014FEA02701FBF12F07F4300
:1005600093F07F4F81F06051704792F0000F14BFFD
:1005700093F07F4F704730B54FF4607401F0004541
:1005800021F0004120E700BF50EA010208BF704798
:1005900030B54FF000050AE050EA010208BF70478D
:1005A00030B511F0004502D5404261EB41014FF4F6
:1005B000806404F132045FEA915C3FF4DCAE4FF0FA
:1005C00003025FEADC0C18BF03325FEADC0C18BFE1
:1005D000033202EBDC02C2F1200300FA03FC20FA32
:1005E00002F001FA03FE40EA0E0021FA02F114447F
:1005F000C1E600BF70B54FF0FF0C4CF4E06C1CEA94
:1006000011541DBF1CEA135594EA0C0F95EA0C0F08
:1006100000F0DEF82C4481EA030621EA4C5123EA7B
:100620004C5350EA013518BF52EA033541F48011AA
:1006300043F4801338D0A0FB02CE4FF00005E1FB5D
:1006400002E506F00042E0FB03E54FF00006E1FBA7
:1006500003569CF0000F18BF4EF0010EA4F1FF04EA
:10066000B6F5007F64F5407404D25FEA4E0E6D412A
:1006700046EB060642EAC62141EA55514FEAC5203B
:1006800040EA5E504FEACE2EB4F1FD0C88BFBCF5B7
:10069000E06F1ED8BEF1004F08BF5FEA500E50F168
:1006A000000041EB045170BD06F0004646EA01012E
:1006B00040EA020081EA0301B4EB5C04C2BFD4EB60
:1006C0000C0541EA045170BD41F480114FF0000E59
:1006D000013C00F3AB8014F1360FDEBF002001F0C7
:1006E000004170BDC4F10004203C35DA0C341BDC41
:1006F00004F11404C4F1200500FA05F320FA04F013
:1007000001FA05F240EA020001F0004221F0004146
:1007100010EBD37021FA04F642EB06015EEA430EB9
:1007200008BF20EAD37070BDC4F10C04C4F12005E9
:1007300000FA04F320FA05F001FA04F240EA02009C
:1007400001F0004110EBD37041F100015EEA430E6D
:1007500008BF20EAD37070BDC4F1200500FA05F28D
:100760004EEA020E20FA04F301FA05F243EA02030C
:1007700021FA04F001F0004121FA04F220EA02001B
:1007800000EBD3705EEA430E08BF20EAD37070BD61
:1007900094F0000F0FD101F00046400041EB010141
:1007A00011F4801F08BF013CF7D041EA060195F023
:1007B000000F18BF704703F00046520043EB0303DD
:1007C00013F4801F08BF013DF7D043EA06037047CA
:1007D00094EA0C0F0CEA135518BF95EA0C0F0CD0D5
:1007E00050EA410618BF52EA4306D1D181EA03011B
:1007F00001F000414FF0000070BD50EA410606BF15
:100800001046194652EA430619D094EA0C0F02D159
:1008100050EA013613D195EA0C0F05D152EA03369E
:100820001CBF104619460AD181EA030101F00041BC
:1008300041F0FE4141F470014FF0000070BD41F005
:10084000FE4141F4780170BD70B54FF0FF0C4CF4DF
:10085000E06C1CEA11541DBF1CEA135594EA0C0FFE
:1008600095EA0C0F00F0A7F8A4EB050481EA030E4B
:1008700052EA03354FEA013100F088804FEA033332
:100880004FF0805545EA131343EA12634FEA022200
:1008900045EA111545EA10654FEA00260EF00041C1
:1008A0009D4208BF964244F1FD0404F5407402D213
:1008B0005B084FEA3202B61A65EB03055B084FEAA4
:1008C00032024FF480104FF4002CB6EB020E75EBA1
:1008D000030E22BFB61A754640EA0C005B084FEAC9
:1008E0003202B6EB020E75EB030E22BFB61A754646
:1008F00040EA5C005B084FEA3202B6EB020E75EB91
:10090000030E22BFB61A754640EA9C005B084FEA08
:100910003202B6EB020E75EB030E22BFB61A754615
:1009200040EADC0055EA060E18D04FEA051545EA04
:1009300016754FEA06164FEAC30343EA52734FEAAD
:10094000C2025FEA1C1CC0D111F4801F0BD141EA26
:1009500000014FF000004FF0004CB6E711F4801F8B
:1009600004BF01430020B4F1FD0C88BFBCF5E06F6B
:100970003FF6AFAEB5EB030C04BFB6EB020C5FEA7B
:10098000500C50F1000041EB045170BD0EF0004ED0
:100990004EEA113114EB5C04C2BFD4EB0C0541EA02
:1009A000045170BD41F480114FF0000E013C90E6FF
:1009B00045EA060E8DE60CEA135594EA0C0F08BFC3
:1009C00095EA0C0F3FF43BAF94EA0C0F0AD150EAC2
:1009D00001347FF434AF95EA0C0F7FF425AF104655
:1009E00019462CE795EA0C0F06D152EA03353FF47D
:1009F000FDAE1046194622E750EA410618BF52EAFA
:100A000043067FF4C5AE50EA41047FF40DAF52EACD
:100A100043057FF4EBAE12E74FF0FF3C06E000BF6A
:100A20004FF0010C02E000BF4FF0010C4DF804CD77
:100A30004FEA410C7FEA6C5C4FEA430C18BF7FEA37
:100A40006C5C1BD001B050EA410C0CBF52EA430C65
:100A500091EA030F02BF90EA020F0020704710F1E5
:100A6000000F91EA030F58BF994208BF90422CBF74
:100A7000D8176FEAE37040F0010070474FEA410C6D
:100A80007FEA6C5C02D150EA013C07D14FEA430C8B
:100A90007FEA6C5CD6D152EA033CD3D05DF8040BFC
:100AA000704700BF8446104662468C46194663462E
:100AB00000E000BF01B5FFF7B7FF002848BF10F105
:100AC000000F01BD4DF808EDFFF7F4FF0CBF01204A
:100AD00000205DF808FB00BF4DF808EDFFF7EAFFC6
:100AE00034BF012000205DF808FB00BF4DF808ED81
:100AF000FFF7E0FF94BF012000205DF808FB00BF76
:100B00004DF808EDFFF7CEFF94BF012000205DF8FF
:100B100008FB00BF4DF808EDFFF7C4FF34BF01200C
:100B200000205DF808FB00BF4FEA410212F50012F9
:100B300015D211D56FF47873B3EB625212D94FEA24
:100B4000C12343F0004343EA505311F0004F23FA0E
:100B500002F018BF404270474FF00000704750EA63
:100B6000013005D111F0004008BF6FF00040704720
:100B70004FF00000704700BF4FEA4102B2F1E0437E
:100B800024BFB3F5001CDCF1FE5C0DD901F0004C74
:100B90004FEAC0024CEA5070B2F1004F40EB8300C4
:100BA00008BF20F00100704711F0804F21D113F1F0
:100BB0003872BCBF01F00040704741F480114FEA29
:100BC0005252C2F11802C2F1200C10FA0CF320FAB2
:100BD00002F018BF40F001004FEAC1234FEAD323CF
:100BE00003FA0CFC40EA0C0023FA02F34FEA430339
:100BF000CCE77FEA625307D150EA01331EBF4FF0C2
:100C0000FE4040F44000704701F0004040F0FE40DC
:100C100040F40000704700BF80F0004002E000BFD9
:100C200081F0004142001FBF5FEA410392EA030FD7
:100C30007FEA226C7FEA236C6AD04FEA1262D2EB21
:100C40001363C1BFD218414048404140B8BF5B4226
:100C5000192B88BF704710F0004F40F4000020F0BF
:100C60007F4018BF404211F0004F41F4000121F0D5
:100C70007F4118BF494292EA030F3FD0A2F101021F
:100C800041FA03FC10EB0C00C3F1200301FA03F15D
:100C900000F0004302D5494260EB4000B0F5000F80
:100CA00013D3B0F1807F06D340084FEA310102F13F
:100CB0000102FE2A51D2B1F1004F40EBC25008BFF1
:100CC00020F0010040EA03007047490040EB0000BB
:100CD00010F4000FA2F10102EDD1B0FA80FCACF1EA
:100CE000080CB2EB0C0200FA0CF0AABF00EBC250E9
:100CF00052421843BCBFD0401843704792F0000FD7
:100D000081F4000106BF80F400000132013BB5E729
:100D10004FEA41037FEA226C18BF7FEA236C21D09F
:100D200092EA030F04D092F0000F08BF0846704704
:100D300090EA010F1CBF0020704712F07F4F04D1D2
:100D4000400028BF40F00040704712F100723CBFE5
:100D500000F50000704700F0004343F0FE4040F40F
:100D6000000070477FEA226216BF08467FEA2363CD
:100D70000146420206BF5FEA412390EA010F40F4B8
:100D8000800070474FF0000304E000BF10F0004304
:100D900048BF40425FEA000C08BF704743F09643EB
:100DA00001464FF000001CE050EA010208BF704706
:100DB0004FF000030AE000BF50EA010208BF70478D
:100DC00011F0004302D5404261EB41015FEA010CA2
:100DD00002BF84460146002043F0B64308BFA3F19A
:100DE0008053A3F50003BCFA8CF2083AA3EBC2537C
:100DF00010DB01FA02FC634400FA02FCC2F120029B
:100E0000BCF1004F20FA02F243EB020008BF20F0D1
:100E10000100704702F1200201FA02FCC2F1200237
:100E200050EA4C0021FA02F243EB020008BF20EA2C
:100E3000DC7070474FF0FF0C1CEAD0521EBF1CEA5A
:100E4000D15392EA0C0F93EA0C0F6FD01A4480EA48
:100E5000010C400218BF5FEA41211ED04FF0006331
:100E600043EA501043EA5111A0FB01310CF000405D
:100E7000B1F5000F3EBF490041EAD3715B0040EA83
:100E8000010062F17F02FD2A1DD8B3F1004F40EB53
:100E9000C25008BF20F00100704790F0000F0CF026
:100EA000004C08BF49024CEA502040EA51207F3AEA
:100EB000C2BFD2F1FF0340EAC250704740F40000C5
:100EC0004FF00003013A5DDC12F1190FDCBF00F0B6
:100ED00000407047C2F10002410021FA02F1C2F164
:100EE000200200FA02FC5FEA310040F1000053EA00
:100EF0004C0308BF20EADC70704792F0000F00F04E
:100F0000004C02BF400010F4000F013AF9D040EA53
:100F10000C0093F0000F01F0004C02BF490011F4E7
:100F2000000F013BF9D041EA0C018FE70CEAD153E5
:100F300092EA0C0F18BF93EA0C0F0AD030F0004C65
:100F400018BF31F0004CD8D180EA010000F0004019
:100F5000704790F0000F17BF90F0004F084691F0D7
:100F6000000F91F0004F14D092EA0C0F01D1420211
:100F70000FD193EA0C0F03D14B0218BF084608D1DA
:100F800080EA010000F0004040F0FE4040F4000024
:100F9000704740F0FE4040F4400070474FF0FF0CB7
:100FA0001CEAD0521EBF1CEAD15392EA0C0F93EAFE
:100FB0000C0F69D0A2EB030280EA010C49024FEA50
:100FC000402037D04FF0805343EA111143EA101309
:100FD0000CF000408B4238BF5B0042F17D024FF4C1
:100FE000000C8B4224BF5B1A40EA0C00B3EB510F9C
:100FF00024BFA3EB510340EA5C00B3EB910F24BF85
:10100000A3EB910340EA9C00B3EBD10F24BFA3EB09
:10101000D10340EADC001B0118BF5FEA1C1CE0D1D1
:10102000FD2A3FF650AF8B4240EBC25008BF20F084
:10103000010070470CF0004C4CEA50207F32C2BFD8
:10104000D2F1FF0340EAC250704740F400004FF075
:101050000003013A37E792F0000F00F0004C02BFA6
:10106000400010F4000F013AF9D040EA0C0093F070
:10107000000F01F0004C02BF490011F4000F013BCA
:10108000F9D041EA0C0195E70CEAD15392EA0C0F32
:1010900008D142027FF47DAF93EA0C0F7FF470AF6A
:1010A000084676E793EA0C0F04D14B023FF44CAFAD
:1010B00008466EE730F0004C18BF31F0004CCAD142
:1010C00030F000427FF45CAF31F000437FF43CAF7E
:1010D0005FE700BF4FF0FF3C06E000BF4FF0010CA0
:1010E00002E000BF4FF0010C4DF804CD4FEA400282
:1010F0004FEA41037FEA226C18BF7FEA236C11D0CC
:1011000001B052EA530C18BF90EA010F58BFB2EB7E
:10111000030088BFC81738BF6FEAE17018BF40F0FE
:10112000010070477FEA226C02D15FEA402C05D1B2
:101130007FEA236CE4D15FEA412CE1D05DF8040B37
:10114000704700BF844608466146FFE70FB5FFF7CA
:10115000C9FF002848BF10F1000F0FBD4DF808ED82
:10116000FFF7F4FF0CBF012000205DF808FB00BF73
:101170004DF808EDFFF7EAFF34BF012000205DF8CD
:1011800008FB00BF4DF808EDFFF7E0FF94BF01201A
:1011900000205DF808FB00BF4DF808EDFFF7D2FF17
:1011A00094BF012000205DF808FB00BF4DF808ED5A
:1011B000FFF7C8FF34BF012000205DF808FB00BF27
:1011C0004FEA4002B2F1FE4F0FD34FF09E03B3EB54
:1011D00012620DD94FEA002343F0004310F0004F94
:1011E00023FA02F018BF404270474FF000007047EA
:1011F00012F1610F01D1420205D110F0004008BF89
:101200006FF0004070474FF00000704742000ED270
:10121000B2F1FE4F0BD34FF09E03B3EB126209D431
:101220004FEA002343F0004323FA02F070474FF0E7
:101230000000704712F1610F01D1420202D14FF05C
:10124000FF3070474FF00000704700BF0B4601466B
:10125000184600F001B800BF13460A4601460220B6
:1012600000F0C0BE014B1868704700BF4898FF1FD0
:1012700070B50F4E0F4D761BB61018BF002405D069
:10128000013455F8043B9847A642F9D10A4E0B4D5C
:10129000761B03F0FFFDB61018BF002406D0013402
:1012A00055F8043B9847A642F9D170BD70BD00BF08
:1012B000A04E0100A04E0100B44E0100A04E01005E
:1012C000024B0146186800F00BB800BF4898FF1F9A
:1012D000024B0146186800F049BF00BF4898FF1F45
:1012E0002DE9F04F01F10B05162D83B0064640F2B3
:1012F0009F8035F0070500F1BF80A94200F2BC8055
:1013000000F058FBB5F5FC7FC0F09C826B0A00F042
:10131000BA80042B00F28381A80900F1390E4FEA4C
:101320004E033830C44F07EB8303A3F108015C6818
:10133000A14207D1ACE0002A80F2AC80E468A1426F
:1013400000F0A680636823F003035A1B0F2AF2DD26
:10135000B9493C6901F1080E744500F0B381636836
:1013600023F003035A1B0F2A00F39981002AC1F8C6
:1013700014E0C1F810E080F29E80B3F5007F80F0A9
:101380006781DB0803F1010C01229B1002FA03F3D1
:101390004A6851F83C80C4F8088001EBCC091A4334
:1013A000A9F10803E3604A6041F83C40C8F80C40EA
:1013B000831001249C40944200F28A80144206D19A
:1013C00020F003006400144200F10400FAD007EB9F
:1013D000C009CC468046DCF80C108C4507D173E17F
:1013E000002A80F28181C9688C4500F06D814B68CC
:1013F00023F003035A1B0F2AF2DD0C46D1F80CC070
:1014000054F8088F4B1945F001054D6042F0010179
:10141000C8F80CC03046CCF808807B613B61C3F84B
:101420000CE0C3F808E059609A5000F0C5FA1FE0DC
:10143000102921D800F0BEFA1025062302207E4F85
:1014400007EB8303A3F108025C68944200F0458136
:101450006368E168A56823F00303234430465A68B3
:10146000E96042F001028D605A6000F0A5FA08348C
:10147000204603B0BDE8F08F00240C2320463360E3
:1014800003B0BDE8F08F80234FF0400E3F2049E7C6
:1014900070465DE72344E1685A68A56842F001029E
:1014A000E96030468D605A6000F086FA08342046C4
:1014B00003B0BDE8F08F234430465A6842F0010281
:1014C0005A6000F079FA0834204603B0BDE8F08F86
:1014D000BC68636823F00308A84504D3C5EB080380
:1014E0000F2B00F38C80554BDFF860911A68D9F808
:1014F000003001332A4404EB080A00F0608102F551
:1015000080520F3222F47F6222F00F0211463046E1
:10151000019200F04BFCB0F1FF3F8346019A00F0CE
:101520005881824500F2FC80454B1968DA45114428
:10153000196000F05381D9F80000DFF810E10130A4
:101540001BBFCAEB0B0A5144CEF800B019601BF068
:10155000070100F01781C1F10800C1F580518344F3
:1015600008315A44C2F30B02C2EB01094946304626
:10157000019300F01BFC431C019B00F03F81CBEB6F
:1015800000024A4442F001021968C7F808B0494411
:10159000BC42CBF804201960DFF8A49016D0B8F153
:1015A0000F0F40F2FD806268A8F10C0323F00703DF
:1015B000E01802F001024FF0050E1A430F2B626093
:1015C000C0F804E0C0F808E000F21C811D4BBC68C4
:1015D0001A68914288BF19601B4B1A689142626871
:1015E00088BF196022F003029542A2EB050301D8DF
:1015F0000F2B04DC304600F0DFF9002438E76219D5
:1016000043F0010345F0010565603046BA60536060
:1016100000F0D2F90834204603B0BDE8F08F142B57
:1016200071D9542B00F2A480280B00F16F0E4FEA01
:101630004E036E3076E600BF4C98FF1F20A3FF1FBD
:1016400024A3FF1F1CA3FF1F18A3FF1F589CFF1FED
:101650005A0A042A5ED9142A00F2B38002F15C010E
:1016600049005B3207EB810C57F82110DFF8DC8171
:10167000ACF1080C8C4500F088804A6822F0030227
:10168000934202D289688C45F7D1D1F80CC07A68B0
:10169000C4F80CC0A160CCF80840CC6088E663199F
:1016A00042F0010745F00105656030464B610B6172
:1016B000C3F80CE0C3F808E05F609A50083400F00B
:1016C0007BF9D5E64A6873E608F1010818F0030FC4
:1016D0000CF1080C7FF47FAE30E0DC68A34208BF59
:1016E00002303FF435AEB3E60B440C465A68C96885
:1016F00054F8085F42F001025A603046E9608D609C
:1017000000F05AF9B4E603F15C0E03F15B004FEA16
:101710004E0307E69A0902F1390149003832A1E780
:10172000BC424A4B3FF400AF9C68626822F003025F
:101730005AE759F80839994540F0828010F0030FB4
:1017400000F1FF30F5D17B6823EA04037B6064007D
:101750009C423FF6BDAE002C3FF4BAAE1C42404660
:101760007FF435AE64001C4200F10400FAD02EE68E
:10177000B3F5AA7F18D8E80B00F1780E4FEA4E03B4
:101780007730CFE54FF48051EBE60121D8F80430F3
:10179000921001FA02F21A43C8F80420614677E772
:1017A0000123CBF8043025E740F25452934220D86D
:1017B000A80C00F17D0E4FEA4E037C30B2E51032EA
:1017C000A4E6542A26D81A0B02F16F0149006E32A2
:1017D00048E7BC68626822F0030205E7CAF30B0021
:1017E00000287FF4A8AE4244BB6842F001025A6070
:1017F000ECE6FE234FF07F0E7E2093E501224FF0B2
:101800000009C1E604F10801304600F0AFFCD9F848
:101810000010DBE6B2F5AA7F05D8DA0B02F17801F9
:10182000490077321EE740F254518A4205D89A0C9B
:1018300002F17D0149007C3214E7FE217E2211E78E
:101840007B6884E7E808431C5B00F8E54C98FF1FC1
:101850008842F0B50DD98B1898420AD28118002A17
:1018600051D09A1A13F8014D01F8014D9342F9D164
:10187000F0BD0F2A48D941EA00039B0746D100F189
:10188000100401F11003154653F8106C44F8106C65
:1018900053F80C6C44F80C6C53F8086C44F8086C62
:1018A000103D53F8046C44F8046C0F2D03F1100341
:1018B00004F11004E8D8A2F1100323F00F0302F0A2
:1018C0000F0E1033BEF1030F1944034421D91E1F1C
:1018D0000D467446043C55F8047B46F8047F032CFF
:1018E000F8D8AEF1040424F0030404342344214462
:1018F00002F0030262B1013B0A4411F8014B03F804
:10190000014F8A42F9D1F0BD0346F3E70346F2E7FF
:10191000F0BD7246EEE700BF70B4840746D0541E97
:10192000002A41D0CDB2034602E0621EE4B3144661
:1019300003F8015B9A07F8D1032C2ED9CDB245EA02
:1019400005250F2C45EA054519D903F11002264655
:10195000103E0F2E42F8105C42F80C5C42F8085C16
:1019600042F8045C02F11002F2D8A4F1100222F055
:101970000F0204F00F041032032C13440DD91E463D
:101980002246043A032A46F8045BFAD8221F22F0C2
:1019900003020432134404F003042CB1C9B21C4402
:1019A00003F8011BA342FBD170BC704714460346E9
:1019B000C2E700BF704700BF704700BF024B0A4636
:1019C0000146186800F002B84898FF1F2DE9F04F53
:1019D000174683B0002900F0C1800E46814607F10A
:1019E0000B05FFF7E7FF56F804EC162D2EF0030465
:1019F000A6F1080840D810221546AF4241D89442BB
:101A000075DAC94B996808EB04008842416800F018
:101A1000D98021F0010303445B68DB077DD51EF00C
:101A2000010F35D039464846FFF75AFC0746E0B16A
:101A300056F8043C23F001034344A0F108029A4203
:101A400000F04481221F242A00F23181132A00F27F
:101A500004810346324611681960516859609268E2
:101A60009A603146484600F081FB4846FFF7A4FFE4
:101A7000384603B0BDE8F08F25F00705002D2A4653
:101A8000BBDA0C230020C9F8003003B0BDE8F08FAA
:101A900056F8083CC3EB080ADAF8043023F0030CCC
:101AA00004EB0C039342BDDB5746DAF80C1057F8F1
:101AB000080F221F242AC160886000F21781132AB0
:101AC00040F212813168CAF808107168CAF80C1027
:101AD0001B2A00F22B8108360AF1100231681160CE
:101AE00071685160B16891603E461C46D046631BE8
:101AF0000F2B1DD8D8F8043003F0010323434444CE
:101B0000C8F80430636843F0010363604846FFF798
:101B100053FF304603B0BDE8F08F21F003012144AC
:101B2000914221DBC36882680C46D3609A60DEE78D
:101B3000D8F8042008EB050102F00102154343F038
:101B400001020B44C8F804504A605A6842F001028E
:101B500008315A60484600F009FBD7E7114603B048
:101B6000BDE8F04FFFF7BCBB1EF0010F7FF45AAF8A
:101B700056F8083CC3EB080ADAF8043023F0030CEB
:101B800001EB0C0E96458BDBC36882685746D36029
:101B90009A6057F8081FDAF80C30CB60221F242A0D
:101BA000996000F29980132A62D93368CAF8083024
:101BB0007368CAF80C301B2A00F2A08008360AF1BC
:101BC000100356E021F0030BA34405F110008345F8
:101BD00059DA1EF0010F7FF425AF56F8081CC1EB4F
:101BE000080ADAF8041021F0030CE34458453FF7E3
:101BF00057AF5746DAF80C1057F8080F221F242A5F
:101C0000C160886000F2B480132A40F2A580316878
